:020000040800F2
:1000000000000120DD380008E1160008E3160008B2
:10001000E5160008E7160008E916000800000000D1
:10002000000000000000000000000000EB160008C7
:10003000ED16000800000000EF160008F116000899
:100040002D390008000000002D3900082D39000866
:100050002D3900082D3900080000000000000000C4
:100060002D3900082D3900082D3900080000000046
:10007000000000002D390008000000000000000012
:100080002D3900082D3900082D3900082D390008B8
:100090002D3900082D3900082D3900082D390008A8
:1000A0002D3900082D3900082D3900082D39000898
:1000B0002D3900082D3900082D3900082D39000888
:1000C0002D3900082D3900082D3900082D39000878
:1000D0002D3900082D3900082D390008F5160008C3
:1000E0002D390008011700080D1700082D390008E8
:1000F00019170008251700082D3900082D390008A8
:100100002D3900082D3900082D3900083117000855
:100110002D3900082D3900082D3900082D39000827
:100120002D3900082D3900083D170008491700082F
:100130002D3900082D3900082D3900085517000801
:100140002D3900082D3900082D3900082D390008F7
:100150002D3900082D3900082D3900082D390008E7
:100160002D3900082D3900082D3900082D390008D7
:100170002D3900082D390008611700086D17000897
:100180002D3900082D3900082D3900082D390008B7
:100190002D390008791700082D3900082D3900087D
:1001A0002D3900082D3900082D3900088517000861
:1001B0002D3900082D3900082D3900082D39000887
:1001C00000000000000000002D3900082D39000853
:1001D0002D3900082D3900082D3900082D39000867
:1001E0002D3900082D3900082D3900082D39000857
:1001F0002D3900082D390008000000000000000023
:100200002D3900082D3900082D3900082D39000836
:100210002D3900082D3900082D3900082D39000826
:100220002D3900082D3900082D3900082D39000816
:100230002D3900082D3900082D3900082D39000806
:100240002D3900082D3900082D3900082D390008F6
:100250002D3900082D3900082D39000891170008A4
:100260002D3900082D3900082D3900082D390008D6
:100270002D3900082D3900082D3900082D390008C6
:100280002D3900082D3900082D3900082D390008B6
:100290002D390008000000000000000000000000F0
:1002A0002D3900082D3900082D3900082D39000896
:1002B00010B5054C237833B9044B13B10448AFF3A0
:1002C00000800123237010BDF8030024000000000B
:1002D0004CC7000808B5034B1BB103490348AFF3F3
:1002E000008008BD00000000FC0300244CC700088B
:1002F000034613F8012B002AFBD1181A0138704766
:1003000053B94AB9002908BF00281CBF4FF0FF317C
:100310004FF0FF3000F088B9ADF1080C6DE904CE64
:1003200000F006F8DDF804E0DDE9022304B07047D0
:100330002DE9F047089D8E4604468846002B4AD199
:100340008A42174662D9B2FA82F64EB1C6F120034C
:1003500001FA06F820FA03F3B74043EA0808B4406C
:100360004FEA174E1FFA87FCB8FBFEF1230C0EFB79
:10037000118843EA084301FB0CF29A4209D9FB18A1
:1003800001F1FF3080F0EA809A4240F2E7800239C2
:100390003B449A1AA3B2B2FBFEF00EFB102243EAD2
:1003A000024300FB0CFC9C4509D9FB1800F1FF320D
:1003B00080F0D6809C4540F2D3803B44023840EA2E
:1003C0000140A3EB0C0300211DB1F3400022C5E95D
:1003D0000032BDE8F0878B4205D90DB1C5E90001B7
:1003E00000210846F5E7B3FA83F1002946D17345A9
:1003F00002D3824200F20581841A6EEB03020120CF
:100400009046002DE5D0C5E90048E2E7002A00F05B
:100410009080B2FA82F6002E40F0A4808A1A030C73
:100420004FEA174E80B2BCB20121B2FBFEFC0EFBBC
:100430001C2243EA024304FB0CF29A4207D9FB1840
:100440000CF1FF3802D29A4200F2E080C4469B1AB7
:10045000B3FBFEF20EFB123340EA034302FB04F44B
:100460009C4207D9FB1802F1FF3002D29C4200F2F5
:10047000CA8002461B1B42EA0C40A5E7C1F12006D8
:100480008B4022FA06F71F430EFA01F420FA06F316
:100490002EFA06FE4FEA1749234300FA01F81FFA25
:1004A00087FCBEFBF9F01C0C09FB10EE44EA0E447D
:1004B00000FB0CFEA64502FA01F209D93C1900F135
:1004C000FF3A80F09C80A64540F2998002383C4477
:1004D000A4EB0E041FFA83FEB4FBF9F309FB1344EB
:1004E0004EEA044403FB0CFCA44508D93C1903F173
:1004F000FF3E80F08280A4457FD9023B3C4443EA22
:100500000040A4EB0C04A0FB02EC64457346E146FA
:1005100062D35FD05DB1B8EB030264EB090404FA67
:1005200006F622FA01F31E43CC40C5E9006400211F
:100530004FE7B1FBF2FC010C41EA0E4180B240EA08
:1005400001423B4638463C46B846BE462026B1FBF3
:10055000F7F1A2EB080241EA0C4166E7014618E711
:1005600010462CE7C6F120022EFA02F3B740B14044
:1005700020FA02F24FEA174E0A43B3FBFEF8BCB270
:100580000EFB1833110C41EA034108FB04F9B0409B
:1005900089454FEA104380B23ED9791808F1FF3CF3
:1005A00001D289451FD8A1EB0901B1FBFEF909FB76
:1005B00004F80EFB191192B242EA0142424529D2D7
:1005C000BA1809F1FF31C4D24245C2D2A9F10201E1
:1005D0003A44BEE7F0459DD2BEEB02036CEB070C3C
:1005E0000138E14696E7A7EB09094944A8F1020C56
:1005F000B1FBFEF909FB04F8DBE773467FE75046E1
:1006000066E70846FDE63B44023A33E7ACF1020CEC
:100610003B441CE749469CE7A1EB0901C446B1FBFA
:10062000FEF909FB04F8C4E7704700BF0E4B1B78C6
:1006300010B5044633B103F04FFC0C4902460020CC
:1006400003F0FAFB0A4B84F001041C70094B1B7881
:10065000022B96BF084A0122D25C4FF48063B3FBA1
:10066000F2F3064A136010BD1C04002488C9000878
:100670001D04002414040024E6DA000818040024F1
:10068000F8B500250C4E04460C4F2A464FF48071F5
:1006900030463D6004F086FC80216208304604F05C
:1006A00081FC04F001024021304604F07BFC044B45
:1006B0003D601C70F8BD00BF0004025818040024FF
:1006C00014040024014B1868704700BF180400246C
:1006D000F8B52E4F0D463C688C4208D203F0FCFB67
:1006E0002B4902460020BDE8F84003F0A5BB0122DB
:1006F000284B294E1B783270284A012B12780CBFE8
:100700004FF400634FF48063032A0AD8DFE802F055
:100710002D1D0E021B1B2249AA0001EB83010CF0C8
:1007200007F8641B00233C603370F8BDA3EB44035F
:100730001B4A013302EB83020023AB42F1D052F893
:10074000331040F823100133F7E7154AA3EB840375
:1007500002EB830300EB8502904203F11003E0D02B
:1007600053F8041C40F8041BF6E70D4AA3EBC4033E
:1007700002EB830300EB8502904203F12003D0D00B
:1007800053F8041C40F8041BF6E700BF18040024CB
:10079000C7C900081D0400241C04002414040024FC
:1007A000200400240020FFF741BF0120FFF73EBFD7
:1007B00037B5044603F090FB0546204608F057FD88
:1007C000D4F8841094F88920034691F8541000203E
:1007D000CDE900212A46024903F02EFB03B030BDCB
:1007E00014CA00080421014809F0F2B9482800247D
:1007F00073B500220C4640484FF4806104F0D2FBF0
:100800003E4808F0CDFB3E4803F0AEFD3B4808F003
:100810005DF904213B4809F0DBF9B4F5FA7F33D0E8
:100820000FDC7D2C34D0FA2C30D003F055FB23465E
:10083000042402463449002003F0FEFA204602B0A8
:1008400070BDB4F57A7FF0D10320FFF719FF2D4872
:1008500000252B4C036804215D6209F055FA2046FF
:1008600003F02EFC254808F021F894F85430012BB1
:1008700010D003F031FB94F8543002462349284647
:10088000032403F0D9FAD9E70220DEE70120DCE7F0
:100890000020DAE7204603F01AFF012808D020469E
:1008A00003F062FD204603F00BFC08B100F0DCFB16
:1008B0004FF400521649114808F084FA044698B1E2
:1008C00003F00AFB05460D4808F0D1FC06460C482B
:1008D00003F000FF23462A460E490224CDE90060BA
:1008E000002003F0A9FAA9E701224FF48061024831
:1008F00004F058FBA2E700BF00000258B82700240C
:10090000E42500244828002461CA000895CA00088C
:1009100020040024CBCA000810B50A4C00224FF472
:100920008061094804F03EFB204601224FF400712B
:1009300004F038FB204601220221BDE8104004F0FB
:1009400031BB00BF0004025800000258C068B0FA72
:1009500080F0400940007047D0E9032310B59A4267
:10096000044613D0828AD0E9003000FB02300BF03D
:10097000DFFE636822690020013393FBF2F102FB82
:1009800011336360E3680133E36010BD0120FCE7CD
:1009900010B504460846E3689BB1A28A2368A168A3
:1009A00001FB02310BF0C4FEA36822690020013371
:1009B00093FBF2F102FB1133A360E368013BE360B8
:1009C00010BD0220FCE708B503460846DA6842B1CC
:1009D0009A8A99681B6801FB02310BF0A9FE00207E
:1009E00008BD0220FCE703460020C3E90100D860EF
:1009F0007047000007EE901A9FED167AF8EEE77A3E
:100A000070B567EE877A144D144E2846FDEEE77AEE
:100A100017EE903A03F5004383F310031A12737034
:100A2000327008F021FC0446D5F8800003F04FFE38
:100A3000012C0CD1012808D102223146284608F0A9
:100A4000DBF8041E18BF01246400204670BD012499
:100A5000FBE700BF17B7514198260024202400244B
:100A60000B4A08B5D2F8FC3043F08073C2F8FC3072
:100A70000022084B5A601A6842F001021A6006F020
:100A80001BFF054BB0FBF3F0044B186008BD00BF23
:100A900000ED00E0001000E040420F00242400249C
:100AA0001F4B07B5D3F83821272042F01002C3F8B6
:100AB00038210022D3F8383111460193019B03F00D
:100AC00043FA272003F072FA00222920114603F08E
:100AD0003BFA292003F06AFA00222A20114603F08B
:100AE00033FA2A2003F062FA00222C20114603F088
:100AF0002BFA2C2003F05AFA00222D20114603F085
:100B000023FA2D2003F052FA00228720114603F029
:100B10001BFA872003B05DF804EB03F047BA00BF6F
:100B2000004402582DE9F04714228AB00021DFF872
:100B300040A10DEB0200DFF83C910BF0C5FD494BE5
:100B4000494E5046D3F8402147F2C33100244FF0BC
:100B5000030842F0040208270125C3F84021D3F816
:100B600040210092009AD3F8402142F00102C3F8DC
:100B70004021D3F840210192019AD3F8402142F05C
:100B80000202C3F84021D3F840210292029AD3F81E
:100B9000402142F48042C3F84021D3F8402103921F
:100BA000039AD3F8402142F48052C3F84021002236
:100BB000D3F840310493049B04F0F4F94846002232
:100BC000022104F0EFF9002230464FF4806104F076
:100BD000E9F905A925480794CDE9058404F0D4F87E
:100BE000042305A930460794CDE9053404F0CCF878
:100BF0004FF4881305A930460794CDE9057304F036
:100C0000C3F847F2C33305A95046CDE90535CDE910
:100C1000074404F0B9F8022305A94846CDE9053593
:100C2000CDE9074404F0B0F84FF48063304606F590
:100C3000405605A9CDE90535CDE9074404F0A4F8EF
:100C400005A930460794CDE9058404F09DF805A96F
:100C500030460795CDE9057404F096F80AB0BDE872
:100C6000F08700BF004402580000025800080258F4
:100C7000000402580038025808B51248124A134BB3
:100C8000C0E9002300230122C0E90433C0E9023295
:100C9000C0E90633036204F079FB08B100F0E4F91F
:100CA0000021084805F037FC08B100F0DDF900210B
:100CB000044805F056FC18B1BDE8084000F0D4B96E
:100CC00008BD00BF1825002400580040FF63E00065
:100CD00070B5A8B006461422002102A80BF0F4FC5F
:100CE0008422002107A80BF0EFFC3268454B9A42A2
:100CF00040F086804FF4806307A8079307F0C4F89C
:100D000008B100F0B1F9404C4FF4406100253F4874
:100D1000D4F8403143F00203C4F84031D4F84031F4
:100D20000093009B1223CDE90213042302A906932A
:100D3000CDE9045504F028F8D4F84831344843F498
:100D40008003C4F84831D4F84831324C0193019BF8
:100D5000452325616563C4E900034FF40023204661
:100D6000C4E905350123C4E90255C4E90755C4E9BE
:100D70000933C4E90B5503F0A3F908B100F074F985
:100D8000F4634FF080712348E66503F0A5FC08B1D9
:100D900000F06AF9204C4623204A2046C4E900238B
:100DA00000234FF48062C4E90232082223626363A5
:100DB000C4E904230122C4E90633C4E90922C4E9D1
:100DC0000B3303F07DF908B100F04EF9B4634FF036
:100DD00080711148E66503F07FFC08B100F044F92A
:100DE00000224E20114603F0AFF84E2003F0DEF84B
:100DF00000224F20114603F0A7F84F2003F0D6F849
:100E000028B070BD00580040004402580004025849
:100E100050130240A024002428240024D0120240B1
:100E200038B5044607480D4608F01EFA012806D1D9
:100E30002A4621460348BDE8384007F05FBE02203D
:100E400038BD00BF2827002410B5044688B10068CB
:100E500078B1A2880021023292000BF035FC2368A1
:100E600000224FF0FF311A60A3882268013342F854
:100E7000231010BDF0B5F8B1F1B10B784C78828831
:100E80001C44944218DC8A784E791F2A0F7991F815
:100E900003C028BF1F2242F0E0029C4201DC002078
:100EA000F0BD0568013305EB830105F823204E7082
:100EB0008F7081F803C0F0E70120F1E730B181883D
:100EC00000680231890089B2FFF7AABF012070478C
:100ED00000B5B1B09C22002109A80BF0F5FB20223F
:100EE000002101A80BF0F0FB012006F0FFF808B18B
:100EF00072B6FEE701224FF4A02332212690CDE9FD
:100F000009230223CDE91B0009A81493CDE912336C
:100F1000CDE91512CDE91733CDE9193306F0B2FA50
:100F200008B172B6FEE703233F2208210390402058
:100F3000CDE901230423CDE904134FF48063372165
:100F4000CDE906034FF4804301A8089306F058FD4D
:100F500008B172B6FEE731B05DF804FB1FB50021A1
:100F6000102268460BF0B0FB03F066F80123002264
:100F70006846ADF8003048F21F73CDE9012340F216
:100F80000113039303F06AF8042003F043F800F020
:100F900013FC02F085FF0E4B0322C3F82C28FFF749
:100FA00097FFFFF7BFFDFFF77BFD0BF03BF900F06C
:100FB0000FF900F03BF900F003FD00F067F9FFF7CF
:100FC0005BFE00F043FF00F0FFFE00F0BBFDFCE71E
:100FD000004002580268034B9A4201D1FFF7E2BB7E
:100FE000704700BF003000420268034B9A4201D1B3
:100FF000FFF7DBBB704700BF003000420268034BC5
:101000009A4201D1FFF7D4BB704700BF00300042C5
:1010100070470000024B834201D1FFF7E3BB7047EA
:10102000482800240268034B9A4201D101F074B9A8
:10103000704700BF004C00400268034B9A4201D148
:1010400001F046B9704700BF004C0040026808B587
:10105000044B9A4205D102F05BF9BDE8084002F06A
:1010600007BC08BD0058004072B6FEE7002310B56B
:10107000934201D1002010BD31F91340844201D0C8
:101080000133F5E70120F6E770B5002345689D427E
:1010900001D1002009E004685A01A25C04EB431668
:1010A0008A4203D1B368B3F9000070BD0133EEE7A3
:1010B0002DE9F74300230E460746144641688B424C
:1010C00029D03A684FEA431802EB431512F808207A
:1010D000B2423FD12B7D012B0DD0022B31D023B357
:1010E00002F0FAFE334602461B49002003B0BDE879
:1010F000F04302F0A1BED5E903122046FFF7B6FF88
:10110000814658B902F0E8FE234602461349484694
:10111000009602F091FE03B0BDE8F083AB681C803E
:101120003B68012243445A75F5E7B5F90230A34202
:1011300004DCB5F90430A342A8BF2346AA68138093
:10114000EEE702F0C9FE334602460549002002F0F0
:1011500073FEE5E70133B2E7B8CB000826CB000801
:1011600069CB00082DE9F34100240546174F2646B8
:101170006B689C4202D302B0BDE8F0812B684FEA55
:10118000441803EB44135A7DF2B19A69BAB19968D5
:10119000D869B1F900109047012814D902F09CFEDB
:1011A0002B680246002003EB080113F80830896819
:1011B000B1F90010CDE90011394602F03DFE2B686F
:1011C00043445E7500E0FAD10134D1E7FBCB00085F
:1011D00008B514480023144A4FF48021C363036503
:1011E000C0E900230722C0E902124FF00071C0E9F4
:1011F0000A32C0E904134FF000424FF08061C0E9A9
:1012000008338161C0E90D33C0E91233C0E9152309
:10121000C0E9173307F04AFB18B1BDE80840FFF7F3
:1012200023BF08BDB82700240030004208B5154888
:101230004FF48003144A4FF0806C4FF0E041C0E956
:1012400000234FF400330722C0E902320023C0E933
:1012500006C1C0E90433C0E90833C0E90A32C0E975
:101260000D33C3630366C0E91233C0E91433C0E928
:10127000163307F01BFB18B1BDE80840FFF7F4BEBA
:1012800008BD00BF282700240038004008B51648D4
:101290004FF48003154A4FF0005C4FF0A041C0E9C5
:1012A000002307224FF40033C0E902320023C0E9D3
:1012B0000A324FF08042C3630366C0E90433C0E9D9
:1012C00006C1C0E90833C0E90D23C0E91233C0E903
:1012D0001433C0E9163307F0E9FA18B1BDE8084045
:1012E000FFF7C2BE08BD00BF9826002400140058B6
:1012F0002DE9F041CAB006461422002109A80BF0DE
:10130000E3F96C2200210EA80BF0DEF98422002103
:1013100029A80BF0D9F93368AC4A934240F0828097
:101320004FF4000329A8299306F0AEFD08B1FFF79A
:101330009BFEA74BA020002409A9D3F8502121250A
:1013400042F48052C3F85021D3F850210092009A01
:10135000D3F8402142F00102C3F84021D3F84031D4
:101360000193019B0223CDE90903052399480D93BD
:10137000CDE90B4403F008FD332397490EA81294DE
:1013800015941B941F94CDE90E534FF40023CDE91F
:1013900013340123CDE91044CDE91733CDE91944C5
:1013A000CDE91C4403F064FB08B1FFF75DFE8A4AF7
:1013B00000218A4803F0FAFB08B1FFF755FE874881
:1013C00003F063FC08B1FFF74FFE854C854B2046C8
:1013D00023600023C4E90E33C4E910338123A364DE
:1013E00003F02EFA08B1FFF73FFE7C497C4803F07A
:1013F0007DFC08B1FFF738FE4FF080717848C6F8E1
:101400008440E66503F068F908B1FFF72DFE00227D
:101410003A20114602F098FD3A2002F0C7FD4AB08A
:10142000BDE8F081704A934248D14FF0807329A8FB
:10143000299306F029FD08B1FFF716FE644B00243E
:1014400002270326D3F84821052509A9674842F455
:101450008042C3F84821D3F848210292029AD3F877
:10146000402142F00202C3F84021D3F84021039208
:10147000039AD3F8402142F00102C3F84021D3F887
:1014800040310D950493049B4FF40043CDE90B4686
:10149000CDE9093703F078FC4FF4007309A94D48F2
:1014A0000D95CDE90937CDE90B4603F06DFC3B20E6
:1014B0002246214602F048FD3B20AEE74C4A9342CB
:1014C000ADD14FF0806329A8299306F0DDFC08B167
:1014D000FFF7CAFD3E4B002502244FF00508D3F864
:1014E0005421012709A93B4842F02002C3F85421A6
:1014F000D3F854210592059AD3F8402142F0010215
:10150000C3F84021D3F840210692069AD3F840212F
:1015100042F00402C3F84021D3F840210792079A11
:10152000D3F8402142F00202C3F84021D3F8403101
:10153000CDF834800893089BCDE90974CDE90B55AB
:1015400003F022FC4FF4805309A92A48CDF83480D7
:101550004FF00808CDE90934CDE90B5503F014FC30
:101560002023224809A9CDF83480CDE90934CDE9FA
:101570000B55214C03F008FC3E23204A2046A56071
:101580006563C4E900234FF48063C4E90555C4E9E9
:101590000338C4E90755C4E90977C4E90B5502F0DB
:1015A0008FFD08B1FFF760FD4FF080711248C6F85B
:1015B0008040E66503F090F808B1FFF755FD002282
:1015C0003F20114602F0C0FC3F2026E700300042D9
:1015D0000044025800000258742600245C260024AF
:1015E000E425002450100240003800400004025856
:1015F00000140058000802586C25002450150240C1
:101600000368274A934210B5044613D1254AA02106
:101610002548D2F8503123F48053C2F8503103F0FA
:1016200053FCD4F8840002F09FFE3A20BDE810403D
:1016300002F0CABC1D4A934212D11A4A4FF400412B
:101640001B48D2F8483123F48043C2F8483103F0F4
:101650003BFC15484FF4007103F036FC3B20E5E7F6
:10166000144A93421AD102F50C3201210E48D2F8E5
:10167000543123F02003C2F8543103F025FC4FF419
:1016800080510D4803F020FC2021094803F01CFC88
:10169000D4F8800002F068FE3F20C7E710BD00BF0D
:1016A0000030004200440258000002580038004058
:1016B00000040258001400580008025808B502201F
:1016C00005F0DEFC08B1FFF7CFFC05F049FD05F0A1
:1016D00027FD08B1FFF7C8FCBDE8084005F038BD9C
:1016E000FEE7FEE7FEE7FEE7FEE77047704770475C
:1016F00002F0E6BB014802F02CBF00BFE425002445
:10170000014802F026BF00BF04290024014802F06E
:1017100020BF00BF7C290024014802F01ABF00BF8F
:1017200028240024014802F014BF00BFA024002494
:10173000014807F0AFBE00BF48280024014807F069
:101740008DBC00BFB8270024014807F087BC00BF4C
:1017500028270024014807F081BC00BF98260024F8
:10176000014804F0D0B800BF18250024014804F057
:10177000A3BC00BF18250024014808F069BC00BFC5
:10178000F4290024014805F0DBB800BF8863002479
:10179000014802F0DEBE00BF6C250024044B054A60
:1017A0009A60D3F8882042F47002C3F8882070470A
:1017B00000ED00E000000008454A136903F038031B
:1017C000102B00F082800CD86BB1424B404A9269DA
:1017D000110742BF02F00F02073AD3403E4A13609E
:1017E0007047182B05D012683C4BC2F3C102D3409E
:1017F000ECE7916A936AD06AC3F30513C0073AD540
:10180000526BC2F3CC0206EE902AF8EEE66A002B89
:10181000DCD007EE903A01F00302F7EE005A2C4BB1
:10182000B8EEE77A012ADFED2E7A66EEA76A25D0B8
:10183000022A31D11B6B9FED2B6AC3F3080307EE1D
:10184000903AF8EEE77A77EEA67A77EEA57AC6EECA
:10185000076A67EEA67A1E4B1B6BC3F34623013360
:1018600007EE103AF8EEC76A87EEA67AFCEEC77A62
:1018700017EE903AAAE7DFED1C6AC8E71B6B9FEDF5
:101880001B6AC3F3080307EE903AF8EEE77A77EEA7
:10189000A67A77EEA57ADAE71968104AC1F3C10192
:1018A0001B6BCA40C3F3080307EE902AB8EEE76A41
:1018B000C6EE077A07EE103AB8EEC77A37EE267A08
:1018C00037EE257A67EE877AC5E7094B7EE700BFDA
:1018D0000044025800093D00000000240090D0039D
:1018E00000000039001BB74B000000000024744AC0
:1018F00000366E0110B588B004461422002103A8FA
:101900000AF0E2FE2368B3F1804F29D1154B012480
:1019100003A91548D3F8482142F00102C3F8482131
:10192000D3F848210192019AD3F8402142F00102F4
:10193000C3F840214FF40042D3F840310293029B98
:101940000223CDE903230323CDE9063403F01CFA77
:1019500033200022214602F0F7FA332002F026FB62
:1019600008B010BD004402580000025810B586B0FF
:1019700004461422002101A80AF0A6FE2368B3F150
:10198000804F16D10C4B03210C48D3F8402142F074
:101990000202C3F840210822D3F840310093009B93
:1019A0000223CDE901230123CDE9041301A903F0AA
:1019B000EBF906B010BD00BF004402580004025805
:1019C00010B590B000241422002104A80AF07CFE77
:1019D0001C22214609A80394CDE901440AF074FEB3
:1019E00024484FF0804384608461C0E900344FF0A4
:1019F000FF33C0E9033407F07DFE08B1FFF734FB85
:101A00001C4807F0A7FE08B1FFF72EFB0821194874
:101A100007F0D0FE08B1FFF727FB06205023002473
:101A200004A9CDE9040313480694089408F046F885
:101A300008B1FFF719FB01A90E480194039408F0BF
:101A400065F908B1FFF710FB702240F2251309A9D0
:101A50000848CDE90923022304220B9300230D93A8
:101A600007F010FF08B1FFF7FFFA0248FFF77EFF0B
:101A700010B010BD4828002407EE901AB2EE040AF8
:101A8000F8EEE77A08B587EE800A01F0BBF8003877
:101A900018BF0120400008BD08B5A1F11403044897
:101AA0004FF480515A425A4103F07CFA002008BD9D
:101AB0000004025821B1034B1A780AB901221A70A6
:101AC000002070479428002410B513460C4638B106
:101AD000012823D016490020BDE8104002F0ACB91F
:101AE00009B1042A06D0224612490020BDE8104060
:101AF00002F0A2B90978CB0705D5B4F9022049084C
:101B00000D48FFF7D5FA21780B484908FFF7BCFAD2
:101B100060802046BDE8104000F0F0BA0A8800213D
:101B2000064B0132C3E900111A81054B588010BDE4
:101B30008ACC00083DCC0008080000249828002426
:101B4000180200242DE9FF410DF1070203A902A8A4
:101B5000764D01F017FB00283DD1F2EE046ADDED71
:101B6000027A9FED737A67EEA67AF4EEC77AF1EE09
:101B700010FA00F18C809FED6F6AF4EE467AF1EE78
:101B800010FA76FE277AFDEEE77A17EE903ADDED51
:101B9000037A67EEA67A6B81F4EEC77AF1EE10FA5B
:101BA00078D49FED647AF4EE477AF1EE10FA77FE7E
:101BB000277AFDEEE77A04215F4817EE903AEB8131
:101BC0009DF807302B8203F0E7F92B8A002864D1B7
:101BD000C3F30E032B82594AB5F91030B2F9001045
:101BE000994210D0002B13805549ACBF00231F230E
:101BF00054488B70FFF73EF953495248FFF73AF9C2
:101C00005048FFF75BF9514CB5F902302668002BBC
:101C100048D10EB1B3712360002363604C48FFF7D5
:101C2000A1FA00F071FA4B4801F00CFA4A4B1A780D
:101C3000002A77D00025C8201D7002F053F9474BC9
:101C4000039372B64FF0E024256106F001F84FF0DF
:101C5000FF33434AC2F88030C2F88031C4F884317F
:101C6000C4F88432C4F88831C4F88832C4F88C319E
:101C7000C4F88C32C4F89031C4F8903262B6039B39
:101C8000039A126882F308885B689847FEE7F0EED3
:101C9000477A78E7DFED267A8BE76FEA43436FEA0E
:101CA000534397E72EB900F06BFA20600028B5D0B7
:101CB00066606768D7F5FE7611D02368D3F8008098
:101CC000FEF700FD864228BF064646B1381D314664
:101CD00008EB8000FEF7FCFC6368334463606268D5
:101CE000B2F5FE7F9AD320689E210368197021897E
:101CF0004E1C5980910004322681D9819200298896
:101D00009980E988D98069891981298A9981E98925
:101D10005981828000F0C6F900287FF47FAFC4E9C2
:101D200000007BE704B0BDE8F08100BF180200248A
:101D3000000000C700FEFF46000002580400002417
:101D4000AA28002410020024A42800249828002493
:101D50000800002434020024942800240080F11F8D
:101D600000E100E00AB201460148FFF7A1B900BF57
:101D7000080000240F4BB3F91630012B0E4B0BBF9C
:101D800011221322002002209A8000220B4B1A708D
:101D90009A700B4A587011889278A3F803105A7100
:101DA000084B18701120A3F8031058701F205A71A7
:101DB000987070471802002410020024AA280024FA
:101DC00064C70008A428002470B5082192B0174801
:101DD00003F0E2F80028164B0AAC14BF01220222DD
:101DE000144D0AAEDA82FFF7C5FF00F0DBF91248A6
:101DF000FFF72AF8FEF790FDFEF732FE0FCD0FC475
:101E000095E80F0001AD84E80F000FCE0FC594E8F0
:101E10000F0085E80F00094B4FF40051084A00936A
:101E2000084B094800F080FE12B070BD0030025827
:101E30001802002468C70008100200242824002487
:101E400018250024A02400240004025808B51648D0
:101E50004FF46143154AC0E9002300230C22C0E976
:101E600002330361C0E90523C0E90733C0E9093340
:101E700008F014FD08B1FFF7F7F800210A4808F050
:101E800007FE08B1FFF7F0F80021074808F020FE30
:101E900008B1FFF7E9F8044808F0DFFD18B1BDE824
:101EA0000840FFF7E1B808BDF4290024004C0040C9
:101EB00070B5A8B006461422002102A80AF004FC5E
:101EC0008422002107A80AF0FFFB3268414B9A42A6
:101ED0007ED14FF0005307A8079305F0D5FF08B156
:101EE000FFF7C2F83C4B4FF4C05100253B48D3F8F4
:101EF00048213B4C42F40022C3F84821D3F8482142
:101F00000092009AD3F8402142F00102C3F8402128
:101F1000D3F840310193019B0223CDE9021306233C
:101F200002A90693CDE9045502F02EFF2D484F2358
:101F300025616563C4E900034FF400232046C4E92A
:101F400005350123C4E90255C4E90755C4E909333D
:101F5000C4E90B5502F0B4F808B1FFF785F84FF06B
:101F600080711F48C6F88040E66502F0B5FB08B1F5
:101F7000FFF77AF81C4C50231C4A2046C4E9002382
:101F800000234FF48062C4E90232082223626363B3
:101F9000C4E904230122C4E90633C4E90922C4E9DF
:101FA0000B3302F08DF808B1FFF75EF84FF0807147
:101FB0000D48F467E66502F08FFB08B1FFF754F8AF
:101FC00000225520114601F0BFFF552001F0EEFF21
:101FD00028B070BD004C0040004402580000025878
:101FE0007C290024D0110240042900245011024011
:101FF00000487047F4290024004870477C290024D9
:10200000004870470429002410B50446006838B120
:10201000A18829B10AF06EF908B90223A37110BD95
:102020000320FCE7012810B50C4606D0022819D081
:10203000B8B9BDE81040FFF747BD144B1A688A4293
:1020400007D0134B1A688A4203D0124B1A688A428F
:1020500007D100229A71E278A37843EA02230E4A5C
:10206000138010BD02460C490120FFF72DFD0B48DF
:10207000FEF7B9FC0A48FEF7B6FC0023034A937149
:10208000034A9371034A9371EBE700BF7C0200247B
:10209000740200246C0200248C2A002454020024C0
:1020A0003C02002407B5019008B1838853B901F0C0
:1020B00013FF0F490246002001F0BEFE042003B0CA
:1020C0005DF804FBB3F5006F08D901F005FF09497D
:1020D0000246002001F0B0FE0520F0E701A9064805
:1020E000FEF73AFC0028F7D1019B01229A71E6E73E
:1020F000AACC0008E2CC00083C02002401460148BA
:10210000FEF72ABC5402002473B5194C194D1A4E1F
:102110002046FEF71BFC98B1184C2046FEF716FC33
:1021200020BB01A92046FEF74EFCF8B90198FFF745
:102130006BFF0028F1D101A92046FEF729FCECE74E
:1021400001A92046FEF73FFC80B996F89C32019821
:10215000032B286004D001A92046FEF719FCD7E71D
:10216000042128460AF0C6F80028F4D002B070BD59
:1021700054020024882A00248C4C00243C020024B1
:10218000054883793BB10548837923B104488379B5
:10219000002B18BF002070477C020024740200242A
:1021A0006C02002470470000024B00221989586815
:1021B00002F0F8BEF846002430B5ADF5017D0446C6
:1021C0000D464FF400720B4968460AF0B1FA2544F7
:1021D00023460020AB4202D10DF5017D30BD13F83E
:1021E000012B82EA102200023DF8122080B25040FA
:1021F000F0E700BF88C700082DE9F8432E4F8E4650
:10220000194615463B7803F0FF064BB101F064FE1A
:102210002A490246002001F00FFE0520BDE8F883A0
:1022200002F1030C264CFF2302F10A081FFA8CFC72
:102230002071237004F108006370FD2384F805C049
:102240004FEA1C2C84F807E01FFA88F884F806C0CF
:102250004FF00109A370E6700AF06AFA05F108016F
:102260002046184D89B2FFF7A7FF04EB08030122AF
:10227000298903F8020C000A03F8010C686802F0CF
:1022800091FE4FF4807231460F4887F800900AF0B3
:102290001BFA42462146286807F0D0FD0028BDD031
:1022A00001F01AFE09490246304601F0C5FD3E70B4
:1022B000FFF77AFF4846B1E7F444002417CD000841
:1022C000F5450024F8460024F544002462CD0008BA
:1022D00038B50D4C2378012B14D100252570FFF75C
:1022E00063FF0223072209492370094B186808F08D
:1022F0006DFB38B101F0F0FD06490246284601F0B9
:102300009BFD257038BD00BFF4440024F544002433
:10231000F84600249DCD00082DE9F041284D2B788A
:10232000022B1BD12749284B0A7907311A7031F843
:10233000022C9A809A88254B92B2186808F046FBC6
:1023400018B903232B70BDE8F08101F0C5FD2049C9
:102350000246002001F070FD0423F3E72B78032BE5
:10236000F1D1194E174CB788B01DB288BFB21949C8
:1023700092B207F10708043A0AF0DAF9E3791FFA92
:1023800088F8791DB3702046237A444489B273706B
:10239000FFF712FF14F8012C14F8023C43EA022361
:1023A000834204D001F098FD0B490246D1E74FF477
:1023B0008372314609480AF0BBF90023C2E700BF27
:1023C000F4440024F5440024EE430024F84600249D
:1023D000D5CD0008FE4400241DCE0008E8420024AC
:1023E00010B5FFF705FE084C084B20606360012321
:1023F0002381FFF701FEE060FFF702FE2061FFF797
:10240000D3FE002010BD00BFF8460024000402588F
:1024100008B5054B186807F06DFDFFF7C5FE034BC7
:1024200000221A7008BD00BFF8460024F4440024BE
:102430004FF48372024908B50AF07AF9002008BD0A
:10244000E8420024014B1878704700BFF444002490
:1024500007B5ADF8041001ABADF806200221042247
:10246000FFF7CAFE03B05DF804FB2DE9F041144606
:102470000D46694600AF093402F102080646E40839
:10248000A1EBC4018D4619468DF800502D0A0DF1BF
:1024900002008DF801500AF04BF96B461FFA88F2E2
:1024A00003213046FFF7A8FEBD46BDE8F0810000DD
:1024B0000C4B10B51A790446824212D00022032830
:1024C000187118BF1A76C3E9022201F005FD064B08
:1024D0000246064953F824300020BDE8104001F0C0
:1024E000ABBC10BD0C4700248402002444CE00087D
:1024F0007E230B41DB0710B50C4612D5837983B1DF
:1025000001F0EAFC074B0246074953F8243000204B
:1025100001F092FC054B03201C76BDE81040FFF74C
:10252000C7BF10BD9402002476CE00080C470024DB
:10253000DFED9A7A60EE277A2DE9F041FDEEE77A39
:10254000974C0746656917EE901A2669551B8E1B36
:10255000C4E904122279032A00F2B780DFE812F0FE
:10256000B80004009600F00007EE903AF8EEE77A23
:10257000002D5CD0B7EE007AB4EEC70AF1EE10FA87
:1025800013DDF4EEC07AF1EE10FA00F30481002EB0
:10259000D4BF4FF000084FF00108B0EE007AB4EE5F
:1025A000C70AF1EE10FA4ADC17E0BFEE007AB4EE8B
:1025B000C70AF1EE10FA63D5F4EEC07AF1EE10FA24
:1025C0005BDD4FEAD678B8EE007AB4EEC70AF1EEDA
:1025D00010FA02D5734A964234DC0A22B7EE005B49
:1025E00030EE677A93FBF2F306EE103AB0EEC77A5C
:1025F000B8EEC66BB7EEC77A86FE056BBDEEC66B4E
:1026000016EE103A142BA8BF142306EE103AB8EEBB
:10261000C66BB4EEC67BF1EE10FA34D5A368013375
:10262000032BA36012D90220FFF742FF0EE0B0EEA9
:10263000007AA846B4EEC70AF1EE10FAC3DD5A4A92
:102640009642CADA01213846FFF752FF2379032B5D
:1026500000F09E80B8F1000F40F09A8085EAE573A3
:10266000A3EBE573FA2B40F39380002D6FDAB6F5F8
:10267000FA6F6FDB0023E36075E04FF00008A2E71C
:102680004FF00008A9E70023A360DFE7A268B0F9D4
:10269000001001328A42A26011D307EE903AB7EEE1
:1026A000007AF8EEE77A77EEC07AF0EEE77AF4EEA9
:1026B000C77AF1EE10FA02D80020FFF7F9FEA368FE
:1026C0002C2B02D90020FFF7F3FE4FF00008BDE7E6
:1026D00022689A4202D001202360F4E707EE903A84
:1026E000B3EE047AF8EEE77A77EEC07AF0EEE77AA6
:1026F000F4EEC77AF1EE10FA07DD0320FFF7D8FEFB
:1027000003213846FFF7F4FEDFE7002B07DD15F164
:102710000F0FACBF0023012333B9A360D5E70F2D02
:10272000D4BF00230123F7E7A368B7F902200133E0
:102730009342A360C9D30320FFF7BAFE0421E0E768
:1027400022680AB12360C0E7002BBED0C3E716F5AC
:10275000FA6F8FDDE3680133022BE36003D90521B3
:102760003846FFF7C5FE07EE906AF8EEE76A07EE17
:10277000905AF8EEE77A86EEA77ADFED0C7AB4EE9F
:10278000E77AF1EE10FA03DB06213846FFF7B0FED8
:10279000207EBDE8F0814FF00008FEE600007A449C
:1027A0000C470024400D0300C0F2FCFF000048422B
:1027B000014B1879704700BF0C47002408B5002072
:1027C000FFF776FE044B00221A761A60C3E9022254
:1027D000C3E9042208BD00BF0C470024FFF7EEBF89
:1027E00008B5062814D8DFE800F0041A23131313E1
:1027F0002A00154B002293F83310022909D003292F
:102800000AD0012901D183F83020002283F8332037
:1028100008BD83F83120F8E783F83220F5E701F0AE
:102820005BFB0A4902460020BDE8084001F004BBFA
:10283000054B0A685A62012283F82E20E8E70A88CD
:10284000014B1A84E4E700BFB00200246BCF0008FC
:10285000034B012283F82F00002083F831207047BA
:10286000B0020024034B01221884002083F830209A
:10287000704700BFB002002408B500F0EFFEB0FAC8
:1028800080F0400908BD0000014B93F82C00704710
:10289000B0020024094B93F82C0060B940F20112F9
:1028A000187398601877986118849A8583F82E00B9
:1028B000C3E9090070470320704700BFB00200243D
:1028C000054BD3E90903C01A0028B8BF4042CB2802
:1028D000CCBF002001207047B0020024084BD3E990
:1028E0000902B3F92030002B04DD9042D4BF002050
:1028F000012070479042ACBF00200120704700BF0C
:10290000B002002408B50A4AFFF7DAFF60B9094BA4
:10291000D2E909018842B8BF4FF4007301200121B8
:10292000138482F8301008BD00231846F7E700BF73
:10293000B002002400FEFFFF094AD2E909329FEDF0
:10294000067B9B1A00EE103AB8EEC00B20EE070B88
:10295000B7EEC00B704700BFE72AAB23262C8A3E98
:10296000B0020024014B586A704700BFB002002437
:1029700010B5084CA188206802F00EFB38B1A18A7E
:10298000206902F009FBB0FA80F0400910BD012077
:10299000FCE700BFB0020024F8B500F06BFE00F0C9
:1029A00027FE78B300F05AFE60BB444C94F82C30FC
:1029B000012B1CD1424B94F82D501E78A188B542B2
:1029C000206818BF1D70013D02F0E6FAA18A074693
:1029D000206902F0E1FA042D09D8DFE805F00318B8
:1029E00022334E00012E0ED0012384F8323094F8A9
:1029F0003030002B45D0B4F9200000F022FE012336
:102A000084F83330F8BD022384F82D30EFE7022E2E
:102A100005D0012384F8313084F82F30E7E7032311
:102A2000F2E7032E06D0012384F830304FF4007310
:102A30002384DCE7002FDAD1636AA36001232373C8
:102A40000423E1E7042E1FBF012384F830304FF444
:102A50007E4323840028CAD10122636A208484F83B
:102A6000302022770522A36184F82D20A268134428
:102A700003EBD3735B10A362B9E7022384F82C3015
:102A8000B5E794F831302BB194F82F0000F0B6FD83
:102A90000223B5E794F832301BB100F0CFFD0323D9
:102AA000AEE7084D01F018FA04462B68C31A322B22
:102AB000A8D900F0B0FD2C60A4E700BFB00200244C
:102AC000284700242C47002408B5074800F0CCFD17
:102AD00000F0E6FD38B101F0FFF90449024600209C
:102AE00001F0AAF9012008BDE127000899CF0008EC
:102AF00008B5044B01221988034B186802F052FAFA
:102B0000002008BD684700246C47002408B5044B2A
:102B100000221988034B186802F044FA002008BD0F
:102B2000684700246C4700242DE9F04F1E4687B00B
:102B30000123DFF8CC80824689461746DDF840B095
:102B400088F80030FFF7C0FF054660B1042601F0A9
:102B5000C3F92B4602462349002001F06DF93046A7
:102B600007B0BDE8F08FFFF739FE6846CDF808B032
:102B7000CDE9007600F066FB044648B101F0ACF9FF
:102B80002346024618492846052601F055F9E6E78E
:102B900003A8CDF814B0CDE9037600F099FD064600
:102BA00048B101F099F933460246104920460626FD
:102BB00001F042F9D3E70E4B11AD0E4CC3F800A063
:102BC0000D4BA3F800900FCD0FC495E80F0084E8DB
:102BD0000F00022388F8003001F07EF9074B58619E
:102BE000BDE700BFCDCF00081ED000086CD00008A4
:102BF0006C470024704700246847002444470024A1
:102C00009047002408B50F4B1A78022A08D0012AF1
:102C100008D801F061F90C490246002001F00CF9D6
:102C2000012008BDB5EE400A084981ED030AF1EE26
:102C300010FA05D1042A01D003221A700020F0E70F
:102C40000622FAE790470024BDD000087047002410
:102C5000F8B5214E0027214C05462DED028B337827
:102C600084F82070062B2FD101F036F9E369C01AE1
:102C7000B0F5967F28D3FFF75FFEB0EE408AFFF7EE
:102C800071FE174B02462846B7EEC80AD3ED037A09
:102C90009FED0F6BFDEEE77A20EE060B17EE903AF4
:102CA000FDEEC07B94ED010A17EE901AFFF740FC91
:102CB00084F8200040B101F00FF90A490246384675
:102CC00001F0BAF803233370BDEC028BF8BD00BFEE
:102CD0000000000080842E419047002444470024D7
:102CE0007047002444D100082DE9F043B64E87B068
:102CF000B64F804601F0F0F833783A780446B44D88
:102D00009A42A3F102031CBF01222A70062B00F293
:102D10008981DFE813F00700300048000C008F00C5
:102D200054017B01FFF7B0FD78B1022820D02B7849
:102D30003278002B40F07F813B789B1A18BF01232B
:102D40002B703A7007B0BDE8F083FFF7D1FEFFF7B4
:102D5000A1FD80460028EAD001F0BEF843460246B5
:102D60009C49002001F068F89B4B06221A70DEE7B0
:102D700003233370DBE72B7863B1984B0022DA60D2
:102D8000FFF7B6FE00214520FEF7ECFFFFF7BAFD86
:102D9000FFF714FDFFF7A2FD0028C8D00020FFF7C1
:102DA00061FD0423E5E72B78DFF85C8273B1002036
:102DB000FFF74EFD8A4A00230021546113605360DF
:102DC000884AC8F800401160874A1360D8F800307C
:102DD00040F2DB52E31A9342A9D940F6B73293424C
:102DE00012D803A800F0EAFA0028A0D17E4BDDED4E
:102DF000037A93ED007A7B4A77EE877AC3ED007A07
:102E000013680133136092E7764B754A1B68764965
:102E1000002B0ADD07EE903AD1ED006A5461F8EE1E
:102E2000E77A86EEA77A82ED007A00230B60536082
:102E300005239EE72B7843B10120FFF709FDFFF73B
:102E400065FE01F049F8664BD8614046FFF700FF88
:102E5000FFF712FD00283FF46AAF684600F0AEFAB3
:102E6000804628B101F038F8434602465F4978E7CA
:102E70005B4C03A8DDED007A94ED007A77EEC77A1B
:102E8000CDED007A00F010FD814628B101F024F864
:102E90004B460246564964E7039BA36101F01CF8C8
:102EA0006369B7EE005A9FED537A8046C31A94EDDA
:102EB000016A07EE903A494BF8EE677AD3ED036A60
:102EC000C7EE875A9DED007AD3ED047A37EE466A55
:102ED00076EEC76AC4ED026A86EE257A94ED036A3F
:102EE00065EEA77A35EE675A27EE277AD4ED047A95
:102EF000A5EE277AD3ED017A66EEA77AA5EEA76A4A
:102F0000D3ED057A84ED047AB4EEE76A84ED036AC2
:102F1000F1EE10FA02DDC4ED037A06E0F1EE677A15
:102F2000B4EEE76AF1EE10FAF5D4F0EEE67A93ED3E
:102F3000066AF4EEC67AF1EE10FA38D493ED006A20
:102F4000D4ED037AE6EE867AD3ED026AE7EE267ACE
:102F5000D3ED076AF5EEC07AF1EE10FACCBF01228C
:102F600000224CBF01210021521A07EE102AB8EEB0
:102F7000C77AE6EE877A9FED207A67EEC77AFDEE94
:102F8000E77A17EE903A18B21C4B9842B8BF184631
:102F9000B0F5007FA8BF4FF40070FFF763FC8146D7
:102FA00040B100F099FF4B4602461549D9E6DFEDE6
:102FB000157AE0E7009BC4F814806360B7E6002050
:102FC000FFF750FCB3E600BF904700243C470024C5
:102FD000E402002484D100089147002470470024B3
:102FE000444700243447002440470024D1D100083E
:102FF00019D2000800007A440000004400FEFFFFE0
:1030000064D2000800000000384700242B78002B11
:103010003FF48DAE00F060FF08490246002000F04A
:103020000BFF84E62B78002B3FF481AE00F054FFB9
:1030300003490246F2E7002382E600BFA7D2000858
:10304000F2D20008F8B5374F064600F045FF0546B6
:10305000FFF7A2FC3B78012B08D800F03DFF324976
:1030600002460020BDE8F84000F0E6BE2F4C237871
:10307000052B1CD8DFE803F0031C2A3842502C4EE5
:103080003368EB1A632B12D9FFF772FC60B13B78FF
:10309000023B012B08D900F01FFF26490246002001
:1030A00000F0CAFE03233B70012335602370F8BD96
:1030B00000F0B0FB08B90223F8E700F00DFF1E494D
:1030C0000246002000F0B8FE0623EFE700F000FC07
:1030D00008B90323EAE700F0FBFB0228E7D100F080
:1030E000FBFE16490246ECE700F0E2F808B90423BB
:1030F000DCE700F0F1FE12490246E2E700F074F965
:1031000008B90523D2E700F06FF90228CFD100F00B
:10311000E3FE0C490246D4E73046FFF7E5FD002305
:10312000C4E700BF90470024BDD0000891470024A9
:10313000304700243FD300089FD30008E8D300089D
:1031400032D4000878D4000808B50D4B1B78062B44
:1031500007D8DFE803F00404130A0A11080000206E
:1031600008BD0320FCE70220FAE7FFF721FB032854
:103170000CBF05200620F3E70420F1E70120EFE76C
:1031800090470024124B10B51B781446012B08D829
:1031900000F0A2FE0F490246002000F04DFE012083
:1031A00010BD08B101B142B900F096FE0A490246CD
:1031B000002000F041FE0220F2E7084B5A689B69AC
:1031C00002600B60FFF7C0FF20700020E8E700BF3F
:1031D00090470024BDD00008BFD400084447002415
:1031E00010B5044640B900F077FE14490246204667
:1031F00000F022FE042010BDC9B2062908D8DFE87D
:1032000001F0111704090C0F1A000D4B03221A705C
:103210000020F0E70A4B0222F9E70123A371F7E748
:103220000023FBE7064B1A78062AF1D10722EEE7C6
:10323000034B0622EBE700F0D5F8E9E705D50008D7
:1032400090470024034610B528B1006818B15A68A9
:103250000AB19B684BB9042400F03EFE0F490246B8
:10326000002000F0E9FD204610BD0D4B0322502147
:103270001860642302F0C6FA044648B100F02CFE40
:103280002346024607490020022400F0D5FDEAE764
:10329000054B01221870054B1A70E4E76FD5000842
:1032A0009C470024AFD5000898470024924700248B
:1032B000114B1B7870B5DBB1104D2B7803F0FF0676
:1032C000C3B901230E480F4A50212B700223006816
:1032D00002F0E0F9044648B100F0FEFD2346052463
:1032E00002460949304600F0A7FD2E70204670BD09
:1032F0000124FBE70624F9E79247002498470024BD
:103300009C47002499470024F2D5000800000000E3
:1033100070B5254E3378012B0ED1244B244C1A88DE
:1033200052BA95B2B5F5804F11D3AD0B022D04D131
:10333000072323720023337070BD00F0CDFD2B46B0
:1033400002461C49002000F077FD0323F1E7A2F2BA
:103350006662194B12B207EE902A9FED0F5BB8EE32
:10336000E77B9FED0F6BA7EE056BD3ED007AB6EE12
:10337000007A67EE877AB7EEC66BE6EE077AC3EDA2
:10338000007AC4ED007A00F0A7FD0023606023728C
:10339000D1E700BFAFF3008085B69C4B7155D83F95
:1033A00014AE47E17A77A3C09847002499470024D8
:1033B000E802002438D6000894470024074A034650
:1033C000127832B138B1064A07CA83E807000020F4
:1033D0007047012070470420704700BF92470024C7
:1033E000E802002400207047014B1878704700BFA6
:1033F0009847002470B54E4CC4B0FFF723F8267AE6
:10340000032E00F28C80DFE806F005021D2108B9CA
:10341000022323720025237A8BB100F05DFDE3685F
:10342000C01AC8280BD900F057FD424902460020B7
:1034300000F002FD0425FEF7EBFF0023237228466F
:1034400044B070BD0028E5D10323E2E702A8FEF7EF
:10345000EFFF0546002856D10190207C022807D0B6
:1034600003284ED000F038FD237C024632490EE09E
:10347000638A642B36D00ED8402B39D0462B22D00D
:103480000B2B26D000F028FD638A02462B49002032
:1034900000F0D2FC24E07A2B0CD0842BF2D1DDF8A2
:1034A0000E30019300232372E369002BB3D001A9EE
:1034B0009847B0E79DF80E303046003B18BF012317
:1034C0008DF80430EEE79DF80E300120ADF80430A1
:1034D000E8E79DF80E30A3F1100253425341A37662
:1034E0000720DFE7BDF80E300620ADF80430D9E73D
:1034F0009DF80E300520003B18BF01238DF80430E5
:10350000D0E72846CEE700F0E7FC2B4602460C4900
:103510000020012500F090FC002323727BE700F0DF
:10352000DBFC237A02460749002000F085FC71E7A6
:10353000A047002471D70008BED6000876D6000840
:1035400010D7000842D700082DE9F843244D8046E3
:103550000C46164695F800901F46B9F1000F0AD1A7
:10356000052400F0B9FC1F490246484600F064FCFF
:103570002046BDE8F8832B7A43B100F0ADFC1A4930
:1035800002460020062400F057FCF1E72874698207
:10359000AA8227B1394605F1160009F0C9F8B8F139
:1035A000020F10D1324621460120FEF751FF04469A
:1035B00080B100F091FC234602460C490020012412
:1035C00000F03AFCD4E73B46324621460120FEF7A4
:1035D0004CFFECE701232B7200F07EFCE860C7E7AC
:1035E000A0470024BBD70008E8D700080AD8000885
:1035F000014B1878704700BFA047002407B501228F
:103600000DF1070340218DF807000320FFF79CFF11
:1036100003B05DF804FB0023042284210220FFF79D
:1036200093BF07B501220DF107030B218DF80700A9
:103630000320FFF789FF03B05DF804FB1020FFF7BC
:10364000F0BF07B5022201AB6421ADF804000320EE
:10365000FFF77AFF03B05DF804FB0000014B187A16
:10366000704700BFA0470024014BD861704700BFDE
:10367000A047002438B5094C257845B900F02CFC4A
:103680006368C01AB0F57A7F05D301232370BDE8C3
:103690003840FFF7AFBE284638BD00BFA047002422
:1036A00010B5FEF79DFE044648B1012400F014FC5D
:1036B00005490246002000F0BFFB204610BD00F087
:1036C0000BFC024B5860F8E73ED80008A0470024E6
:1036D0002DE9F041034686B028B1006818B15A6858
:1036E0000AB19B685BB9042400F0F6FB3F4902462F
:1036F000002000F0A1FB204606B0BDE8F0813C4E62
:10370000642303229221306002F07CF8044640B129
:1037100000F0E2FB234602463649002000F08CFB15
:103720004BE043F20123642705AA9221ADF814303F
:10373000402300978DF816300323306801F07CFE9B
:10374000054628B100F0C8FB2B4602462A49E4E7AB
:103750004FF00108052000F0C5FB009743460DF12E
:103760000F02922130688DF80F8001F065FE04464B
:1037700040B90097022304AA9221306801F0F2FEBA
:10378000044628B100F0A8FB234602461B49C4E7C3
:10379000BDF810506DBAADB285F44953C3F30B03B5
:1037A0006BB1C5F30B0500F097FB4FF410730246A5
:1037B00013492046009500F03FFB02249BE7114A85
:1037C0009221137043460097306801F035FE04469D
:1037D00028B100F081FB234602460B499DE70B4BC5
:1037E00000221A7001220A4B1A7084E77ED8000862
:1037F000C8470024C1D8000807D9000852D90008DA
:10380000A1D90008C247002400DA0008C1470024FB
:10381000C0470024114B1B7870B5DBB1104D2B78DD
:1038200003F0FF06C3B901230E480F4A92212B7003
:103830000223006801F02EFF044648B100F04CFB63
:103840002346052402460949304600F0F5FA2E7059
:10385000204670BD0124FBE70624F9E7C047002499
:10386000C1470024C8470024C34700244FDA00089A
:1038700038B50A4D2B78012B0FD1094B094C1B8809
:10388000DBBA07EE903AFAEEEC7AC4ED007A00F07B
:1038900023FB0023606023722B7038BDC1470024D6
:1038A000C3470024F4020024074A0346127832B1C9
:1038B00038B1064A07CA83E8070000207047012094
:1038C00070470420704700BFC0470024F402002462
:1038D000014B1878704700BFC14700240D4885464A
:1038E000FDF75CFF0C480D490D4A002302E0D45857
:1038F000C4500433C4188C42F9D30A4A0A4C00233A
:1039000001E013600432A242FBD308F0E5FEFDF7AC
:1039100025FBFEE70000012000000024F80300243E
:1039200050DB0008F80300246C680024FEE70369FC
:10393000C26893429CBF81685B18013B981A70472C
:103940002DE9F041D0E9028405464068A8EB040661
:103950000F4620441444964206D908F0E9FEBFF30E
:103960005F8FEC60BDE8F081A4EB0804324608F0FC
:10397000DFFEB91922466868EFE72DE9F8430646ED
:1039800089461746C5684FF0000833694946B46850
:103990009D42706828BF1B19641B2844BC4203F178
:1039A000FF3328BF3C465B1B9C4228BF1C46224677
:1039B000254408F0BDFEB368A044A1443F1BAB42C0
:1039C00008BF0025BFF35F8FF560002FDDD14046B3
:1039D000BDE8F88310B50323134C144A2361E01D9E
:1039E0006361134BA261E3614FF480631149236269
:1039F0000023A3626362E36222660F4A62661022BA
:103A0000A2662367E366636708F08AFEBFF35F8FF1
:103A10000A49204608F084FEBFF35F8F2023A3717C
:103A2000BFF35F8F10BD00BFDC4B002498DA0008A5
:103A3000DC470024A1DA0008CC470024A5DA0008FE
:103A4000F8B51827134B0E46144600FB07751D44A6
:103A500007FB0033DB6A012B0AD0022B14D023B9F9
:103A60002846FFF764FF844208D900242046F8BDA9
:103A70002846FFF75CFF844228BF044622463146B1
:103A80002846FFF75DFFF1E72846BDE8F840FFF75D
:103A900074BF00BFDC4B0024F8B50B4B04460D4649
:103AA00016461B780BB9FFF795FFEFF311874FF020
:103AB000200181F31188324629462046FFF7C0FFD6
:103AC00087F31188F8BD00BFDC4B0024826810B575
:103AD000531C04464068834205D820688154A36083
:103AE000E3680133E360D4E901329A420BD12168E3
:103AF0002069FFF7D1FFA368984215BF4FF0FF334D
:103B00000023E360A36010BD2DE9F84F17469946E6
:103B1000064688460A464FF0010ADDE90A43BA42E2
:103B200012D2CA4538BFCA4613F0010B01D184B97D
:103B30000024F368002B3DDB0125B9F1010F1FD9EB
:103B400009F1FF397D43F8E7B2FBF7F20AF1010A08
:103B5000E5E79B0711D5B9F1000F0CBF30252025F3
:103B6000A245E6D229463046FFF7B0FFF368013C94
:103B7000002BDEDB002CF3D1DAE72025F0E77D43D4
:103B8000B8FBF5F39F42FAD9DFF848903046B8FB0E
:103B9000F5F319F8031005FB1388FFF797FFF36897
:103BA000002B03DBBD42B5FBF7F305D2BBF1000FE1
:103BB00000D05CB9BDE8F88F1D46E7E7202130460C
:103BC000FFF784FFF368013C002BF3DB5445F5D885
:103BD000F0E700BF08DB00082DE9F04F9BB00023A1
:103BE0000E4615460DF1280A40210390CDF814A089
:103BF000CDE90613CDE9083016F8011B39B9089D47
:103C0000002D00F30E8108981BB0BDE8F08F252928
:103C100040F0BA804FF0000907E0302B0FD149F097
:103C2000020901E049F001090E46314611F8013B55
:103C30002D2BF7D0F1D8232B13D02B2B0ED0002413
:103C4000314611F8013BA3F1300009280CD80A22B3
:103C50000E4602FB0433A3F13004F1E749F00409F6
:103C6000E2E749F00809DFE72E2B11D10E464FF0AD
:103C7000000B0A27304610F8011BA1F1300CBCF1F3
:103C8000090F07D807FB0B110646A1F1300BF1E72E
:103C90004FF0000B304610F8011B01F0FB07064601
:103CA000682FF8D0782909D86F290BD8632967D0F5
:103CB00020D8252968D0582900F09380089B002B34
:103CC0009ADA9CE770390829F8D801A050F821F059
:103CD000133E0008BD3C0008BD3C0008F33D000851
:103CE000BD3C0008D13D0008BD3C0008BD3C0008BB
:103CF000E33D00086429E1D129684FF001080F680D
:103D0000081D87EAE77128600A20A1EBE7710929FD
:103D10003EDCD84538BFD8462CB1002F02DB19F065
:103D2000040F00D0013C19F0020F02D0BBF1000FCC
:103D300004D019F0010F01D17CBB0024089900299F
:103D4000BCDB002F34DA7F422D2105A8FFF7BEFE31
:103D500008990029B2DB09F00301022904D1BBF163
:103D6000000F01D14CBB002408990029A6DB5B465B
:103D70000A223946CDE9004905A8FFF7C5FE9DE7AF
:103D80002B681A1D19782A6005A8FFF79FFE95E792
:103D9000B1FBF0F108F10108B9E74445CED9202183
:103DA00005A8FFF793FE0899013C0029C4DAC5E78E
:103DB00019F0040FCFD02B21C7E74445D4D93021C7
:103DC00005A8FFF783FE0899013C0029CADACBE772
:103DD00029685B460A22081D2860CDE90049096868
:103DE000CAE729685B46081D2860CDE90049102212
:103DF000F5E72B681A1D2A601C6814F8011B0029BE
:103E00003FF45CAF05A8FFF761FE089B002BF4DAD6
:103E100054E7296800220B1D2B600823CDE90032EE
:103E2000E5E7079C24B1224651460398FFF734FE8C
:103E30002C440894E7E600BF0EB403B503AB01AA17
:103E400053F8041B0193FFF7C7FE02B05DF804EBC3
:103E500003B0704738B50F4B05461A780AB90120F0
:103E600038BD4FF47A73B3FBF2F30B4A1068B0FB22
:103E7000F3F000F0BBF804460028F0D10F2DEED887
:103E8000024629464FF0FF3000F05EF8034B204613
:103E90001D60E5E700030024000000240403002463
:103EA00010B5032000F03EF80F20FFF7D3FF0446C3
:103EB00018B9FDF703FC204610BD0124FBE7000004
:103EC000034A044B11681B780B441360704700BF12
:103ED000844C002400030024014B1868704700BF85
:103EE000844C002438B50446FFF7F6FF0546631CF2
:103EF0001EBF044B1B78E418FFF7EEFF431BA342E1
:103F0000FAD338BD000300244FF0E022136923F0F8
:103F10000203136170474FF0E022136943F002037C
:103F20001361704707490302CA6803F4E06322F48F
:103F3000E0621204120C134343F0BF6343F40033F6
:103F4000CB60704700ED00E0164B30B5DC68C4F381
:103F50000224C4F10703251D042B28BF0423062DCA
:103F60004FF0FF358CBF033C002405FA03F3002813
:103F700005FA04F521EA030322EA050203FA04F331
:103F800043EA02034FEA0313DBB206DB00F16040B1
:103F900000F5614080F8003330BD00F00F00024AA8
:103FA0001354F9E700ED00E014ED00E0002807DB12
:103FB0000123410900F01F00024A834042F82130EA
:103FC000704700BF00E100E000280CDB430901223C
:103FD00000F01F0004492033824041F82320BFF342
:103FE0004F8FBFF36F8F704700E100E00138B0F1F1
:103FF000807F0BD24FF0E023054AF021586100206A
:1040000082F82310072298611A61704701207047D7
:1040100000ED00E0BFF35F8F064B40F00100C3F8F6
:1040200094005A6A42F480325A62BFF34F8FBFF352
:104030006F8F704700ED00E0BFF35F8F064B5A6A49
:1040400022F480325A620022C3F89420BFF34F8FCB
:10405000BFF36F8F704700BF00ED00E0174A437851
:10406000C2F89830D2F8A03023F00103C2F8A03093
:10407000D2F8A03023F00103C2F8A0304368C2F8A0
:104080009C30C37A017B1B0643EA017301780B4322
:10409000817A43EAC143417B43EA8143817B43EA1E
:1040A0004143C17B43EA0143417A43EA0123017A58
:1040B00043EA4103C2F8A030704700BF00ED00E0C2
:1040C00038B50446FFF708FF0546002C00F03A819A
:1040D0000023226884F84C30022384F8543053695A
:1040E00043F00603536123685A69D20700F11F8128
:1040F0005A69216A22F4430296480A43E1695A61E7
:1041000062690A4321690A43A1690A4392498B42C1
:104110005CD080318B4259D080318B4256D0803177
:104120008B4253D080318B4250D080318B424DD066
:1041300080318B424AD080318B4247D080318B42D4
:1041400044D080318B4241D080318B423ED080318F
:104150008B423BD080318B4238D080318B4235D07E
:1041600080318B4232D080318B422FD07B498B42C1
:104170002CD080318B4229D080318B4226D08031A7
:104180008B4223D080318B4220D080318B421DD096
:1041900080318B421AD080318B4217D080318B42D4
:1041A00014D080318B4211D080318B420ED08031BF
:1041B0008B420BD0834209D001F580718B4205D030
:1041C00080318B4202D080318B420DD1A16A0139FE
:1041D000090501F07C711143E26A1143626A013AF8
:1041E000120102F47C720A43A1681A64226B114323
:1041F000626802F07F021143E268B2F5806F40F01E
:10420000A380554A93425CD08032934259D0803289
:10421000934256D08032934253D08032934250D052
:10422000803293424DD0803293424AD080329342C2
:1042300047D08032934244D08032934241D0803282
:1042400093423ED0803293423BD08032934238D06A
:104250008032934235D08032934232D080329342C2
:104260002FD03E4A93422CD08032934229D08032C4
:10427000934226D08032934223D08032934220D082
:10428000803293421DD0803293421AD080329342C2
:1042900017D08032934214D08032934211D08032B2
:1042A00093420ED0803293420BD0834209D002F564
:1042B0008072934205D08032934202D08032934282
:1042C00001D141F480615A6C8342656B22F0434214
:1042D00022F47F1222F4F35222F01F0242EA050276
:1042E00042EA01025A644FF000029A6414D01C4A58
:1042F000934211D0803293420ED0803293420BD041
:10430000184A934208D08032934205D080329342BB
:1043100002D08032934202D100225A659A65002071
:10432000D8670123A065256584F854300BE0FFF7BA
:10433000D3FD401B05287FF6D6AE1023A3650323CB
:1043400084F85430012038BDB2F5007F08BF41F435
:104350000071B8E750160240500000525010024061
:10436000D01602405006005238B50446FFF7B4FD9F
:104370000546002C4BD02268536943F00603536175
:1043800023685A6912F0010237D11A605A611A641F
:104390005A649A64DA641A65DA671E4A934214D042
:1043A0008032934211D0803293420ED080329342B9
:1043B0000BD0194A934208D08032934205D0803204
:1043C000934202D08032934202D100225A659A650C
:1043D0004FF4FE42DA600023E26DC4E91833C4E909
:1043E0001A33C4E91C3302B1E365A36500202365D9
:1043F00084F8543084F84C300AE0FFF76DFD401B20
:104400000528BDD91023A365032384F85430012067
:1044100038BD00BF501602405006005230B500288B
:1044200034D090F84C40012C32D0012480F84C401C
:1044300090F85440012C4FF0000423D1022580F85D
:10444000545084650468A56C63F30F054FF4FE4374
:10445000A564E360E1642265636943F4BA43636180
:10446000436E1BB1636943F400736361036F1BB157
:10447000636943F4005363616369002043F00103FF
:10448000636130BD402380F84C4083650120F8E72C
:104490000220F6E738B50446FFF71EFD054644B195
:1044A00094F85430022B06D02023A365002384F80F
:1044B0004C30012038BD2268536943F00403536136
:1044C000052384F8543023681A69900419D55A6971
:1044D000216D42F0020209065A614FF0040284F88D
:1044E00054204FF4FE42DA604FF0010284F8542069
:1044F00003D5616F0A7300229A64002084F84C008F
:10450000D8E7FFF7E9FC401B0528DCD9A36D43F091
:104510001003A365032384F85430236D1D06C5D50D
:10452000636F01221A73C1E728B190F85430022B4F
:1045300003D020238365012070470268042380F89C
:1045400054300020536943F4005343F00403536193
:1045500070470368012123F47F6222F00F0210B537
:104560000446D068C3F30B02503AC2F3C41201FAF6
:1045700002F2024200F0AA801A69500508D55A6971
:10458000520505D54FF48062DA60A26D0A43A26538
:104590001A69100509D55A69110506D54FF400624C
:1045A000DA60A26D42F00202A2651A69D20409D54E
:1045B0005A69D00406D54FF48052DA60A26D42F0F9
:1045C0000402A2651A69510409D55A69520406D534
:1045D0004FF48042DA60A26D42F00802A2651A69C7
:1045E000900509D55A69910506D54FF40072DA6035
:1045F000636E0BB12046984723681A6992042DD543
:104600005A6990042AD54FF40052DA6094F8542085
:10461000042A1CD15A69216D22F4005209065A61FC
:104620005A6942F002025A614FF0010284F85420A4
:1046300003D5616F0A7300229A64002384F84C301A
:10464000E36E002B42D02046BDE8104018470523FA
:1046500084F85430236F0BB12046984723681A69B9
:10466000D20518D55A69D00515D5226D110626D563
:10467000DA6F32B99A6C22B90122616F84F8542042
:104680000A734FF44072DA60002384F84C30236ED2
:104690000BB120469847A36DC3B12268536943F01C
:1046A000020353610123226D84F85430120601D5B0
:1046B000626F1373002384F84C30A36EC1E79A6CC9
:1046C000002ADED1012284F85420DAE710BD90F8E8
:1046D00054007047806D7047D0B1CB0101D40020E9
:1046E00070470368012023F47F62C3F30B03503B40
:1046F00022F00F02C3F3C41300FA03F300F1807039
:10470000884351680CBF0B4321EA03035360E6E77B
:104710000120704741EA0203034318B949B9002A4E
:1047200018BF10465840B0F5803F34BF002001202C
:1047300070470846F6E750B190F8203059B992B169
:1047400092F82000984214BF03200020704741B126
:1047500091F82030F3E791F820109942EFD0022031
:104760007047084670471046704700002DE9F04337
:10477000D2F800C0866861B34FF6FC7E0024DFF8F3
:1047800094804FEA8C097746234625460F40B54270
:104790003CD09F4226D12E4606E0056891B905EA35
:1047A00007030131B142F8D1016896606FF30F0140
:1047B0000B430C43D36053F82C305460FBB90020FA
:1047C000BDE8F08308EB030405EA0E0565591C46B5
:1047D000E5E70C460B46DFF83CE04FEA8C084FF665
:1047E000FC77DFE701681DB901EA0E030135CEE76A
:1047F00009EB030401EA080161581C46F4E723F0C1
:1048000003031B041B0C0B431361D8E79F42CBD05F
:104810000120D5E70000FFFF830706D509B1064B4D
:104820000B600AB107231360704709B1034B0B609B
:10483000002AF9D00523F6E7000001FE000001F888
:1048400038B50446FFF748FB0546002C00F0B2805F
:104850000023226884F84C30022384F854305369D2
:1048600043F00603536123685A69D20700F1978029
:10487000D4E90E1250481143504A93425CD0803222
:10488000934259D08032934256D08032934253D0D3
:104890008032934250D0803293424DD08032934246
:1048A0004AD08032934247D08032934244D0803203
:1048B000934241D0803293423ED0803293423BD0EB
:1048C0008032934238D08032934235D08032934246
:1048D00032D0803293422FD0394A93422CD080324A
:1048E000934229D08032934226D08032934223D003
:1048F0008032934220D0803293421DD08032934246
:104900001AD08032934217D08032934214D0803232
:10491000934211D0803293420ED0803293420BD01A
:10492000834209D002F58072934205D080329342CF
:1049300002D08032934201D1226C11435A698342E2
:1049400022F4430242EA0102616C5A614FF0000214
:104950001A6459649A64DA641A6514D0194A934245
:1049600011D0803293420ED0803293420BD0164A3F
:10497000934208D08032934205D08032934202D0D5
:104980008032934202D100225A659A650020D8678E
:10499000A36CA0652365012384F854300BE0FFF776
:1049A0009BFA401B05287FF65EAF1023A365032307
:1049B00084F85430012038BD501602405000005297
:1049C00050100240D016024050060052034637B540
:1049D00000284BD0426F002A48D090F85410046849
:1049E0000129CDB2606903D0022D3AD1C10338D577
:1049F00093F854100129CDB22CD193F84C10022019
:104A000001292CD0002183F8540083F84C501073F6
:104A100099651161616941F4BA416161596E19B1D9
:104A2000616941F4007161611B6F1BB1636943F4FB
:104A300000536361156801A90022286AFFF7ECFEA4
:104A40002B0C25F003051B042D0423602D0C019B6A
:104A50001D43E5676369002043F00103636103B010
:104A600030BD40229A65002283F84C200120F6E7F1
:104A7000F0B5002800F09480002900F09180C3690F
:104A8000456902681D43C36B12F0600445EA0305E3
:104A9000036945EA0305836945EA03050D6010D003
:104AA000836AC66A013B876B1B053E4303F07C7338
:104AB0003343466A013E360106F47C7633432B438A
:104AC0000B604368056B23F4C0739B059B0D2B4360
:104AD000C568B5F5806F4B603ED114B143F4806377
:104AE0004B604D68436B446C1D434D6044B1836C17
:104AF000066C1B04344303F47C132C4323434B60A8
:104B0000B0F8685012F002068D601BD0C36C5C1EBA
:104B1000244B03EA0443046D2B43002C446DB8BFBF
:104B200043F08053002C846DB8BF43F00053002C39
:104B3000C46DB8BF43F08043002C8B60BCBF43F012
:104B400000438B60036ECB60436E0B6156B942F439
:104B5000A06200200A62F0BDB5F5007FC1D143F428
:104B60000073BDE7036D42F4E062456D002B0E4C0F
:104B7000B8BF5B42002DB8BF6D42C3F30C0304EA1B
:104B8000054423434B61836DC06D002BB8BF5B426E
:104B900000289BB2B8BF404243EA00438B61D8E78C
:104BA0000120D8E70000FF070000FF1F2DE9F041BA
:104BB0000E4688B01546044628B122B14369012B40
:104BC00005D104232361012008B0BDE8F081D0F8AD
:104BD00000804046FFF79EFD08B10523F2E74046FE
:104BE000FFF7A9FD0028ECD1022702AA01A927732B
:104BF0002061286AFFF710FEB8F1000F13D13EB90B
:104C00000127256000200123A76020612373DBE7D3
:104C100025F00305019B26602D042D0C1D43029BEE
:104C200046F82350EEE7029F76B928F00308019B6F
:104C30004FEA08484FEA184848EA030345F8273086
:104C40002560A3685F1CDDE703AA31462046039771
:104C5000FFF78CFDB8B94FF6FC7CA3680598019965
:104C600005EA0C02984242EA010209D1636823B1C5
:104C700003EA0C030B4345F8273046F82720E0E70A
:104C800056F82730F7E706239CE7F0B5044689B0CD
:104C900018B1066826B902232361012009B0F0BDCE
:104CA00045681DB1AE421FD00423F5E74369012BCF
:104CB000FAD0022302AA01A903730561306AFFF743
:104CC000ABFD029F03AA294620460397FFF74EFD3E
:104CD0004FF6FC73019A33401343069A42F827308B
:104CE00001232561666023730020D7E770B169B1A5
:104CF00090F8543090F85420DBB2022A01D0052BF2
:104D000006D140238365002380F84C300120704792
:104D10000B7B022B02D101230B61F7E70368154AD5
:104D200093421AD08032934217D08032934214D0EB
:104D30008032934211D0104A93420ED08032934277
:104D40000BD08032934208D08032934205D00B685A
:104D50001B6A9B0701D50323DEE7026D4B68812A9E
:104D600002D11BB90423D7E7002BFBD141670020F8
:104D7000704700BF50160240500600520368186981
:104D8000C0F30740704700004E4B03EA90232DE923
:104D9000F74F4FF00F0901934FF0B04400230A681A
:104DA00032FA03F502D103B0BDE8F08F012505FA10
:104DB00003F818EA020200F083804E6803274FEAE6
:104DC000430E06F0030507FA0EFC6F1E6FEA0C0C8B
:104DD000012F32D8876807EA0C0ACF6807FA0EF766
:104DE00047EA0A078760476827EA0808C6F30017FA
:104DF0009F4047EA08074760C768022D07EA0C088A
:104E00008F6807FA0EF747EA0807C76017D14FEA1D
:104E1000D30803F0070A00EB88084FEA8A0AD8F89B
:104E2000207009FA0AFB27EA0B0B0F6907FA0AF749
:104E300047EA0B07C8F8207001E0032DDCD10768B2
:104E400005FA0EF516F4403F07EA0C0745EA070598
:104E5000056035D023F0030703F0030516F4801F27
:104E600007F1B0484FEA8505019FD8F830C509FA27
:104E700005FE07FA05F56FEA02072CEA0E0C45EA73
:104E80000C05C8F8305525680CBF3D40154316F495
:104E9000001F256065680CBF3D40154316F4003FB8
:104EA0006560D4F884500CBF3D401543F603C4F848
:104EB0008450D4F8805054BF3D401543C4F880500E
:104EC00001336CE77FFF29002DE9F04F314F0023BC
:104ED0004FF001084FF00F0E07EA90274FF003093B
:104EE0004FF0B04231FA03F401D1BDE8F08F08FA77
:104EF00003FC1CEA01064BD023F0030403F0030576
:104F000004F1B044AD00D4F830A50EFA05FB07FA61
:104F100005F504F580640BEA0A0A554519D1D2F863
:104F2000805025EA0605C2F88050D2F8845025EA60
:104F30000605C2F88450556825EA060555601568CF
:104F400025EA06051560D4F8305125EA0B05C4F8AA
:104F500030515C000568DE0809FA04F400EB8606AF
:104F60002543056003F00705D6F820A0AD000EFA32
:104F700005F52AEA05053562856825EA0405856098
:104F8000456825EA0C054560C56825EA0404C46047
:104F90000133A7E77FFF29000369194214BF0120ED
:104FA000002070470AB181617047816270470368D1
:104FB0009A69910701D500229A629A69D20703D4AF
:104FC0009A6942F001029A617047000030B5039D72
:104FD000C1F3090104682B43606843EA0243054AB0
:104FE0000B4342EA555223F0004320EA02000343F8
:104FF000636030BDFF63FF03204B426B9A4201F0B8
:10500000010370B50DB201F002041FD01C4EB24274
:105010001CD01C4EB24219D0002DC3F10003B4BF06
:10502000B822002203F0F20313430CB143F0F4035F
:10503000102902D143F0900303E0202901D143F06D
:10504000200301680A6813430B6070BD002DC3F193
:105050000003B4BFB822002203F0F20313430CB1E3
:1050600043F0F4031029E5D0202902D143F0600376
:10507000E7E7402908BF43F04003E2E72D5F00085F
:10508000D5620008055E000811F0010307D090F812
:10509000413003F02803282B14BFF22342238A0750
:1050A00009D590F8412002F02802282A0CBF43F0CD
:1050B000440343F0F4030A04016848BF43F0B80313
:1050C0000A6822EA03030B60704703682DE9F04188
:1050D0009C6905460F46164614F010046FD0002454
:1050E0001022A046DA612B689A69900661D4B8F163
:1050F000000F35D044F0040401202E68B369D905AF
:1051000005D54FF4807244F001040120F2615A0584
:1051100005D54FF4806244F008040120F2619B053C
:105120004FD54FF4007344F00204F3612846FFF7B3
:105130003EFF7368012023F0FF7323F48B3323F4C5
:10514000FF7323F0010373606B6C23436B642023B4
:1051500085F84130002385F8423085F8403032E050
:105160007A1CC1D0FEF7B8FE801BB84201D8002FD0
:10517000B9D12B68596895F842209869D2B20004D9
:105180000AD5490408D4202A06D05A6842F480423D
:105190005A60FEF7A1FE06462B689B699B06A2D4C7
:1051A000FEF79AFE801B1928F6D920244FF001083B
:1051B00099E7B8F1000F9DD12022DA619AE72046E5
:1051C0009BE70028B2D1BDE8F08170B504460D46DA
:1051D000164623689B699B0701D500201FE03246D5
:1051E00029462046FFF771FFC0B96A1CF1D0FEF7CF
:1051F00073FE801BA84201D8002DEAD123689B6969
:1052000013F00203E5D1626C84F8403042F02002D2
:105210006264202284F8412084F84230012070BD6D
:105220002DE9F041DDF8188004460F4616461D466C
:1052300023689B6937EA03030CBF01230023B342B1
:1052400001D0002025E0424629462046FFF73DFFD9
:10525000F0B96B1CECD0FEF73FFEA0EB0800A842B3
:1052600001D8002DE4D123689B6937EA03030CBF02
:1052700001230023B342DBD1636C43F0200363645A
:10528000202384F84130002384F8423084F84030F1
:105290000120BDE8F08170B504460D46164623682E
:1052A0009B699B0601D500201DE032462946204619
:1052B000FFF70BFFB0B9FEF70FFE801BA84201D825
:1052C000002DECD123689B6913F02003E7D1626CB9
:1052D00084F8403042F020026264202284F84120A9
:1052E00084F84230012070BD2DE9F84305460E4692
:1052F000174600244FF01008DFF88C902B689B694C
:105300005B0700D414B12046BDE8F8833A46314625
:105310002846FFF7DAFE2B6804469A6990060CD4FB
:10532000003C18BF0124FEF7D7FDC01BB04201D8D6
:10533000002EE3D1D4B10124E0E79CB99A699A69BF
:10534000D10611D504222021C3F81C806A64D961DA
:105350005A6802EA09025A6085F8411085F840400F
:1053600085F842400124DEE76C64DCE72B689B692A
:105370005A07C3D46B6C85F8404043F020036B643C
:10538000202385F84130D6E700E800FE10B504463A
:1053900000284ED090F8413003F0FF021BB980F88E
:1053A0004020FBF795FC242384F8413023681A68D9
:1053B00022F001021A60626822F070621A619A6833
:1053C00022F400429A60D4E90221012906D142F474
:1053D00000429A605A6822F4006207E042F40442F4
:1053E00002299A60F6D15A6842F400625A6000209D
:1053F0005A6842F0007242F400425A60DA6822F4BD
:105400000042DA60D4E904210A43A16942EA012298
:10541000DA60D4E907210A431A601A6842F00102EF
:105420001A602023606484F84130206384F84200CD
:1054300010BD0120FCE700002DE9F347984690F8E5
:10544000413004460E46202B91460A9F40F086804C
:1054500090F84030012B00F081804FF0010A80F875
:1054600040A0FEF739FD19230546009052464FF43F
:1054700000412046FFF7D4FE18B1012002B0BDE87C
:10548000F0872123C4F82490606384F8413010230E
:1054900084F842306064A4F82A80638D9BB2FF2BAD
:1054A0002F4B26D9FF22228500934FF0807331467F
:1054B0002046FFF78BFD638D2A46394620469BB276
:1054C000FBB9FFF7E8FE0028D7D123682021D96176
:1054D0005A6822F0FF7222F48B3222F4FF7222F01B
:1054E00001025A6084F8411084F8400084F84200B8
:1054F000C4E7628D92B2228500934FF00073D2B25E
:10550000D5E7FFF762FE0028B7D1636A226813F877
:10551000011B91626362638D228D013B013A9BB254
:1055200092B26385638D22859BB2002BC3D0002A83
:10553000C1D13B46802120460095FFF771FE00282F
:105540009BD1638D9BB2FF2B03D9FF222285009054
:10555000ABE7628D92B222850090CEE702208DE704
:10556000002000802DE9F347984690F8413004462A
:105570000E46202B91460A9F40F0878090F84030DD
:10558000012B00F082804FF0010A80F840A0FEF766
:10559000A3FC19230546009052464FF400412046D3
:1055A000FFF73EFE18B1012002B0BDE8F0872223CC
:1055B000C4F82490606384F84130102384F84230AA
:1055C0006064A4F82A80638D9BB2FF2B304B26D9F0
:1055D000FF22228500934FF0807331462046FFF76B
:1055E000F5FC638D2A46394620469BB2FBB9FFF78E
:1055F00052FE0028D7D123682021D9615A6822F0B1
:10560000FF7222F48B3222F4FF7222F001025A6000
:1056100084F8411084F8400084F84200C4E7628DA9
:1056200092B2228500934FF00073D2B2D5E7FFF714
:105630005BFE0028B7D123685A6A636A1A70636AEE
:10564000228D0133013A6362638D92B2013B228560
:105650009BB26385638D9BB2002BC2D0002AC0D160
:105660003B46802120460095FFF7DAFD00289AD1BD
:10567000638D9BB2FF2B03D9FF2222850090AAE7FE
:10568000628D92B222850090CDE702208CE700BFA8
:10569000002400802DE9F34190F8415004460F4664
:1056A000202D40F0A0800668B56915F4004540F053
:1056B0009A8090F840C0BCF1010F00F094804FF048
:1056C000010C426280F840C04FF0220C80F841C0CB
:1056D0004FF0100C80F842C045644385434BC362D1
:1056E000434B4363438D9BB2FF2B37D9FF254FF0CC
:1056F00080780585E06B00284CD03E4B03663E4B1E
:10570000836600234366C366036D1B063CD5436F67
:105710005BB31B6824369D60C3E90362FFF756F94B
:105720000546002842D1354B3946268D2046009348
:10573000434694F82820FFF749FC638D102120464A
:105740009B1B84F840509BB26385FFF755FC226891
:10575000136843F400431360002012E0458DADB29E
:10576000058585B34FF00078C4E7202284F84030E7
:1057700084F8412084F84230626C42F08002626416
:10578000012002B0BDE8F0812B4606F12401FEF7AE
:1057900045FEC5E7202384F8400084F8413084F8B2
:1057A0004200636C43F080036364E9E72023002236
:1057B00084F8413084F84220636C84F8402043F040
:1057C00010036364DCE70E4B2A4643630B4B0093E4
:1057D0004FF00073FFF7FAFB0221204684F8405097
:1057E000FFF70AFCB8E70220CBE700BF0000FFFF8D
:1057F0002D5F00084360000831600008002400802D
:10580000E35C00082DE9F0431D4685B00023044603
:105810001746039390F84130202B72D103689B699F
:1058200013F400436DD190F84020012A69D0C1F3F0
:105830000906012246F0007880F84020242248F42E
:10584000205880F841204364E3682268012B0ABF96
:1058500046F00073434643F400535360FEF73CFBAD
:105860008146226893699269C3F34013C2F3001220
:10587000134316D023689A692B46CDF8009012F096
:10588000100224D120212046FFF7CAFCE8B92023CA
:105890002268D36184F8413084F8400005B0BDE847
:1058A000F0836B1CDDD0FEF717FBA0EB0900A842CC
:1058B00001D8002DD5D1202384F84130636C43F00A
:1058C00020036364002384F840300120E6E70022CF
:1058D00020212046FFF7A4FC0028F6D123681022DF
:1058E000DA612022DA61039B01330393039BBB42FD
:1058F000AAD384F84120636C84F8400013436364A6
:10590000E3E70220CAE70268436B9169126803B1BA
:1059100018477047704738B5002580F8425090F816
:105920004130212B4FF0200380F841300AD1112360
:10593000012145630363FFF7A7FB80F84050FFF7A1
:10594000E9FF38BD1223022145630363FFF79CFB87
:1059500080F84050FBF77AFBF3E77047704708B5D3
:10596000036800211A6880F84210510415D51A689E
:1059700022F480421A6090F84130292B13D1282359
:10598000012180F8413021230363FFF77DFB0023D1
:1059900080F84030FFF7E1FF08BD1204EBD51A682C
:1059A00022F40042E6E790F841302A2BF4D1282374
:1059B000022180F8413022230363FFF765FB0023B7
:1059C00080F84030FFF7CAFFE6E7704790F84120C3
:1059D00002F02802282AF8B5036835D19E69C2680A
:1059E0009D69C6F30046022A99684FEA1545DF68AB
:1059F00005F0FE051FD185EAD115C1F3090215F0A6
:105A000006050ED1816C01318164816C022907D1B8
:105A100008218564D96180F840503146FFF7D5FFF1
:105A2000F8BD4FF40041FFF72FFB002307F0FE0203
:105A300080F84030F1E74FF40041FFF725FB0023E9
:105A40002A4680F84030E8E70822DA61002380F82F
:105A50004030E5E77047000008B5164B2022C362CE
:105A600000230363436380F8412080F842304B07F2
:105A700012D503685A6A436A1A70436A0133436253
:105A8000038D4BB1013B0385438D013B9BB24385A5
:105A9000436C43F00403436448F20301FFF7F4FA54
:105AA00003681022DA61002380F84030FFF7D2FF4C
:105AB00008BD00BF0000FFFF704770477047704788
:105AC00090F84120602A4FF0000208B508D120214B
:105AD00080F8402080F841100263FFF7F0FF08BD16
:105AE000026380F84020FFF7E9FFF8E770B5002275
:105AF00090F841303C4D044680F84220283BC56276
:105B00004285022B426C42EA010242642AD80321F8
:105B1000FFF7BAFA282380F84130344BA06B636357
:105B2000236B002841D0112B01D0212B3DD12368BC
:105B30001A68510403D51A6822F480421A60FEF7ED
:105B4000C6FD01282CD02A4BA06BC366002384F825
:105B50004030FEF7E9FC002845D0A06BC36EBDE8DD
:105B60007040184748F20301FFF78EFAFFF71FFA5B
:105B700090F84130602B11D0202380F84130036829
:105B80009A6995060AD59A69D00605D51022DA6178
:105B9000626C42F0040262642022DA610023BDE7F5
:105BA0002046BDE87040FFF78BBFE06B0028F7D0C0
:105BB000122B01D0222BF3D123681A68120403D5CB
:105BC0001A6822F400421A60FEF781FD0128E7D02E
:105BD000074BE06BC366002384F84030FEF7A4FC5B
:105BE00008B1E06BBAE770BD0000FFFFEF6300088B
:105BF0000165000873B52023056804460E46EB6175
:105C000090F84130212B36D10121FFF73DFA1123C5
:105C100023636B68F20623F0FF7323F48B3323F4C2
:105C2000FF7323F001036B604FF000036363A3F580
:105C30008033E36205D51023EB61636C43F004030A
:105C4000636494F84130602B05D1730703D56B6A08
:105C5000DBB20193019B2046FFF7A9F9636C94F82E
:105C60004120602A00D07BB1616C204602B0BDE8C3
:105C70007040FFF73BBF90F84130222BC9D1022181
:105C8000FFF702FA1223C3E794F84120212A12D128
:105C9000202284F8403084F84120236394F8422085
:105CA00084F84230402A03D1FFF706FF02B070BDEE
:105CB000FFF730FEFAE794F84120222AF6D120229D
:105CC00084F8403084F84120236394F8422084F81B
:105CD0004230402A02D1FFF7F0FEE7E7FBF7B6F9C2
:105CE000E4E773B590F8403004460D461646012BA4
:105CF00000F086800123CA0680F8403017D5F306ED
:105D000015D503681022DA61436C43F00403436441
:105D1000FFF74DF9AA0605D5B30603D52946204657
:105D2000FFF768FF002084F8400002B070BD6807EC
:105D300012D5710710D5236825F004055A6A636AE5
:105D40001A70636A01336362238D013B2385638D7F
:105D5000013B9BB26385DDE7AA0707D5B30705D5ED
:105D6000636A226813F8011B9162ECE7280632D5BA
:105D7000710630D5638D22689BB203B3208DF0B9D4
:105D80005168638DC1F309019BB2FF2B08D9FF2233
:105D90004FF08073228500902046FFF717F9B9E78E
:105DA000628DE36A92B213F5803F2285D2B202D0AF
:105DB000E36A0090F0E74FF000730090ECE753685F
:105DC0009A0103D42046FFF7A6FDA3E74021204611
:105DD000FFF78CFE9EE76B069CD570069AD5638D07
:105DE0009BB2002BF2D123685A68910192D4E26AE7
:105DF00012F5803FE6D15A6842F480425A6089E742
:105E0000022092E713B590F840300446012B00F0D1
:105E10008680012380F84030CB0612D5D30610D5FA
:105E2000036810222021DA61436C43F004034364C9
:105E3000FFF7E2F8FFF7BBF8002084F8400002B05B
:105E400010BD880708D5930706D52368226D9A628E
:105E50004FF0FF332365EFE7080636D5530634D5F8
:105E600001212046FFF710F91021FFF7C5F8638DD7
:105E70009BB233B3638D9BB2FF2B18D9FF22E16C29
:105E80000023228500934FF0807389B2FFF79EF8BC
:105E9000638D228D9B1A9BB2638594F84120236801
:105EA000222A1A6830D142F400421A60C4E7628D97
:105EB0000023E16C92B222850093D2B24FF00073BE
:105EC000E3E74021FFF712FEB6E748061FD5530669
:105ED0001DD501212046FFF7D7F81021FFF78CF8D8
:105EE00094F841100F4A104B222918BF1346628DB7
:105EF00092B2FF2A03D9FF22E16C2285C2E7628DAC
:105F0000E16C92B22285D7E742F48042CDE7880661
:105F100092D5930690D52046FFF76CFE8CE70220C1
:105F20008DE700BF002000800024008073B590F84A
:105F300040300446012B79D0012380F84030CB0655
:105F400012D5D60610D5036810222021DA61436CE1
:105F500043F004034364FFF74FF8FFF728F80020ED
:105F600084F8400002B070BD0D0642D5500640D501
:105F700025682B6823F040032B60638D9BB263B3CD
:105F80006968638DC1F309019BB2FF2B1AD9FF2306
:105F900023854FF080730022268D2046009294F8CE
:105FA0002820FFF713F8638D9B1B9BB2638594F841
:105FB0004130222B2B680CBF43F4004343F4804351
:105FC0002B60CCE7638D2385E36A13F5803F01D016
:105FD000E36AE0E74FF00073DDE76B689A0103D4F2
:105FE0002046FFF798FCBAE740212046FFF77EFDE8
:105FF000B5E74B0612D5560610D5638D9BB2002B24
:10600000F2D123685A689501A9D4E26A12F5803F5B
:10601000E6D15A6842F480425A60A0E788069ED5CD
:1060200093069CD52046FFF7E5FD98E7022099E707
:10603000C06D10210268536843F400435360FFF7BA
:1060400055BD38B5C46D21680B6823F400430B605F
:10605000638D9BB22BB920212046BDE83840FEF766
:10606000CBBF238D626A1A44638D9BB26262FF2BA1
:1060700016D8638D9BB2E06B2385056D2D0617D571
:10608000456F7DB12D682431AB60C5E90312FEF781
:106090009DFC58B120461021BDE83840FFF726BDD1
:1060A000FF23E8E710212046FFF720FD4021D3E73A
:1060B0002431FEF7B3F9ECE7036899691A6810B464
:1060C000CC0508D5140606D5446C44F0010444649C
:1060D0004FF48074DC614C0508D5140606D5446C79
:1060E00044F0080444644FF48064DC61890508D5F9
:1060F000120606D5426C42F0020242644FF400726E
:10610000DA61416C11F00B0F03D05DF8044BFFF71F
:10611000EDBC5DF8044B70472DE9F0410568202285
:1061200004460E46D5F80080C76A90F84130EA610F
:10613000213B092B0CD8DFE803F0056F0B0B0B0B91
:106140000B75056F48F20101FEF79EFF21232363C3
:106150006B68204643F400436B606B6823F0FF7369
:1061600023F48B3323F4FF7323F001036B60FEF7FA
:106170001EFF18F4804F5BD02B68A06B23F4804384
:106180002B6030B103689D6CFEF7F8FD0544ADB29D
:106190006585720710D5236826F004065A6A636A7B
:1061A0001A70636A01336362238D2BB1013B23852F
:1061B000638D013B9BB26385638D9BB21BB1636CA6
:1061C00043F004036364F30611D518F0100F0ED0EA
:1061D000638D9BB2002B45D194F84130282B30D1F0
:1061E000B7F1007F2DD131462046FFF735FC002363
:1061F00084F84230656C6363002D42D0616C2046A8
:10620000FFF774FC94F84130282B4CD131462046DE
:10621000BDE8F041FFF720BC48F20201FEF734FF71
:10622000222394E748F20301FEF72EFF00238EE7B6
:1062300018F4004FADD02B68E06B23F400432B60C3
:106240009FE794F841202368292A4FF01002DA6171
:10625000CDD117F5803FCAD02046FEF7A8FEFFF744
:106260007EFBC4E723681022DA61636C43F0040309
:10627000636437F08073BAD1616C2046FFF736FC57
:10628000B5E7E36A13F5803F0FD02046FFF767FBC1
:106290000F4B204684F84050E362202384F84130BD
:1062A0002563FFF7D7FBBDE8F08194F84130204625
:1062B00084F84050222B4FF0200384F841302563AE
:1062C00002D1FFF74BFBEEE7FFF747FBEBE700BF21
:1062D0000000FFFF2DE9F04190F8403004460E46E3
:1062E000C76A012B00F0818001238D0680F84030C1
:1062F00008D5930606D5FFF70FFF002084F840006D
:10630000BDE8F081F50668D5D00666D5C2F38038C1
:1063100002F4004558EA05035BD0E06BC8B145B113
:1063200003689D6CFEF72AFD10FA85F5B5FA85F530
:106330006D09A06B78B9012D2BD194F84130282B31
:1063400016D1B7F1007F13D131462046FFF784FB09
:10635000D3E70546EDE7B8F1000FECD00368D3F8BA
:106360004880FEF70BFD10FA88F00028E3D1E4E73F
:1063700094F841202368292A4FF01002DA61BCD139
:1063800017F5803FB9D02046FEF711FEFFF7E7FA78
:10639000B3E723681022DA6137F08072636C43F050
:1063A0000403636494F84130DBB2A6D1213B092B8E
:1063B00008D8DFE803F0050C070707070707050CF7
:1063C00021232363616C2046FFF790FB95E722238E
:1063D000F7E723681022DA618FE731078DD51307BD
:1063E0008BD52046FFF7F2FA87E7022088E770B5E1
:1063F00090F8406004460B46C56A012E7ED0012607
:1064000080F840608E0607D5960605D5FFF784FE16
:10641000002084F8400070BDD90630D5D6062ED5B0
:10642000628D92B2E2B994F84120282A07D1B5F1E1
:10643000007F04D119462046FFF70EFBE8E794F8E9
:1064400041202368292A4FF01002DA61E0D115F5C6
:10645000803FDDD02046FEF7AAFDFFF780FAD7E7A0
:1064600023681022DA61636C43F00403636435F03F
:106470008073CDD1616C2046FFF738FBC8E7580721
:106480001BD5510719D5638D9BB26BB123685A6A2E
:10649000636A1A70636A01336362238D013B23854B
:1064A000638D013B9BB26385638D9BB2002BAFD1A3
:1064B00015F5803FACD02046CFE71E0705D5100765
:1064C00003D52046FFF782FAA2E79907A0D59307E4
:1064D0009ED5638D9BB26BB1636A226813F8011B72
:1064E00091626362638D013B9BB26385238D013BA7
:1064F00023858DE735F080738AD1DCE702208AE7B7
:10650000C06D836B0BB10022DA66C36B0BB1002246
:10651000DA66FFF7D5BA10B590F841200346202A75
:10652000D4B21CD190F84020012A18D0242280F83F
:1065300041200268106820F001001060106820F40B
:10654000805010601068014300201160116841F014
:106550000101116083F8414083F8400010BD022022
:10656000FCE710B590F841200346202AD4B21BD195
:1065700090F84020012A17D0242280F84120026898
:10658000106820F001001060106820F4706040EA8C
:10659000012100201160116841F00101116083F8B0
:1065A000414083F8400010BD0220FCE7F7B50446E7
:1065B00018B390F89534056803F0FF021BB980F812
:1065C000942405F025FF0323206884F89534314B8B
:1065D0009D4204F1040504BF0023A37104F06AFB8B
:1065E000237C8DF80030206895E80E0004F0B4FAA2
:1065F000014630B1022384F895340125284603B0C2
:10660000F0BD206804F05CFB0028F3D1267904F18A
:10661000140301270246C1B224338E4220D8002140
:1066200004F515730A46C8B22433864226D8237C63
:106630008DF80030206895E80E0004F0BBFB05469D
:106640000028D7D10123607484F89534237B012B73
:1066500002D1204600F0FFFC206804F0F1FECDE7F7
:1066600023F80A0C013003F8237C03F8241C03F8F8
:10667000202C43F8142C43E90722CCE7013103F81E
:10668000232C03F8240C03F8202C43F8142C43E9A2
:106690000722C8E70000084010B50446006894F8D7
:1066A0009434012B15D0012384F89434C3685B061D
:1066B00006D5637B012B03D1836B43F48033836363
:1066C00004F0F2FA206804F0ADFE002084F894048F
:1066D00010BD0220FCE710B590F894240446012A6E
:1066E0000AD00122417480F89424006804F08AFEE4
:1066F000002084F8940410BD0220FCE770B501F07E
:106700000F0611F0800F05464FF0240006EBC6047B
:106710004FEA84041ED004F1140100FB065001244A
:10672000294444758A604A780E700B7102B14E8319
:10673000022B04BF00234B7195F89434012B12D027
:106740000123286885F8943404F01BFC002085F8A8
:10675000940470BD04F5157100FB06500024294413
:1067600080F85542DEE70220F3E710B5044601F059
:106770000F0011F0800F4FF0240200EBC0034FEA2E
:10678000830315D003F1140102FB004201232144CD
:106790005375087094F89434012B12D001232068AB
:1067A00084F8943404F02CFC002084F8940410BD88
:1067B00003F5157102FB00420023214482F8553293
:1067C000E7E70220F3E770B501F00F052424164631
:1067D00004FB050104FB050401F5157184F854520E
:1067E000C4E998230023C4F8683284F855328279CA
:1067F0000068012A08BFC4F8706204F0ADFC0020F4
:1068000070BD01F00F01242303FB0100D0F86802E2
:10681000704770B501F00F052424164604FB0501EE
:1068200004FB050414312575C4E908230023A36281
:1068300001236375827900689A4208BF266304F0D9
:106840008BFC002070BD38B501F00F0503790446BC
:10685000AB422BD311F0800F4FF024001DD000FB72
:106860000541012300FB05401431437501230D70E0
:106870008B7094F894249A421AD0206884F8943447
:1068800004F06CFD2DB904F29C42A179206804F05B
:1068900025FE002084F8940438BD00FB01431A460D
:1068A00003F51571002382F85532DFE70120F3E785
:1068B0000220F1E738B501F00F0203790446934254
:1068C00029D302EBC20311F0800F4FF024004FEAEE
:1068D000830317D003F1140100FB0240012321447C
:1068E000437500250A708D7094F89434012B14D0F0
:1068F0000123206884F8943404F05BFD284684F872
:10690000945438BD03F5157100FB02400023214467
:1069100080F85532E5E70120F3E70220F1E701F0C6
:106920000F030A0603EBC3034FEA83034CBF03F1D3
:10693000140103F515710144006804F0B7BB0000B1
:106940002DE9F04F066889B00446304604F0B4FDE6
:106950000390002840F07181206804F07FFD00283A
:1069600000F06B81D6F8083806F500652068C3F39F
:106970000D23C4F8D43404F071FD870704D52268D0
:10698000536903F002035361206804F067FDC006F9
:106990002DD52268936923F010039361D6F82080E7
:1069A00008F4F01308F00F07B3F5802F40F048818A
:1069B00047F6F07318EA030F14D02423C8F30A191A
:1069C000304603FB07474A46D7F8601204F0A6FC9E
:1069D000D7F860324B44C7F86032D7F868324B447E
:1069E000C7F868322268936943F010039361206806
:1069F00004F034FD010300F13681206804F02EFD1F
:106A000042030DD5274606F5106B4FF0000A2068AB
:106A100004F030FD0490049B2068002B40F0ED81D1
:106A2000206804F01BFD002813DA6B6823F00103D3
:106A30006B6094F8CC34012B40F085820021204615
:106A400084F8CC1400F01AFB2268536903F0004369
:106A50005361206804F002FD00050AD5AB68D90730
:106A600002D5204605F058FD2268536903F40063FF
:106A70005361206804F0F2FC020114D523685A69BE
:106A800002F000625A6194F8CC24002A40F05F8240
:106A90000121204684F8CC145B6DC3F38303C4F852
:106AA000D03400F0EBFA206804F0D8FCC30433D5EE
:106AB0006B681021206823F001036B6004F02EF94D
:106AC000207906F510634FF67F31039A904200F269
:106AD0004282EB6943F00113EB61E37B002B00F092
:106AE0005982D5F8843043F00B03C5F884306B6CC1
:106AF00043F00B036B64D6F8003804F29C42206824
:106B000023F4FE63C6F80038A17904F0E7FC22689C
:106B1000536903F480535361206804F09FFC870499
:106B200016D5206804F0CCFC206804F01FFA276812
:106B3000E07101F073F8E2790146384604F044F858
:106B4000204605F0D6FC2268536903F400535361D4
:106B5000206804F083FC000707D5204605F0C5FC3B
:106B60002268536903F008035361206804F076FC3F
:106B7000010600F11A82206804F070FCC2020CD5F4
:106B8000A04606F5126901272379BB4200F226824E
:106B90002268536903F480135361206804F05EFC9B
:106BA00083022DD594F804E0234606F532600121D6
:106BB0008E4520D993F87CC20268BCF1010F40F0E9
:106BC0002382002A80F22082D4F8D47402F4803226
:106BD00007F00107BA4240F0178283F87BC2B2691E
:106BE00042F08002B2617269170600F10D826B6893
:106BF00043F400736B602268536903F4001353611C
:106C0000206804F02BFC410007D5204605F0B8FCB5
:106C10002268536903F080435361206804F01EFC2E
:106C200042070AD523685D686B0702D5204605F048
:106C3000ABFC226853682B43536009B0BDE8F08F6A
:106C4000B3F5402F7FF4CEAE082204F29C413046CB
:106C5000C8F30A1804F062FB242303FB0747D7F8A4
:106C600068324344BCE606F53068A2460027206837
:106C700004F0F8FB0490049B2068002B3FF4BDAEA9
:106C8000049BDB0778D55FFA87FB594604F0FAFBD3
:106C900010F0010F81461FD001232068C8F808308A
:106CA00000F5306394F806C003EB4713016CBCF1A8
:106CB000010F9A6840F08B8012F0080F07D0B3489C
:106CC000814209D9120407D54FF4004203E012F0C3
:106CD000200F5AD020229A6019F0080F21D00823E3
:106CE000AA49C8F8083023681A6C03F530638A4251
:106CF00003EB4713986804D9010402D54FF4004010
:106D000098602046059205F0D9FB059A9F498A4272
:106D100007D9A179012904D104F29C42206804F02A
:106D2000DDFB19F0100F02D01023C8F8083019F05D
:106D3000020F14D073691A0603D56B6843F480639D
:106D40006B609AF85732012B06D100235946204632
:106D50008AF8573205F00CFC0223C8F8083019F005
:106D6000200F02D02023C8F8083019F4005F03D0A8
:106D70004FF40053C8F80830049B013708F120088D
:106D80000AF1240A5B08049375E7DFF800C2614545
:106D900001D9120498D41A69DAF87432C2F31202D3
:106DA0009B1ACAF868326FB9D4F864222AB904F27F
:106DB0009C42012104F092FB04E0D4F860221A44C2
:106DC000C4F860225946204605F07EFB84E7DFF8D0
:106DD000C0C1614507D111043FF576AF9006F1D5EA
:106DE00020229A60EEE7002FECD1D4F86432002B19
:106DF000E8D104F29C423946DCE7049BDB0740F112
:106E000099805FFA8AF31946059304F044FB10F069
:106E1000010F80461FD001210AF00F026B6B01FAAF
:106E200002F223EA02036B63CBF80810A17901296F
:106E30000DD1D7E9072313443B62BAF1000F06D105
:106E4000636A23B904F29C42206804F047FB059969
:106E5000204605F042FB18F0080F02D00823CBF8BB
:106E6000083018F0100F02D01023CBF8083018F0BB
:106E7000400F02D04023CBF8083018F0020F0FD09B
:106E80005146304603F04AFFFB7D012B05D100231C
:106E900005992046FB7505F06FFB0223CBF80830FF
:106EA000236818F0800F069344D0D7E909329A423C
:106EB00040D8A3EB0208FB69984528BF9846069B7B
:106EC00008F1030803F510634FEA980803EB4A132F
:106ED0000793079B996989B24145D7E9093227D3BE
:106EE00093420BD8069B0AF00F000121D3F83428F7
:106EF000814022EA0102C3F834281BE0A3EB020917
:106F0000FB69059A9945069828BF9946A37900938D
:106F10001FFA89F3396A09F1030804F009F93B6A99
:106F20004FEA98084B443B62BB6A4B44BB62D0E7D4
:106F30009342D7D9049B0AF1010A24370BF1200BA5
:106F40005B08049367E5204605F0F8FA7CE52046E7
:106F500005F0E2FAA7E59960203353F8202C22F4DB
:106F6000001243F8202CC3F8E811D3F8E02122F4F2
:106F70000012C3F8E021D3F8E02142F00062C3F828
:106F8000E021039A013203929FE500BF0A30544F7B
:106F90000A31544F6B6943F4005343F02B036B6188
:106FA0002B6943F00B032B61A5E5B369012704F2BC
:106FB00057284FF0240923F08003B3612379BB42A3
:106FC0007FF6D9AD09FB07F318F80330012B03D185
:106FD000F9B22046FFF7A3FC0137EFE798F83C3001
:106FE000D9F80020012B09D1002A07DA67F07F01C8
:106FF000204688F83B30C9B2FFF791FC013708F111
:10700000240809F12009BFE5013124332030CFE500
:1070100000681204436A70B519B9134383620020F3
:1070200070BD846A4E1E03EB14430024B44205D3A2
:107030003F31134300EB81004360F0E704F140056A
:10704000013400EB85056D6803EB1543EEE703683B
:10705000002059627047012102680346C0F8D81425
:10706000002083F8CC04936943F000639361536D6F
:1070700043F0805343F003035365704770470000AB
:1070800070B5194D0446EB6803F00703062BEB6857
:1070900005D003F01F03181A18BF012070BD23F09C
:1070A0001F030343EB60FCF717FF06466B689A0764
:1070B00004D51D3C012C09D90020EFE7FCF70CFF9B
:1070C000801BB0F57A7FF1D90120E7E7FCF704FFD8
:1070D000054D0446EB68DB03EED4FCF7FDFE001B18
:1070E000B0F57A7FF6D9EFE70048025838B50B4C77
:1070F000636923F0010303436361FCF7EDFE05467A
:1071000063699B0701D5002038BDFCF7E5FE401BF5
:10711000B0F57A7FF4D90120F6E700BF00480258A5
:1071200038B50A4CE36843F08073E360FCF7D4FEA3
:107130000546E3685B0101D5002038BDFCF7CCFEB5
:10714000401BB0F57A7FF4D90120F6E700480258D9
:10715000024AD36843F00063D36070470048025886
:10716000024AD36843F48043D36070470048025812
:1071700010B5234CA06AA26BC0F3053310F47C3F1A
:1071800007EE103A32D0E16A11F4006102D0E16BEF
:10719000C1F3CC0100F0030001282AD002282AD034
:1071A00058BB1748036813F0200304D00068154B40
:1071B000C0F3C100C34007EE903AB8EEC77AC2F3FD
:1071C00008039FED116AF8EEE77A0133C7EE876A8C
:1071D00007EE901AB8EEE77A07EE903AF8EEE77A03
:1071E000E7EE067A66EEA77ABCEEE77A17EE100AAB
:1071F00010BD064BDFE7064BDDE70023DBE700BFF2
:10720000004402580090D0030000003900093D00FE
:1072100000366E0110B5234CA06A226CC0F30553F2
:1072200010F07C7F07EE103A32D0E16A11F4800151
:1072300002D0616CC1F3CC0100F0030001282AD018
:1072400002282AD058BB1748036813F0200304D043
:107250000068154BC0F3C100C34007EE903AB8EE8A
:10726000C77AC2F308039FED116AF8EEE77A01339B
:10727000C7EE876A07EE901AB8EEE77A07EE903A03
:10728000F8EEE77AE7EE067A66EEA77ABCEEE77AE2
:1072900017EE100A10BD064BDFE7064BDDE70023B3
:1072A000DBE700BF004402580090D0030000003923
:1072B00000093D0000366E012DE9F84F4FF00B0834
:1072C000DFF8A8914FF478724FEA400B08FB00F802
:1072D000D9F82C304FF080754FF0007602FA08F2A2
:1072E000074605FA0BF50C4623EA020306FA0BF6ED
:1072F000C9F82C30D9F8003023EA0503C9F800306A
:10730000FCF7EAFD8246D9F8003033427CD122688E
:107310004FEAC70E022A0EF1040C40F08F8060681D
:1073200000287BD1D9F800104C4BC1F3C101CB40F0
:10733000D4F808904A49B3FBF9F38B4274D2494917
:107340008B4273D848498B4288BF08224FF47C7A1D
:10735000464909FA0CF90AFA0EFE8B6A49EA000955
:107360004EF0030E23EA0E0343EA09038B628B6A95
:1073700003F0030383426ED11B20CB6A02FA08F2AA
:1073800000FA08F023EA00031343CB6223695A1E74
:107390006369013B1B0443EA4223E268013A134359
:1073A000A269013A43EA0263314A42F83730236A5C
:1073B0005A1EE369013B43EA02232E4A42F8273072
:1073C0001FB9CB6A43F02003CB62616A81B12A4ABC
:1073D00052F837306FF3CF0343EAC10342F8373036
:1073E000012352F8081C03FA08F30B4342F8083C47
:1073F0001E4C23681D432560FCF76EFD054623687F
:107400001E4215D0002007E0FCF766FDA0EB0A0045
:1074100032287FF678AF0320BDE8F88F174B184964
:10742000022808BF0B4683E718228FE710228DE75A
:10743000FCF752FD401B3228E1D9ECE74FF47C7297
:10744000D9F8283002FA0CF223EA020343F00303CE
:10745000C9F82830D6E70120DEE700BF0090D0034E
:1074600000127A00FF083D007F841E00004402588D
:1074700030440258C04402583444025800093D00C8
:1074800000366E012DE9F843044610B90120BDE82D
:10749000F8839F4B1E699F6A1B6806F0380607F049
:1074A000030703F028580368DD072AD423689807E8
:1074B00000F185802368D90600F1E58023681A076A
:1074C00000F111812368990600F13B8123685D0773
:1074D00000F15C81636A002B40F0B181E36C002B0A
:1074E00040F0DD81606F0028D1D0012304F17401E8
:1074F0000220C4F89430FFF7DFFE003818BF0120E7
:10750000C5E7102E426804D0B8F1000F04D0022F56
:1075100002D1002ACAD1B9E7B2F5803F7C4B03D132
:107520001A6842F480320BE0EAB91A6822F4803219
:107530001A601A6822F400221A601A6822F4802263
:107540001A60FCF7C9FC63680546DFF8C4918BB389
:10755000D9F800309903A9D4FCF7BEFC401B64287D
:10756000F6D9032093E7B2F5A02F08D11A6842F4A8
:1075700080221A601A6822F400221A60D0E7B2F55D
:10758000502F1A6806D142F480221A601A6842F419
:107590000022F2E722F480321A601A6822F4802274
:1075A0001A601A6822F40022CAE7FCF795FC401B17
:1075B0006428D6D8D9F800309A03F6D476E7E36881
:1075C0001EB1B8F1000F2ED06FBB002B3FF45EAFA1
:1075D0004F4A216913683FB9B8F1000F04D003F096
:1075E00018038B427FF452AF136823F019030B4347
:1075F00043F00103136036B91268464BC2F3C1026F
:10760000D340454A1360454B1868FCF723FC00281B
:107610007FF43CAF3E4A6169536823F0FE4343EA7E
:107620000163536046E73A4DDBB12A68216922F0D5
:1076300019020B4313432B606B68626923F0FE430E
:1076400043EA02636B60FCF747FC81462B685B07EB
:107650003FF530AFFCF740FCA0EB09000128F5D95D
:107660007FE72B6823F001032B60FCF735FC814694
:107670002B6858077FF51EAFFCF72EFCA0EB090026
:107680000128F5D96DE7082E236A04D0B8F1000F60
:1076900005D0012F03D1002B7FF410AFF6E61C4D6F
:1076A00083B12B6843F080032B60FCF715FC074681
:1076B0002B68DB053FF502AFFCF70EFCC01B012871
:1076C000F6D94EE72B6823F080032B60FCF704FC0F
:1076D00007462B68D8057FF5F1AEFCF7FDFBC01B14
:1076E0000128F6D93DE7A369094DCBB16B6F43F093
:1076F00001036B67FCF7F0FB07466B6F9A073FF5DA
:10770000E1AEFCF7E9FBC01B0128F6D929E700BF71
:10771000004402580090D003000000240403002419
:107720006B6F23F001036B67FCF7D6FB07466B6FAB
:107730009B077FF5C7AEFCF7CFFBC01B0128F6D92E
:107740000FE7E3695A4D83B12B6843F480532B60F4
:10775000FCF7C2FB07462B6898043FF5B7AEFCF771
:10776000BBFBC01B0128F6D9FBE62B6823F4805332
:107770002B60FCF7B1FB07462B6899047FF5A6AE9A
:10778000FCF7AAFBC01B0128F6D9EAE6494A484D96
:10779000136843F480731360A368012B13D12B6F1C
:1077A00043F001032B6741F28838FCF795FB404F0B
:1077B00005463B6F9A073FF58DAEFCF78DFB401BEE
:1077C0004045F6D9CDE6D3B92B6F41F2883823F086
:1077D00001032B672B6F23F080032B672B6F23F0A4
:1077E00004032B67FCF778FB07462B6F9B077FF59D
:1077F00071AEFCF771FBC01B4045F6D9B1E6052B15
:1078000008D12B6F43F004032B672B6F23F0800309
:107810002B67C4E7852B2B6F06D143F004032B673E
:107820002B6F43F08003F3E723F001032B672B6FEB
:1078300023F004032B672B6F23F08003B2E7182E8D
:1078400022D1012B3FF422AE194BA16C5A6BC2F32B
:10785000CC0291423FF442AEDA6A22F00102DA62CF
:10786000FCF73AFB0546FCF737FBA842FBD0104A71
:10787000A16C536B6FF3CF0343EAC1035363D36A25
:1078800043F00103D36229E6012304F1240100201F
:107890006364FFF711FD00283FF420AEF6E504F124
:1078A0004C010120FFF708FD00283FF41BAEEDE579
:1078B0000044025800480258494B1A6902F0380245
:1078C000102A30B500F08880182A14D0002A40F021
:1078D0008580186810F0200004D01B684148C3F36D
:1078E000C103D8403E4B9B691A0742BF03F00F0308
:1078F000073BD84030BD996A9D6ADC6A15F47C7FED
:10790000C5F305105A6BEDD0C2F3CC0204F00104AC
:1079100001F003016243012907EE902AB8EEE77AED
:1079200050D0022934D000294CD11A68910650D584
:1079300019682C4AC1F3C1011B6BCA40C3F3080389
:1079400007EE902AF8EEE76A07EE900AF8EEE77A7B
:1079500086EEA76A07EE903ADFED236AF8EEE77A43
:10796000E7EE267AB7EE007A77EE877A67EE867AC8
:107970001B4B1B6BC3F34623013307EE103AF8EEA3
:10798000C76A87EEA67AFCEEC77A17EE900AA9E7D7
:1079900007EE900A9FED156AF8EEE77A1B6BC6EECC
:1079A000276A9FED116AC3F3080307EE903AF8EED9
:1079B000E77AE7EE067AB7EE007A77EE877A67EE37
:1079C000A67AD5E707EE900A9FED096AF8EEE77A06
:1079D000E4E7DFED087ACBE7074883E7074881E76C
:1079E000004402580090D00300000039001BB74B40
:1079F0000024744A0000000000366E0100093D00BA
:107A00002DE9F0410D46044610B90120BDE8F08192
:107A10007E4A136803F03F038B427FD323685F07DE
:107A200000F188801E070BD5794960690A6A02F067
:107A30007002904204D90A6A22F0700202430A627C
:107A4000D8060BD57249A0690A6A02F4E062904236
:107A500004D90A6A22F4E06202430A6299060BD54D
:107A60006B49E0690A6A02F4E042904204D90A6A6A
:107A700022F4E04202430A629A070BD56449E068A7
:107A8000CA6902F00F02904204D9CA6922F00F02BB
:107A90000243CA61DF075BD423689E0700F18D8033
:107AA0005A490A6802F03F02AA4200F2948058073D
:107AB00000F19D8019070BD5554960690A6A02F0EB
:107AC0007002904204D20A6A22F0700202430A62F3
:107AD000DA060BD54E49A0690A6A02F4E0629042C8
:107AE00004D20A6A22F4E06202430A629B060BD5C2
:107AF000474AE169136A03F4E043994204D2136AE6
:107B000023F4E0430B431362FFF7D6FE414B1860AA
:107B1000414BBDE8F0411868FCF79CB9136823F0AD
:107B20003F030B431360136803F03F038B427FF462
:107B30006CAF73E7364920690A6A02F00702904287
:107B40007FF670AF0A6A22F0070202430A6269E711
:107B50002F4BA1689A6922F00F020A439A6161686B
:107B60001A6802291CD112F4003F3FF44EAF1A6983
:107B700041F28838264F22F007020A431A61FCF7C7
:107B8000ABF906463B69626803F03803B3EBC20FFA
:107B900082D0FCF7A1F9801B4045F3D9032035E7DB
:107BA000032902D112F0007FDFE7012902D112F48C
:107BB000807FDAE712F0040FD7E71549E068CA6959
:107BC00002F00F029042BFF46BAFCA6922F00F02BD
:107BD0000243CA6164E70A6822F03F022A430A604E
:107BE0000A6802F03F02AA427FF40FAF5FE708493C
:107BF00020690A6A02F007029042BFF45BAF0A6A8A
:107C000022F0070202430A6254E700BF002000523C
:107C100000440258000000240403002407B50A4A67
:107C20006B461068516803C3FFF746FE074BDB69DC
:107C30001A0706D503F00F0308336B4413F8103C02
:107C4000D84003B05DF804FBACDA000800440258E9
:107C500070B5624CFCF740F90546236843F0010318
:107C600023602368580714D5636843F0804363603A
:107C7000FFF7D4FF5A4B024618685A4B9A4277D9FD
:107C800000222261584A1360FCF7E4F840B1012059
:107C900005E0FCF721F9401B0128E2D9032070BD63
:107CA000FCF71AF94D4D044641F288362B6913F062
:107CB000380F57D14D4A136823F03F0343F00103B7
:107CC0001360464CFCF708F9494B054622681340FF
:107CD00023602368990368D4FCF7FEF823680546FF
:107CE00023F0807323603D4C23689A0163D4FCF732
:107CF000F3F82368054623F080632360374C23683C
:107D00001B015ED4FCF7E8F82368054623F0805396
:107D10002360324C206810F0005058D1354BA061E0
:107D2000354AE0612062A36240F20113E0622263FF
:107D3000C4F8C0306063A263C4F8C430E063226456
:107D4000C4F8C8306064236823F4802323604FF0B4
:107D5000FF332066A366D4F8303143F48033C4F88F
:107D600030319CE7FCF7B8F8001BB0429ED995E78C
:107D70001E4A136823F03F0343F0010313600023FE
:107D80002361FCF767F8002881D1FCF7A5F8134DB3
:107D9000044641F288362B6913F0380F91D0FCF776
:107DA0009BF8001BB042F6D978E7FCF795F8401B2A
:107DB00064288ED972E7FCF78FF8401B322893D9DC
:107DC0006CE7FCF789F8401B322898D966E7FCF786
:107DD00083F8401B32289DD960E700BF0044025859
:107DE000040300240090D00300000024002000526F
:107DF00065EDEEFF000202028002010108B5FFF707
:107E00000DFF044B1B6A5A0742BF03F00703033BF5
:107E1000D84008BD0044025808B5FFF7FFFE044BE8
:107E20001B6A5A0642BFC3F30213033BD84008BD86
:107E30000044025808B5FFF7F1FE044B1B6A5A05CF
:107E400042BFC3F30223033BD84008BD004402589D
:107E5000054B10B59C6BFFF78BF9C4F30644013456
:107E6000B0FBF4F010BD00BF00440258054B10B544
:107E70001C6CFFF7CFF9C4F306440134B0FBF4F0F7
:107E800010BD00BF00440258F8B50368044659030A
:107E90004BD52E4BC06F1A6F12F4407217D000F4FE
:107EA0004071914213D02A4A116841F480711160E7
:107EB0001268D20547D51A6F196F22F4407241F447
:107EC00080311967196F21F4803119671A67B0F58D
:107ED000807F08D0E36F1D4913F47C3F13D10A69FA
:107EE00022F47C5216E0FBF7F7FF184E054641F2EC
:107EF0008837336F9B07EDD4FBF7EEFF401BB8428A
:107F0000F7D9032312E00869124A20F47C5002EAF0
:107F1000131202430A6103F440730C4A116F0B43BE
:107F20001367136F43F40043136700232268D607D7
:107F30001ED56068032800F20881DFE810F0120007
:107F40000D00010112000123F0E700BF00440258B8
:107F500000480258CFFFFF0F9D4DE96A41F04001F4
:107F6000E9622BB99A4DE96C21F003010143E96400
:107F700095070AD5A068102800F0E980202800F0B5
:107F8000F580002800F0E880012350070AD5E0685A
:107F9000402800F0F080802800F0FC80002800F0ED
:107FA000EF800123110706D589482569C16C21F0AE
:107FB00040512943C164970207D5606D002800F045
:107FC000EE80042800F0FA800123D60616D56069F9
:107FD000B0F1807F00F0F780B0F1007F07D000287B
:107FE00040F0F8807A4DE96A41F48031E9622BB9BA
:107FF000774DE96C21F040710143E96495060ED597
:10800000A169B1F5001F00F0008100F2E5800029B0
:1080100000F0EB80B1F5801F00F0F18001235006E5
:1080200006D56B48E569016D21F040512943016592
:10803000110606D56648256AC16C21F440312943F2
:10804000C164D70511D5606A40B1B0F5802F40F00A
:10805000E1805F4DE96A41F08041E9622BB95C4DF6
:10806000E96C21F480210143E96496050CD5A06AEE
:10807000B0F5800F00F0D080B0F5000F00F0DB808D
:10808000002800F0CE80012315050AD5E06AB0F57E
:10809000805F00F0E58000F2D380002800F0D680F9
:1080A000012350050AD5206BB0F5807F00F0EE80EB
:1080B00000F2DC80002800F0DF800123D1040ED51F
:1080C000616BB1F5003F00F0008100F2E58000290E
:1080D00000F0EB80B1F5803F00F0F18001239704C0
:1080E0000ED5A16BB1F5007F00F00D8100F2F2809A
:1080F000002900F0F880B1F5807F00F0FE800123B8
:1081000056040ED5E16BB1F5005F00F01A8100F264
:10811000FF80002900F00581B1F5805F00F00B8140
:108120000123150440F12081206C052800F2B38161
:10813000DFE810F013010E01AC011301130113016C
:10814000234DE96A41F480210AE7012310E7204D1D
:10815000E96A41F40021E962002B7FF416AF1C4D5F
:10816000E96C21F030010143E9640EE7184DE96A3A
:1081700041F48011EFE7164DE96A41F40021E9620C
:10818000002B7FF40FAF124DE96C21F0C0010143C9
:10819000E96407E70E4DE96A41F48011EFE70C4D01
:1081A000E96A41F40021E962002B7FF40EAF084D2B
:1081B000E96C21F004010143E96406E7044DE96A32
:1081C00041F48011EFE7024DE96A41F000510DE7FB
:1081D00000440258012311E721F48010B0F5800F0C
:1081E00003D0B1F5401F7FF419AF002B7FF417AF18
:1081F000564DE86C20F4E0000143E9640FE7534D6D
:10820000E86A40F48030E862EFE7504DE86A40F0F9
:108210000060F8E7012328E74C4DE96A41F040018E
:10822000E962002B7FF430AF484D296D21F4400105
:108230000143296528E7454DE96A41F48031EFE7BC
:1082400020F48051B1F5005F7FF42AAF002B7FF45A
:1082500028AF3E4D296D21F440510143296520E7A7
:108260003A4DE96A41F00051E962EFE720F480718C
:10827000B1F5007F7FF421AF002B7FF41FAF334DAA
:10828000296D21F440710143296517E72F4DE96AF3
:1082900041F00051E962EFE721F48030B0F5802F22
:1082A00003D0B1F5403F7FF419AF002B7FF417AF37
:1082B000264D286D20F4E020014329650FE7234D6A
:1082C000E86A40F48030E862EFE7204DE86A40F069
:1082D0000050F8E721F48070B0F5806F03D0B1F55D
:1082E000407F7FF40CAF002B7FF40AAF174DA86DD1
:1082F00020F4E0600143A96502E7144DE86A40F408
:108300008030E862EFE7114DE86A40F00050F8E78E
:1083100021F48050B0F5804F03D0B1F5405F7FF479
:10832000FFAE002B7FF4FDAE084DA86D20F4E040B9
:108330000143A965F5E6054DE86A40F48030E8623E
:10834000EFE7024DE86A40F00050F8E700440258B9
:10835000A24DE96A41F40031E9622BB99F4DA96D44
:1083600021F007010143A965D00304D59B48C16AE8
:1083700041F00051C162910308D5A06C002800F0C3
:108380008C80B0F1006F00F08D80012317030ED5B3
:10839000E16CB1F5003F00F0AB8000F28D80002968
:1083A00000F09B80B1F5803F00F09D800123D60254
:1083B0000ED5216DB1F5001F00F0BD8000F29D804B
:1083C000002900F0AD80B1F5801F00F0AF800123DF
:1083D00055020ED5A06EB0F1007F00F0CA8000F209
:1083E000AF80002800F0BA80B0F1807F00F0BC8040
:1083F000012310020ED5A16DB1F5007F00F0DA80E7
:1084000000F2BC80002900F0CA80B1F5807F00F046
:10841000CC800123D1010CD5E16D202900F0EB8047
:1084200000F2CD80002900F0DB80102900F0DE8012
:10843000012397010CD5216E202900F0F88000F26D
:10844000DF80002900F0E380102900F0EA8001239A
:1084500056010CD5616E202900F0058100F2EC80F8
:10846000002900F0F080102900F0F7800123D500EA
:1084700040F10A81E06E052800F21581DFE810F076
:10848000FD00F8000E01FD00FD00FD00534DE96AFE
:1084900041F0805160E7012366E7504DE96A41F001
:1084A0000051E962002B7FF471AF4C4DE96C21F073
:1084B00000610143E96469E7B1F5403F03D0B1F5DC
:1084C000802F7FF473AF002B7FF471AF434D686D45
:1084D00020F4E0200143696569E7404DE86A40F017
:1084E0004000E862EFE73D4DE86A40F48030F8E78D
:1084F0003A4DE86A40F00060F3E721F48010B0F5EF
:10850000800F03D0B1F5401F7FF461AF002B7FF4E3
:108510005FAF324D686D20F4E0000143696557E7B5
:108520002E4DE86A40F04000E862EFE72B4DE86A24
:1085300040F48030F8E7294DE86A40F00060F3E746
:10854000B0F1407F7FF454AF002B7FF452AF234D46
:10855000296D21F04071014329654AE71F4DE96A01
:1085600041F04001E962EFE71C4DE96A41F48021E6
:10857000F8E71A4DE96A41F00051F3E7B1F5407FA1
:1085800003D0B1F5806F7FF444AF002B7FF442AF8E
:10859000124D686D20F4E060014369653AE70F4DC4
:1085A000E86A40F04000E862EFE70C4DE86A40F40A
:1085B0008030F8E7094DE86A40F00060F3E73029C1
:1085C00002D040297FF434AF002B7FF432AF034D4B
:1085D000286D20F07000014329652AE70044025805
:1085E0005D4DE86A40F04000E862EDE75A4DE86A08
:1085F00040F48030F8E7584DE86A40F00060F3E757
:1086000021F01000402802D030297FF420AF002B49
:108610007FF41EAF504D686D20F070000143696516
:1086200016E74D4DE86A40F40030E862EFE74A4D46
:10863000E86A40F08050F8E721F01000402802D0AE
:1086400030297FF413AF002B7FF411AF424DA86D9A
:1086500020F070000143A96509E73F4DE86A40F446
:108660000030E862EFE73C4DE86A40F08050F8E700
:10867000394DE96A41F40031E9622BB9364D696D33
:1086800021F007010143696590001AD5206F052884
:108690003ED8DFE800F00F0A380F0F0F2E4DE96AC1
:1086A00041F08051E8E70123EEE72B4DE96A41F400
:1086B0000031E9622BB9284D296D21F007010143F2
:1086C0002965510008D5606FB0F5805F27D0B0F5FF
:1086D000005F1FD018B30123002A06DAA06FB0F59F
:1086E000804F33D024D840B30123120107D51A4953
:1086F000D4F880000A6922F4004202430A61181E7D
:1087000018BF0120F8BD144DE96A41F08051D0E74F
:108710000123D6E7104DE96A41F08051E962002B50
:10872000DAD10D4DE96C21F440510143E964D3E7FE
:1087300020F48041B1F5004FD6D1002BD5D1064DA4
:10874000E96C21F440410143E964CEE7024DE96A56
:1087500041F08051E962F0E700440258436E02683C
:1087600033F8021B11844366B0F86A30013B9BB2B8
:10877000A0F86A30B0F86A309BB21BB9136923F0D5
:10878000020313617047436E026853F8041B1162C1
:108790004366B0F86A30013B9BB2A0F86A30B0F88B
:1087A0006A309BB21BB9136923F00203136170474F
:1087B00003685A69996941F008019961996941F022
:1087C00010019961196821F001011960196921F4FA
:1087D0005B7121F003011961996821F440419960AE
:1087E00090F8891004290BD0910609D5D0F88C1087
:1087F00041F08001C0F88C10996941F02001996125
:1088000090F8891003291BD0510609D5D0F88C1097
:1088100041F00401C0F88C10996941F04001996160
:10882000816AB1F5800F0BD1110609D5D0F88C10F3
:1088300041F00201C0F88C10996941F08001996102
:10884000910509D5D0F88C1041F00101C0F88C10C9
:10885000996941F400719961D20509D5D0F88C204D
:1088600042F00802C0F88C209A6942F480729A6142
:108870000023A0F86A30A0F872307047426E036897
:10888000127883F82020436E01334366B0F86A30D3
:10889000013B9BB2A0F86A30B0F86A309BB223B9B2
:1088A0000268136923F00203136170472DE9F04158
:1088B0000446D8B10368814A806A9342E16803D0D4
:1088C00002F5E052934201D10F290FD8E26B55090E
:1088D00001F10802D20805FB0222784DAB4203D019
:1088E00005F5E055AB4203D1082A15D90120BFE0B8
:1088F000734DAB4209D0734DAB4206D005F5806590
:10890000AB4202D0704DAB4201D1102AEED8B0F587
:10891000800F08D00D040CE0B0F5800FFAD1236B66
:10892000B3F5702FE2D8256B05B90D04B1EB154FE7
:10893000DCD894F8893003F0FF0223B9204684F88C
:108940008820F8F7D5FC02236168D4F838E084F871
:10895000893023681A6822F001021A60A269B2F114
:10896000806F07D1B1F5800F40F08480BEF1000F19
:1089700000F0878011F48008D4F80CC000F08680E5
:10898000BCF1060F40F282801F68206D27F48077CB
:10899000384318600A43E769A06A42EA0E024CEACB
:1089A0000707E66BB0F5800F47EA000747EA0607BE
:1089B00047EA05079F60676B42EA0702676A42EA77
:1089C0000702276942EA0702676942EA0702276A43
:1089D00042EA0702E76C42EA0702A76842EA070296
:1089E000A76C42EA0702A76D42EA0702E76D42EA76
:1089F0000702276E42EA0702DA6021D1226C012ABF
:108A00001A680CBF42F4004222F400421A60626C01
:108A1000012A1A680CBF42F4804222F480421A6094
:108A2000264A934203D002F5E052934232D1B5F583
:108A3000702F3FD11A6842F400521A60E26A1A6439
:108A400019B99A6842F400729A601A6D22F0010214
:108A50001A65B8F1000F05D0DA68616D22F00042A6
:108A60000A43DA6000200123C4F88C0084F88930BE
:108A7000BDE8F08100297FF47DAFBEF1805F7FF417
:108A800079AF186840F48050186073E7186820F4D4
:108A900080707EE70A4A934209D00A4A934206D080
:108AA00002F58062934202D0074A934202D1B5F5A3
:108AB000F81FBEE71A6822F40052BEE700340042F5
:108AC00000300042003800400014005810B5044641
:108AD00088B10268022380F88930136823F001030B
:108AE0001360F8F78DFD0020C4F88C0084F888002E
:108AF00084F8890010BD0120FCE70000034630B572
:108B000090F88800012811D0012083F8880001B175
:108B100022B90022012083F8882030BD93F8890013
:108B200001284FF0000003D083F888000220F4E70A
:108B300003245966A3F8682083F88940DC68C3F8E9
:108B40008C000F2CA3F86A201968D866A3F870006F
:108B5000A3F87200986733D92148814236D0214862
:108B6000814233D000F5806081422FD01E4D1F48D6
:108B70001F4CA94218BF2046D8679868B0F5C02F8F
:108B800026D1086840F40060086048686FF30F0061
:108B900002434A600A6842F001020A600A6942F42C
:108BA0004A7242F002020A615A68B2F5800F03D19C
:108BB0000A6842F400720A60002083F88800ACE77B
:108BC0000B480C4D072C98BF2846D5E70748D3E73C
:108BD000C86820F4C02040F40030C860D5E700BF6A
:108BE0000030004200380040001400588787000819
:108BF0005D8700087D880008F8B590F88830044645
:108C00001646012B09D0012380F8883090F889306E
:108C1000012B04D0002380F888300220F8BD21B950
:108C2000002384F888300120F8E7002AF8D00323D5
:108C30004166056880F889300023C0F88C30A4F8BC
:108C40006820A4F86A20C366A0F87030A0F87230DB
:108C5000C0E91E338368B3F5C02F49D12B6843F4B4
:108C600000632B60E268D4F880000F2A836946D93C
:108C7000022B12D04C4FBD42D2D04C4FBD42CFD070
:108C800007F58067BD42CBD0494FBD42C8D0002B0D
:108C9000C6D00F2A01D8022B35D0464B072A43668F
:108CA000454B0366454B83664FF00003C366AB68D4
:108CB00023F40043AB6036D8A4F86A60036D1B064A
:108CC00045D5436F002B36D0B4F86A2020351B6899
:108CD00092B21D61C3E90221FBF778FE00283ED065
:108CE000D4F88C3043F01003C4F88C30002328E013
:108CF000EB6823F4C02343F40033EB60B2E7072AA8
:108D0000C5D8012B05D1B4F86A309BB201335B089A
:108D100006E0022BC1D1B4F86A309BB203339B0842
:108D2000A4F86A30B9E70F2A94BF7300B3009BB26E
:108D3000A4F86A30C2E7D4F88C2042F01002C4F8DC
:108D40008C2084F88830012384F889306BE7B4F8EC
:108D50006A3005F120029BB2FBF760FBBEE7D4F856
:108D600080202368126D1649812A5A6802EA01029E
:108D700018BF32435A609A6842F400429A601A69F6
:108D800042F448721A611A6842F001021A6062687D
:108D9000B2F5800F03D11A6842F400721A60002302
:108DA00084F888303AE700BF0030004200380040C5
:108DB0000014005805900008B18F000819900008B1
:108DC0000000FFFF70B590F8883004461646012B6E
:108DD00009D0012380F8883090F88930012B04D025
:108DE000002380F88830022070BD21B9002384F868
:108DF00088300120F8E7002AF8D00423C16605680E
:108E000080F889300023C0F88C30A4F87020A4F8D2
:108E10007220A0F86830A0F86A30C0E91E33836879
:108E2000B3F5C02F1DD12B6823F400632B60E268DB
:108E3000D4F884000F2A1BD9C369B3F5003F19D0B9
:108E4000504B9D42D2D0504B9D42CFD003F5806312
:108E50009D42CBD04D4B9D42C8D0C369002BC5D09D
:108E600008E0EB6823F4C02343F48023EB60DEE7E3
:108E7000072AF2D8AB68072A23F48043AB6014D8E2
:108E8000C369B3F5803F05D1B4F872309BB20133AA
:108E90005B0807E0B3F5003F0DD1B4F872309BB228
:108EA00003339B08A4F8723005E00F2A03D8C36986
:108EB000B3F5003FE8D0364B072A4366354B0366CF
:108EC000354B83664FF00003C36619D8A4F872606F
:108ED000036D1B0628D5436FD3B1B4F8722030352B
:108EE0001B6892B2C3E903519A60FBF76FFD20B390
:108EF000D4F88C3043F01003C4F88C3000230DE01C
:108F00000F2A94BF7300B3009BB2A4F87230DFE75E
:108F1000D4F88C2042F01002C4F88C2084F88830F9
:108F2000012384F8893064E7B4F872300A4605F109
:108F300030019BB2FBF772FAD9E7D4F8842023689A
:108F4000126D1649812A5A6802EA010218BF32439B
:108F50005A609A6842F480429A601A6942F45072E8
:108F60001A611A6842F001021A606268B2F5800F55
:108F700003D11A6842F400721A60002384F8883022
:108F800032E700BF003000420038004000140058B3
:108F90000F900008D98F0008199000080000FFFF0B
:108FA000D0F88C3043F48063C0F88C3001207047D7
:108FB000C06D08B590F88930072B06D0D0F8803006
:108FC0001B6D812B02D1F8F723F808BD02681369E5
:108FD00043F008031361F8E7C06D08B590F88930D5
:108FE000072B06D0D0F884301B6D812B02D1F7F708
:108FF000F1FF08BD0268136943F008031361F8E745
:1090000070477047C06D08B5FFF7FBFF08BDC06D26
:1090100008B5F7F7E9FF08BD10B5C46DFBF75AFBBB
:1090200068B12046FFF7C4FBD4F88C3043F010033E
:10903000C4F88C30012384F88930F7F7DFFF10BDC6
:1090400008B5C06D0023A0F87230A0F86A30012383
:1090500080F88930F7F7D2FF08BD70472DE9F04757
:109060000668044633697269D6F80880110590F8DD
:10907000897003EA0205FFB209D51A0707D5B3695B
:1090800043F40063B361FFF7E8FFBDE8F08705F044
:109090006403042B18D1E36F20469847A36F204642
:1090A0009847012305F04509B9F1010F03D1A36FDA
:1090B000204698474B4605F02602022A06D1E36F68
:1090C0002046BDE8F04718470023EBE7002BDCD132
:1090D0002B0751D523689A6942F008029A619A6970
:1090E00042F010029A619A6942F400629A611A6928
:1090F00022F008021A619B6813F4404F1AD02046F0
:10910000FFF756FB012384F88930D4F88C3023B361
:10911000F7F774FFB9E7E268E36E0F2A10D9226807
:10912000126B43F8042BE366B4F87230013B9BB238
:10913000A4F87230B4F872309BB2002BEBD1DEE7AA
:10914000072A03D9328E23F8022BECE7226892F823
:1091500030201A70E36E0133E5E7052F02D1FFF7E7
:109160004FFF92E7042F02D1F7F734FF8DE7032F6B
:109170008BD1F7F74DFF88E715F4587F85D0680647
:109180000AD5D4F88C30226843F00403C4F88C303C
:10919000936943F040039361A9050AD5D4F88C3054
:1091A000226843F00103C4F88C30936943F40073E0
:1091B0009361EA050AD5D4F88C30226843F008039D
:1091C000C4F88C30936943F480739361AB060AD57D
:1091D000D4F88C30226843F08003C4F88C30936953
:1091E00043F020039361D4F88C30002B3FF44DAF53
:1091F000236808F440481A68B8F5404F22F001028D
:109200001A601A6922F45A7222F003021A6124D1F8
:109210009A68D4F8840022F440429A6050B1114B0D
:10922000C366FBF781F928B1D4F88C3043F04003D2
:10923000C4F88C30D4F8800000283FF426AF094BE6
:10924000C366FBF771F900283FF41FAFD4F88C30E8
:1092500043F04003C4F88C3017E70123204684F81C
:10926000893055E74190000890F889007047D0F8A0
:109270008C007047036AB0F1844F026A23F0020346
:1092800022F0010270B50262426884690D6824F41C
:10929000803424F0730444EA05048D6843EA05032E
:1092A0000AD00E4DA84207D005F58065A84203D02C
:1092B00005F58065A8420BD1CD6823F0080322F4A0
:1092C00040722B43D1E9055623F0040335432A436A
:1092D00042604A6884614263036270BD004000429C
:1092E000036AB0F1844F026A23F4007322F480729F
:1092F00070B502624268C4690D6824F4803424F0B9
:10930000730444EA05048D6843EA05230ED123F46F
:109310000063CD6843EA052323F4806322F44052BE
:10932000D1E90556354342EA05120AE0084DA84244
:10933000F4D005F58065A842F0D005F58065A84217
:10934000ECD042604A68C461C263036270BD00BF72
:1093500000400042036AB0F1844F026A23F40053D4
:1093600022F4805270B502624268C4690D6824F02C
:10937000807424F4E64444EA05248D6843EA053306
:109380000ED123F40043CD6843EA053323F4804330
:1093900022F44042D1E90556354342EA85120AE0FB
:1093A000084DA842F4D005F58065A842F0D005F537
:1093B0008065A842ECD042604A68C46102640362DE
:1093C00070BD00BF00400042026AB0F1844F036AE2
:1093D00022F4003223F4803330B503624468036D15
:1093E0000D6823F4803323F0700343EA05038D688E
:1093F00042EA05420AD00B4DA84207D005F5806528
:10940000A84203D005F58065A84204D124F4803435
:109410004D6944EA0524446003654B688364026235
:1094200030BD00BF00400042026AB0F1844F036AC1
:1094300022F4001223F4801330B503624468036DF4
:109440000D6823F0807323F4E04343EA05238D681D
:1094500042EA05520AD00B4DA84207D005F58065B7
:10946000A84203D005F58065A84204D124F48024E5
:109470004D6944EA8524446003654B68C364026215
:1094800030BD00BF004000427047704770477047D2
:1094900070477047036870B5DD6804461E69B207FF
:1094A0000ED5A9070CD56FF002021A6101220277CE
:1094B0009B699A0700F0A480FFF7EAFF0023237757
:1094C000730711D568070FD523686FF00402204693
:1094D0001A61022222779B6913F4407F00F0968084
:1094E000FFF7D6FF00232377310710D52A070ED5C3
:1094F00023686FF0080220461A6104222277DB6994
:109500009B0700F08980FFF7C3FF00232377F10654
:1095100010D5EA060ED523686FF0100220461A61B6
:1095200008222277DB6913F4407F7BD0FFF7B0FF7E
:1095300000232377F30708D5E80706D523686FF0E3
:10954000010220461A61FFF7A1FF16F4025F08D05E
:10955000290606D523686FF4025220461A6100F0EE
:1095600020FCF20508D52B0606D523686FF480721F
:1095700020461A6100F016FC700608D5690606D56B
:1095800023686FF0400220461A61FFF782FFB2069F
:1095900008D5AB0606D523686FF0200220461A6175
:1095A00000F0FEFBF00208D5E90206D523686FF44F
:1095B000801220461A6100F0F6FBB20208D5AB0219
:1095C00006D523686FF4001220461A6100F0ECFB08
:1095D000700208D5690206D523686FF48002204620
:1095E0001A6100F0E2FB320222D52B0220D523685B
:1095F0006FF4000220461A61BDE8704000F0D6BB4F
:10960000FFF745FF2046F7F705FD57E7FFF73FFF58
:109610002046F7F7FFFC65E7FFF739FF2046F7F72D
:10962000F9FC72E7FFF733FF2046F7F7F3FC7FE71B
:1096300070BD0000B0F1844F03680DD0B0F1804FD1
:109640000AD0284A904207D002F58062904203D0A7
:1096500002F58062904208D123F070034A681343F8
:1096600023F44073CA68134318E01F4A9042F7D0AE
:109670001E4A9042F4D002F580629042F0D002F58A
:1096800080629042ECD01A4A9042E9D002F58062A2
:109690009042E5D002F580629042E1D04A6923F021
:1096A0008003B0F1844F43EA020303608B68C36216
:1096B0000B6883620AD00E4B984207D003F5806393
:1096C000984203D003F58063984201D10B6903638C
:1096D000012343610369DB0703D5036923F0010319
:1096E0000361704700040040004C00420018004035
:1096F0000040004210B5044650B390F83D3003F0EE
:10970000FF021BB980F83C20F8F7F4F80223206828
:10971000211D84F83D30FFF78DFF0123002084F8E0
:10972000483084F83E3084F83F3084F8403084F884
:10973000413084F8423084F8433084F8443084F86F
:10974000453084F8463084F8473084F83D3010BD09
:109750000120FCE710B5044650B390F83D3003F00B
:10976000FF021BB980F83C20FFF78EFE0223206821
:10977000211D84F83D30FFF75DFF0123002084F8B0
:10978000483084F83E3084F83F3084F8403084F824
:10979000413084F8423084F8433084F8443084F80F
:1097A000453084F8463084F8473084F83D3010BDA9
:1097B0000120FCE738B50D46044630B390F83D3043
:1097C00003F0FF021BB980F83C20FFF75EFE022386
:1097D000214684F83D3051F8040BFFF72BFF036856
:1097E00023F00803036003682B4303600123002078
:1097F00084F8483084F83E3084F83F3084F84430B0
:1098000084F8453084F83D3038BD0120FCE7000085
:10981000036AB0F1844F026A23F0200322F01002A1
:1098200070B50262426884690D6824F0807424F483
:10983000E64444EA05248D6843EA05130ED123F07B
:109840008003CD6843EA051323F0400322F440620D
:10985000D1E90556354342EA85020AE0084DA8429F
:10986000F4D005F58065A842F0D005F58065A842E2
:10987000ECD042604A6884618263036270BD00BFBD
:109880000040004238B590F83C300446012B73D0BC
:1098900001200C2A84F83C004ED008D8042A2BD092
:1098A000082A39D0BAB1002384F83C3038BD102AD8
:1098B00052D0142AF7D12068FFF7B6FD0A69036D6C
:1098C00043F400630365036D23F480630365036D54
:1098D00043EA02234EE02068FFF7CCFC0A69836963
:1098E00043F008038361836923F004038361836980
:1098F000134383610020D6E72068FFF789FF0A69D8
:10990000836943F400638361836923F48063836123
:10991000836943EA0223ECE72068FFF7E1FC0A6968
:10992000C36943F00803C361C36923F00403C3613F
:10993000C3691343C361DDE72068FFF70BFD0A69C4
:10994000C36943F40063C361C36923F48063C361E3
:10995000C36943EA0223EDE72068FFF735FD0A6992
:10996000036D43F008030365036D23F004030365EF
:10997000036D13430365BDE7022097E710B50A4363
:10998000846842EA032224F47F442243826010BDAB
:1099900000684B688268602B22F4401222F070024B
:1099A00042EA030222F4803210B522F007020C686A
:1099B00042EA0402826063D014D8402B3DD00DD817
:1099C000202B38D005D833F0100314BF012000201D
:1099D00010BDB3F1300018BF0120F9E7502B3FD084
:1099E0000120F5E7702B21D06F2BF9D92E4A934235
:1099F00021D010D8303A93421DD004D823F0100360
:109A0000B3F58010E7E7294A934214D02848181A82
:109A100018BF0120DCE7274A93420CD003D823F07B
:109A200010032548F3E7B3F12010D4E70B69D1E91F
:109A30000221FFF7A3FF0020CAE7052CD0D0B4F124
:109A4000011FCDD0026A036A096923F00103036292
:109A5000836923F0F00343EA011383610262EAE7BA
:109A60008A680C69016A036A21F00A0123F0010384
:109A70000A430362836923F0F00343EA0413ECE72B
:109A8000036A026A8C6823F0A00322F010020969BD
:109A900043EA04130262826922F4704242EA01320C
:109AA00082610362C7E700BF500010003000100061
:109AB00040001000100020006000100038B590F841
:109AC0003C300446012B4FF002031CD0012580F8E6
:109AD0003D3080F83C50FFF75BFF30B10023284653
:109AE00084F83D5084F83C3038BD2368DA6822F0B1
:109AF0004002DA60DA6822F48042DA6084F83D508D
:109B000084F83C00F0E71846EEE710B501F01F01BD
:109B10000124036A8C408A4023EA04030362036A37
:109B20001A43026210BD000038B5044600680022E6
:109B30000D46FFF7EAFFB0F1844F0AD0234B98425D
:109B400007D003F58063984203D003F58063984201
:109B50000DD1026A41F211131A4208D1026A44F28D
:109B600044431A4203D1436C23F400434364026A22
:109B700041F211131A4208D1026A44F244431A42D4
:109B800003D1036823F001030360082D4FF00103A4
:109B900015D006D865B1042D0ED0012384F84330CA
:109BA00008E00C2D0ED0102DF7D184F8423001E0E2
:109BB00084F83E30002038BD84F83F30FAE784F85E
:109BC0004030F7E784F84130F4E700BF004000423E
:109BD000FFF7AABF082908B518D005D859B104293C
:109BE00011D090F8433008E00C2912D01029F8D198
:109BF00090F8423001E090F83E30013B18BF01235D
:109C000053B1012044E090F83F30F6E790F840303F
:109C1000F3E790F84130F0E708294FF002033FD016
:109C200006D861B1042934D0022380F84330E8E734
:109C30000C293CD01029F7D180F84230E1E70268C6
:109C400080F83E30D36843F002030068D3600122FD
:109C5000FFF75BFFB0F1844F0AD0264B984207D044
:109C600003F58063984203D003F58063984225D1C1
:109C7000436CB0F1844F43F40043436402D01D4B66
:109C8000984231D182681C4B1340062B29D1002009
:109C900008BD026880F83F30D36843F00403D4E77E
:109CA000026880F84030D36843F00803CDE70268CB
:109CB00080F84130D36843F01003C6E7B0F1804F1D
:109CC000E0D00E4B9842DDD003F580639842D9D0A6
:109CD00003F580639842D5D0094B9842D2D0094B06
:109CE000CEE7B3F5803FD2D0036843F001030360B1
:109CF000CDE700BF00400042070001000004004023
:109D0000004C004200180040FFF764BF30B590F8E7
:109D10003C3004460220012B38D0236884F83D00F3
:109D2000B3F1844F5A68986802BF4D6822F47002FC
:109D30002A430D68B3F1844F22F0007222F07002C2
:109D400042EA05025A6016D0B3F1804F13D0104A90
:109D5000934210D002F5806293420CD002F58062EB
:109D6000934208D00B4A934205D00B4A934202D04B
:109D70000A4A934204D1896820F080020A439A601B
:109D80000123002084F83D3084F83C0030BD00BF42
:109D900000040040004C0042001800400040004217
:109DA0007047704770477047704770477047026848
:109DB00052E8003F23F0C00342E800310268002966
:109DC000F5D102F1080353E8003F23F4000302F148
:109DD000080C4CE800310029F3D12023C0F888306A
:109DE0007047000010B5026852E8003F23F49073FA
:109DF00042E8003102680029F5D10F4C02F1080356
:109E000053E8003F234002F1080C4CE800310029E0
:109E1000F4D1C36E012B07D152E8003F23F01003A9
:109E200042E800310029F7D12023C0F88C3000230C
:109E3000C366436710BD00BFFEFFFFEF38B5134692
:109E4000D0F888200446202A4CD139B333B30022FD
:109E5000A0F856300165A0F85430C0F890202120B9
:109E6000C4F88800E06F38B31F4D05661F4D456686
:109E70001F4DC0E91A52A268B2F5805F03D1226972
:109E80000AB95B009BB2026D120626D5426F3AB941
:109E90001023C4F890302023C4F8883001201BE040
:109EA0001268002AF4D0C2E9023123682833136112
:109EB000FAF78CFD0028EBD1402223681A62226851
:109EC00002F1080353E8003F43F0800302F1080168
:109ED00041E800300028F3D138BD22682832FAF773
:109EE0009DFAE7E70220F7E79D9F0008E39F00083F
:109EF000F19F000810B50446226852E8003F23F4A1
:109F0000907342E8003123680029F5D1224803F11B
:109F1000080252E8002F024003F1080C4CE800212F
:109F20000029F4D1E26E012A07D153E8002F22F074
:109F3000100243E800210029F7D19A6852061CD587
:109F400003F1080252E8002F22F0400203F108005A
:109F500040E800210029F3D1D4F8800068B1C1663F
:109F6000FAF798FA48B1D4F88000FAF7B3FB102852
:109F700003D1C4F89000032010BD236800200F22F5
:109F8000A4F85E001A629A6942F008029A612023DE
:109F9000C4F88C30E066EFE7FEFFFFEF08B503463C
:109FA000C06D1B6D812B18D00023A0F856300268BD
:109FB00002F1080353E8003F23F08003083242E82F
:109FC000003102680029F2D152E8003F43F040031B
:109FD00042E800310029F7D108BDF7F72DF8FBE77B
:109FE0007047C06D08B5FFF7FBFF08BD70477047AD
:109FF000C06D38B50468D0F88830D0F88C50A268AD
:10A00000120606D5212B04D10023A0F85630FFF705
:10A01000CEFEA3685B0606D5222D04D10023A0F84E
:10A020005E30FFF7DFFED0F8903043F01003C0F849
:10A030009030FFF7DCFF38BD08B5C06D0023A0F8F5
:10A040005E30A0F85630FFF7D2FF08BD7047000021
:10A0500003682DE9F041D96940F60F061A680446F5
:10A0600031429D6810D18E0640F1978002F02006A3
:10A0700005F080573E4300F09080436F002B00F0C6
:10A080008580BDE8F0411847A84EA9482E401040F1
:10A09000304300F08280CF0709D5D00507D50120D5
:10A0A0001862D4F8900040F00100C4F890008F07C7
:10A0B00009D5E80707D502201862D4F8900040F0CF
:10A0C0000400C4F890004F0709D5E80707D504201D
:10A0D0001862D4F8900040F00200C4F890000F0716
:10A0E0000BD502F02000304307D008201862D4F8C6
:10A0F000900040F00800C4F890000E050AD5500109
:10A1000008D54FF400601862D4F8903043F0200373
:10A11000C4F89030D4F89030002B37D08B0609D596
:10A1200002F0200205F080552A4303D0636F0BB183
:10A130002046984726682046D4F89020B36802F05D
:10A14000280203F0400353EA020521D0FFF74AFE3C
:10A15000B3685F0617D5226802F1080353E8003F91
:10A1600023F04003083242E800310029F3D1D4F84B
:10A17000800040B16F4BC366FAF7D6F930B1D4F81E
:10A180008000C36E7DE72046FFF731FFBDE8F08118
:10A19000FFF72DFFC4F89050F8E7E06E012840F07B
:10A1A0008D80CE0640F18A80D00640F18780102253
:10A1B0001A629968B4F85C20490651D5D4F8800039
:10A1C0000168896C89B2002942D0914240D2026D67
:10A1D000A4F85E10812A2FD053E8002F22F4807259
:10A1E00043E800210029F7D103F1080252E8002FCB
:10A1F00022F0010203F1080040E800210029F3D118
:10A2000003F1080252E8002F22F0400203F1080097
:10A2100040E800210029F3D12022C4F88C20E16617
:10A2200053E8002F22F0100243E800210029F7D163
:10A23000D4F88000FAF72EF90223B4F85C102367F3
:10A24000B4F85E30C91A89B22046FFF7FFFE9DE7D9
:10A2500091429BD1036D812B98D102232367F3E7B1
:10A26000B4F85E10B4F85E0089B280B200288DD0D8
:10A27000521A91B2002989D053E8002F22F490722B
:10A2800043E800200028F7D12B4D03F1080252E8E3
:10A29000002F2A4003F1080646E800200028F4D1E8
:10A2A00020226067C4F88C20E06653E8002F22F07B
:10A2B000100243E800200028F7D1CEE7CF0209D5ED
:10A2C0006E0207D54FF4801220461A62BDE8F041B5
:10A2D00000F0C0BB08060BD502F0800005F40005B5
:10A2E000284305D0A36F002B3FF450AF2046C8E6AB
:10A2F0004F0611D556060FD553E8002F22F0400225
:10A3000043E800210029F7D120232046A167C4F8A3
:10A310008830F6F791FE39E70D020FD550000DD5C4
:10A320002046BDE8F04100F097BB00BF01000010DF
:10A330002001000439A00008FEFFFFEFCB017FF5EC
:10A3400025AF002ABFF622AF2046BDE8F04100F05D
:10A3500082BB00BFC06D08B501230367C36E012B2C
:10A3600005D1B0F85C104908FFF770FE08BDFFF793
:10A370003DFEFBE708B50346C06D1B6D812B32D057
:10A380000023A0F85E30026852E8003F23F4807397
:10A3900042E8003103680029F5D103F1080252E8D0
:10A3A000002F22F0010203F1080C4CE800210029E3
:10A3B000F3D103F1080252E8002F22F0400203F12A
:10A3C000080C4CE800210029F3D12022C0F88C2091
:10A3D000C26E012A07D153E8002F22F0100243E891
:10A3E00000210029F7D100230367C36E012B04D19C
:10A3F000B0F85C10FFF72AFE08BDF6F713FEFBE786
:10A4000038B50446C0692169A26823680A436169B6
:10A410001D680A439C49024329400A43E1681A60C7
:10A420005A6822F440520A43A1695A60974A9342FB
:10A430001CBF226A11439A6822F06E4222F43062F5
:10A440000A43616A9A60DA6A22F00F020A43DA620A
:10A450008F4A93421AD18F4B5B6D03F00703052B94
:10A4600000F28B80DFE813F0CB00D100D700DD00D5
:10A470000B010501FDF7FAFC002845D100204FF043
:10A480000113A3660023C4E91D3338BD824A9342F9
:10A4900013D002F5806293420FD002F5806293429E
:10A4A0000BD002F58062934207D002F5205293420E
:10A4B00003D002F5806293420AD1764B1B6D03F004
:10A4C0000703052B5FD8DFE803F09160A6ACDAD470
:10A4D0006E4A934257D102F50E32936D03F0070393
:10A4E000052B50D801A151F823F000BF5DA500084D
:10A4F00057A5000875A4000863A5000877A5000803
:10A5000005A500084FF40040644B626A656833F8A3
:10A51000122005EB4501B0FBF2F3994233D8B3EBBF
:10A52000053F30D800231946F5F7EAFE2A4609020E
:10A530006B0841EA10610002C0184FF0000341F1BE
:10A540000001F5F7DDFE564BA0F540729A421AD88D
:10A550002368D86092E7FDF77BFC8DE7FDF76AFC86
:10A560008AE713684F4813F0200FCDD01368C3F368
:10A57000C103D840C8E74C48C6E78023B0F5004F78
:10A580000BD1082B44D9012079E70423F6E7FDF726
:10A5900035FC00283FF472AF14E0082BF3D8FDF728
:10A5A00057FCF6E7FDF738FCF3E7FDF75FFCF0E753
:10A5B000384B3C481A6812F0200F03D01B68C3F3D5
:10A5C000C103D840616A354B626833F81130B0FB83
:10A5D000F3F303EB5203B3FBF2F34FF6EF72A3F185
:10A5E00010019142CFD82268D36047E7B0F5004F01
:10A5F000CDD1FDF703FC00283FF440AF1EE0B0F5DD
:10A60000004FCFD1FDF708FCF5E7B0F5004FC6D1FC
:10A61000FDF71EFCEFE7B0F5004FC6D1FDF726FCB5
:10A62000E9E7B0F5004FC3D11A4B1E481A6812F083
:10A63000200F03D01B68C3F3C103D840174B626AD5
:10A64000616833F812204B08B0FBF2F203EB4203CF
:10A650004FF6EF72B3FBF1F3A3F11001914292D8E0
:10A6600023F00F02C3F34203216892B21343CB607D
:10A6700004E7B0F5004FE1D04FF40040A2E7B0F599
:10A68000004F09489ED1D9E7F369FFCF000C00586D
:10A6900000100042004402580044004018DB00084B
:10A6A000FFFC0F000090D00300093D00836A1A07E9
:10A6B00010B506D50168846B4A6822F40042224333
:10A6C0004A60DC0706D50168C46A4A6822F4003291
:10A6D00022434A60990706D50168046B4A6822F450
:10A6E000803222434A605A0706D50168446B4A68A3
:10A6F00022F4802222434A60DC0606D50168C46B3E
:10A700008A6822F4805222438A60990606D501683D
:10A71000046C8A6822F4005222438A605A0610D5DB
:10A720000168446C4A68B4F5801F22F4801242EA42
:10A7300004024A6005D14A68846C22F4C0022243B4
:10A740004A601B0606D50268C16C536823F40023D7
:10A750000B43536010BD2DE9F843DDF8209004460B
:10A760000D46174698462268D36935EA03030CBFA5
:10A7700001230023BB4201D0002022E0B9F1FF3FBA
:10A78000F2D0F9F7A9FBA0EB0800484529D8B9F1A8
:10A79000000F26D021680B685A07E4D5802DE2D03F
:10A7A000402DE0D0CE6916F008060CD008252046D2
:10A7B0000D62FFF717FB00230120C4F8905084F8C6
:10A7C0008430BDE8F883CB691B05CCD54FF400631A
:10A7D00020460B62FFF706FB202384F88460C4F850
:10A7E00090300320EDE773B500260446C0F8906072
:10A7F000F9F772FB236805461B681A071CD56FF032
:10A800007E4332464FF40011009303462046FFF783
:10A81000A2FF88B1226852E8003F23F0800342E89B
:10A8200000310029F6D12023C4F88830032000230A
:10A8300084F8843002B070BD23681B685B0724D5A0
:10A840006FF07E4300224FF48001204600932B4698
:10A85000FFF781FFC8B1226852E8003F23F49073EC
:10A8600042E8003122680029F5D102F1080353E8DB
:10A87000003F23F0010302F1080040E80031002905
:10A88000F3D12023C4F88C30D0E720230020C4F873
:10A890008830C4F88C30E0662067C8E710B50446FD
:10A8A00050B3D0F888301BB980F88430F7F700FB3C
:10A8B00024232268C4F88830136823F0010313604E
:10A8C000A36A13B12046FFF7F1FE2046FFF798FD7B
:10A8D000012811D0236820465A6822F490425A6019
:10A8E0009A6822F02A029A601A6842F00102BDE8D2
:10A8F00010401A60FFF777BF012010BD38B5A0F8EF
:10A900005C2013460025222204468165C0F8905041
:10A91000C0F88C20D0F8800038B3294A0266294A52
:10A920004266294AC0E91A25A268B2F5805F03D1C0
:10A9300022690AB95B009BB2056D2A0639D5456FBD
:10A940003DB910230120C4F890302023C4F88C3086
:10A9500038BD2D68002DF4D0AB6023682433C5E9E1
:10A960000331FAF733F80028EBD1226923683AB1B2
:10A9700053E8002F42F4807243E800210029F7D108
:10A9800003F1080252E8002F42F0010203F108002F
:10A9900040E800210029F3D103F1080252E8002F1A
:10A9A00042F0400203F1080141E800200028F3D101
:10A9B000CEE725680A4605F12401F9F72FFDD2E715
:10A9C00075A3000855A30008F19F0008D0F88C304B
:10A9D000202B30B415D1B9B1B2B100230468C366DD
:10A9E0000A4B9C420AD063681B0207D554E8003F1B
:10A9F00043F0806344E80035002DF7D130BCFFF709
:10AA00007DBF022030BC70470120FBE7000C0058DE
:10AA1000436E30B52BB90123A0F86A30A0F8683036
:10AA200030BD0368094D9A689968094CC2F34262C7
:10AA3000490F6B5C615C1B01B3FBF1F3A0F86A305A
:10AA4000AB5CA25C1B01B3FBF2F3E7E738DB000869
:10AA500030DB000870477047704790F88430012B56
:10AA600014D002682423C0F888301168136821F0DC
:10AA7000005123F00103136000234366116020227C
:10AA800080F88430C0F8882018467047022070474C
:10AA900070B590F884300446012B17D00568242344
:10AAA000C0F888302E682B6823F001032B60AB6858
:10AAB00023F060431943A960FFF7AAFF20232E600B
:10AAC000C0F88830002084F8840070BD0220FCE7C4
:10AAD00070B590F884300446012B17D00568242304
:10AAE000C0F888302E682B6823F001032B60AB6818
:10AAF00023F060631943A960FFF78AFF20232E60CB
:10AB0000C0F88830002084F8840070BD0220FCE783
:10AB100082B0002302460193019B01330193019B04
:10AB2000B3F1706F15D81369002BF5DA0023019388
:10AB3000136943F001031361019B01330193019BEE
:10AB4000B3F1706F05D8106910F00100F4D102B0B4
:10AB500070470320FBE7000084B038B505AD04461C
:10AB600085E80E00174988421AD19DF81930032B49
:10AB700003D1CB6823F48003CB601248FFF7C8FFF2
:10AB80009DF81630012B07D18B6843F008038B60CA
:10AB90008B6843F020038B60BDE8384004B07047F9
:10ABA000C36843F04003C360FFF7B2FF9DF81D3058
:10ABB00023B9A36B43F48033A363EDE7A36B23F4C2
:10ABC0008033F9E700000440022A4AD1274B284A83
:10ABD0000B44934239D9274B274A0B44934236D929
:10ABE000A1F57403254AA3F51053934231D9A1F17D
:10ABF0008373234AA3F5E74393422CD3214B224A84
:10AC00000B44934229D9214B214A0B44934226D32A
:10AC1000204B214A0B44934223D3A1F1B7731F4A1F
:10AC2000A3F5585393421ED31D4B1E4A0B44934227
:10AC30002CBF06230723C26822F47052C260C26888
:10AC400042EA8323C360002070470F23F3E70E23FB
:10AC5000F1E70D23EFE70C23EDE70B23EBE70A23E6
:10AC6000E9E70923E7E70823E5E700BF405327FFAB
:10AC7000FF340C00401E1BFF3F420F007F4F1200AD
:10AC800020D6130060B6E5FE5FE3160000D3CEFECB
:10AC900040771B00C05BB3FEC091210020753800D7
:10ACA000E05459FEE09C4100836843F00103836057
:10ACB00000207047836823F0010383600020704701
:10ACC00038B5C368012905460C4623F0C043C3606C
:10ACD00013D1C368002443F00053C3600A200A3430
:10ACE000F9F700F96B69D90702D4C82CF6D1C8244A
:10ACF000A4F1C8035842584138BD69B9C36843F04C
:10AD00008043C3600A200A34F9F7ECF86B69DA076C
:10AD1000EED5C82CF6D1EAE70120EDE782B000239A
:10AD200002460193019B01330193019BB3F1706FC4
:10AD300015D81369002BF5DA8901002341F02001B1
:10AD400001931161019B01330193019BB3F1706F7A
:10AD500005D8106910F02000F4D102B0704703202C
:10AD6000FBE782B0002302460193019B013301936C
:10AD7000019BB3F1706F13D81369002BF5DA002330
:10AD8000019310231361019B01330193019BB3F1E4
:10AD9000706F05D8106910F01000F4D102B0704740
:10ADA0000320FBE7D0F800381943C0F80018002052
:10ADB0007047000084B02DE9F843044609A880E8F4
:10ADC0000E0000239DF824609DF82E50194603F1D3
:10ADD0004002013304EB82020F2B5160F7D1E3688C
:10ADE000580603D4A36B23F00073A36304F5006734
:10ADF000002D77D17B6843F002037B60A36B23F4C3
:10AE00000013A363E368590608D4A36B43F080736F
:10AE1000A363A36B43F40003A36307E0236843F039
:10AE200040032360236843F0800323600023C4F8B9
:10AE3000003EE3685B066FD49DF82710002969D1B6
:10AE400020464FF67F38FFF7ADFF10212046FFF771
:10AE500065FF01462046FFF784FF0843002304F501
:10AE60001062C0B24FF0904C19464FF0006E00389F
:10AE70003B617B6118BF0120FB619E424ED80022DE
:10AE800004F530634FF0904C4FF0006E11464FF6D2
:10AE90007F38964255D83B6923F480733B61002389
:10AEA000A3616FF0804363619DF826301BB9A369ED
:10AEB00043F01003A361A2692B4B1343A3619DF8D8
:10AEC0002A301BB1A36943F00803A361012D05D10A
:10AED000A36943F0804343F00403A361BDE8F84352
:10AEE00004B07047E3685A060BD4A36B23F0807359
:10AEF000A363A36B23F40003A363A36B43F40013C6
:10AF00008AE7236823F040032360236823F080034B
:10AF10002360F2E7012193E7032191E7D2F8009043
:10AF2000B9F1000F0BDA3BB9C2F800E0116101334F
:10AF3000C2F808802032A0E7C2F800C0F6E711602E
:10AF4000F4E7D3F80090B9F1000F0BDA3AB9C3F87F
:10AF500000E019610132C3F80880203399E7C3F893
:10AF600000C0F6E71960F4E700383C80D0F80838F4
:10AF700013F0060004D013F0020F14BF02200F20BC
:10AF8000704730B50C78012200F5006304F00F051E
:10AF900000EB4410AA404D78012D19D1DD692A43F8
:10AFA000DA61D0F800391A0410D48A68D0F8005950
:10AFB000C2F30A030A792B4343EA824343EA8453E8
:10AFC00043F0805343F40043C0F80039002030BD03
:10AFD000DC6944EA0242DA61D0F8003B1B04F5D494
:10AFE0008B68D0F8002BC3F30A0313430A7943EAB2
:10AFF000824343F0805343F40043C0F8003BE5E74D
:10B0000010B50A78497800EB421300F50060012979
:10B0100002F00F0222D1D3F8001900290BDAD3F87D
:10B02000001941F00061C3F80019D3F8001941F08C
:10B030008041C3F800190121C46B01FA02F224EA2D
:10B040000204C463C16921EA0202C261154AD3F84D
:10B0500000190A40C3F80029002010BDD3F8001BD6
:10B0600000290BDAD3F8001B41F00061C3F8001B84
:10B07000D3F8001B41F08041C3F8001B4FF480312E
:10B08000C46B01FA02F224EA0204C463C16921EA32
:10B090000202C261044AD3F8001B0A40C3F8002B25
:10B0A000DAE700BF007833EC0078F3EF002382B0DA
:10B0B0004A780193012A0B784FEA43131ED100F519
:10B0C0001060C258C118002A02DB002002B070478D
:10B0D000C25842F00062C250C25842F08042C25090
:10B0E00042F21072019B01330193019B934201D9FB
:10B0F0000120EBE70B68002BF4DBE6E700F530609E
:10B10000C258C118002AE0DAC25842F00062C250A8
:10B11000C25842F08042C25042F21072019B013389
:10B120000193019B9342E3D80B68002BF6DBCCE73D
:10B1300010B59DF8084044B9033301329B0800EB79
:10B14000023001EB8303994201D1002010BD51F878
:10B15000042B0260F7E70000F7B54B7817460A7832
:10B16000012B0C6900EB4215DFF8A8C1DFF8A8E15C
:10B1700040F0828005F51066336944BB03EA0C0396
:10B180003361336943F400233361336903EA0E0307
:10B190003361012F0C7947D1CB6903B17361012C65
:10B1A0000CD1D0F8083813F4807FD5F800390CBFE3
:10B1B00043F0005343F08053C5F80039D5F8003907
:10B1C00043F00443C5F80039002003B0F0BD03EAA2
:10B1D0000E033361336903EA0C0333618B68BAB938
:10B1E000A34238BF0B61336943F4002333610B6919
:10B1F0003469C3F31203234333610B79012BC8D1A4
:10B20000336923F0C0433361336943F00053BFE730
:10B210001C44D6F810C0013CB4FBF3F43C4B03EAE9
:10B22000C44343EA0C03E1E7D5F80039012C43F0AD
:10B230000443C5F800390B690BD0002BC4D002F0D1
:10B240000F020123D0F8341893400B43C0F8343870
:10B25000BAE7D0F808489BB214F4807FD5F80049CB
:10B260000CBF44F0005444F08054C5F800490097E6
:10B27000C968FFF75DFFA7E7D5F8103B05F5306615
:10B2800003EA0E033361336903EA0C0333618B680D
:10B290003ABB04B10B610B623269C3F3120313436F
:10B2A0003361336943F40023012F336102D1CB684A
:10B2B00003B173610B79012B0CD1D0F8083813F46A
:10B2C000807FD5F8003B0CBF43F0005343F0805320
:10B2D000C5F8003BD5F8003B43F00443C5F8003BFC
:10B2E00072E7002CD8D01C44094AD6F810C0013CA3
:10B2F000B4FBF3F4A4B202EAC442634342EA0C0290
:10B300000B62C3F31203326132691343CCE700BF0F
:10B310000000F81FFFFF07E00000F8FF03460020D1
:10B3200070B5940803F5805502F00302A04210D3D3
:10B3300001EB840062B103F580531C680023D9003F
:10B3400024FA01F1C154013399B28A42F7D1104471
:10B3500070BD2E6841F820600130E7E74A780B782D
:10B36000012A00EB431012D1D0F80029002A06DB95
:10B370002BB1D0F8003923F08043C0F80039D0F861
:10B38000003943F40013C0F8003900207047D0F8AA
:10B39000002B002A06DB2BB1D0F8003B23F08043C2
:10B3A000C0F8003BD0F8003B43F40013C0F8003B6A
:10B3B000EBE70B784A7800EB43100B79012AA3F1F5
:10B3C0000203DBB20FD1D0F80029012B22F40012C6
:10B3D000C0F8002905D8D0F8003943F08053C0F8F0
:10B3E000003900207047D0F8002B012B22F4001206
:10B3F000C0F8002BF5D8D0F8003B43F08053C0F8DC
:10B40000003BEEE7D0F80038090123F4FE6301F4B5
:10B41000FE61C0F80038D0F800381943C0F80018B1
:10B4200000207047D0F8003E23F00303C0F8003E30
:10B43000D0F8043823F00203C0F804380020704725
:10B44000D0F8003E23F00303C0F8003ED0F80438E3
:10B4500043F00203C0F80438002070474269806955
:10B4600010407047D0F8183800F50060C0691840E7
:10B47000000C7047D0F8183800F50060C06918401B
:10B4800080B2704700EB411100F50060D1F8082B45
:10B49000406910407047D0F81028D0F8343800EBDD
:10B4A000411001F00F0100F51060CB408068DB0116
:10B4B000DBB2134318407047406900F00100704749
:10B4C000D0F800396FF30A03C0F80039D0F8043817
:10B4D00043F48073C0F804380020704730B5056C21
:10B4E00000F530630F4CA54203D9D0F8004B002C77
:10B4F00016DB002401291C611C6944F400241C6132
:10B500001C6944F018041C611C6944F0C0441C61AF
:10B5100006D15A61D0F8003B43F08023C0F8003BCD
:10B52000002030BD0A30544FD0F8D43200EB8300F5
:10B5300010B5D0F8C0428CB1D0F8C4321BB194F829
:10B540000002FF2801D1002010BD9B68214694F81D
:10B5500001229847FF2384F80032F4E70320F3E741
:10B560000A230380004870478403002470B58221B9
:10B5700006460F4800F07AFB012105460C4800F012
:10B5800075FB812104460A4800F070FB0DB11022C2
:10B59000AA711CB1402222710022627118B14022AE
:10B5A00002710022427143230148338070BD00BF05
:10B5B00008030024FFF7DABF70B5822106460F4862
:10B5C00000F054FB012105460C4800F04FFB81219F
:10B5D00004460A4800F04AFB0DB11022AA711CB1C2
:10B5E000002222710222627118B10022027102222D
:10B5F000427143230148338070BD00BF080300241B
:10B6000038B5D0F8D4320446B03350F823508DB159
:10B6100001F000F8D4F8D432C5F80C0205F5037136
:10B6200004EB8304D5F80402D4F8C432DB689847ED
:10B63000002038BD0320FCE7F8B5D0F8D4620A46F4
:10B64000D0F8C87200EB8606D6F8C05225B301F0D8
:10B650000F0C142404FB0C04A3697BB14FF0240EDF
:10B660000EFB0C77FF69B3FBF7FC07FB1C332BB910
:10B670001A46A36101F016F80020F8BD0023C5F8B2
:10B680001432D6F8C4321B69002BF5D005F50471CD
:10B69000D5F808029847EFE70320EEE7D0F8D43258
:10B6A00000EB8303F7B50022D3F8C06204460D46D1
:10B6B0008DF80520ADF80620002E65D091F800C069
:10B6C0001CF0600229D0202A5AD1CA884F78F2B1E2
:10B6D0001CF0800F0ED0D3F8C432314638469B6838
:10B6E0009847EA883146072A28BF0722204600F0FB
:10B6F00058FD09E0402A314686F8007228BF4022F2
:10B7000086F8012200F062FD002003B0F0BDD3F8FE
:10B71000C43238469B689847F6E74B780B2B2FD8F6
:10B7200001A252F823F000BF59B7000809B700087A
:10B7300081B7000881B7000881B7000881B7000809
:10B7400081B7000881B7000881B7000881B70008F9
:10B7500069B7000879B7000890F89C32032B0FD125
:10B7600002220DF10601C1E790F89C32032B07D1AC
:10B7700001220DF10501B9E790F89C32032BC3D0EB
:10B780002946204600F0E6FC0320BEE738B5044613
:10B790000025812100F062FF01212046258700F06D
:10B7A0005DFF82212046A4F8785100F057FFD4F8BD
:10B7B000D432E56404EB8303D3F8C0228AB1D3F812
:10B7C000C4325B689847D4F8D432B03354F82300BD
:10B7D00000F028FFD4F8D432B03344F82350C4F832
:10B7E000BC52002038BDF8B504464FF4077000F095
:10B7F00015FF054630B9D4F8D432B03344F82300ED
:10B80000022046E04FF40772002100F05DFFD4F8FB
:10B81000D432B03344F82350237CC4F8BC52CBBBA1
:10B820004FF4007381210222204600F00BFF01211A
:10B830004FF4007321870222204600F003FF012607
:10B840001023032282212046A4F84E300823A4F8B6
:10B850007861002700F0F6FED4F8D432A4F84C60EA
:10B8600004EB8303C5F80472D3F8C4321B6898470D
:10B87000D5F80422C5F81472C5F81872002ABFD092
:10B88000237C8BB94FF400733146204600F013FF40
:10B890000020F8BD402381210222204600F0D2FE84
:10B8A000012140232187C6E74023EDE739B1D0F8D5
:10B8B000D43200EB8300C0F8C4120020704703208C
:10B8C0007047D0F8D432B03350F823302BB1002079
:10B8D000C3F80812C3F81022704703207047D0F84D
:10B8E000D432B03350F823301BB10020C3F8041217
:10B8F000704703207047D0F8D432B03350F823207B
:10B9000010B57AB1D2F8144201236CB9C2F81432DE
:10B910008121D2F81032D2F80822C36200F0C2FEB0
:10B92000204610BD0320FCE71846FAE7D0F8D422E1
:10B93000B03250F8222008B562B1037CD2F804225C
:10B9400033B94FF40073012100F0B5FE002008BDAB
:10B950004023F8E70320FAE778B10023C0F8B832B3
:10B96000C0F8C432C0F8D03209B1C0F8B412012313
:10B97000027080F89C3200F00BBE03207047002359
:10B9800013B50446ADF8063081B1CB6AC0F8B812E1
:10B9900023B10DF106009847C4F8D002D4F8D8328C
:10B9A00000200133C4F8D83202B010BD0320FBE7F9
:10B9B00000F03FBED0F8B8320BB11B6818471846EC
:10B9C000704708B5D0F8B8325B689847002818BFB0
:10B9D000032008BD38B500F2AA250446284600F029
:10B9E000AEFB012394F8AA12C4F89432B4F8B03232
:10B9F000C4F8983201F01F03012B08D0022B0CD0A1
:10BA00008BB929462046BDE8384000F04DB929469B
:10BA10002046BDE8384000F0BFBA29462046BDE8C0
:10BA2000384000F0E8BA204601F08001BDE8384017
:10BA300000F01DBE70B50446164609BBD0F894321E
:10BA4000032B0CD1D0E9573293420AD99B1A3146C5
:10BA50009A42C0F85C3128BF1A4600F0C4FB0020AF
:10BA600070BD90F89C32032B06D1D0F8B8321B6918
:10BA700013B1C0F8D4129847204600F0BCFBEEE7A3
:10BA800090F89C32032BEAD1D0F8B8329B69002B96
:10BA9000E5D00022BDE87040C0F8D422184770B548
:10BAA000044616460D4600293DD1D0F89432022BAB
:10BAB0000ED1D0E90732934212D99A1A3146C261A7
:10BAC00000F07CFB2B462A462946204600F0F3FD79
:10BAD00094F8A03213B1002384F8A032002070BD86
:10BAE0000CD18269934209D8D0F898329A4205D293
:10BAF0000A4600F063FBC4F89852E3E794F89C32DE
:10BB0000032B08D1D4F8B832DB6823B100222046D9
:10BB1000C4F8D42298478021204600F0A8FD204692
:10BB200000F074FBD4E790F89C32032BD6D1D0F808
:10BB3000B8325B69002BD1D00022BDE87040C0F85C
:10BB4000D4221847F8B501230021044680F89C321E
:10BB5000D0F8B832C0F894124160C0F8A41280F84E
:10BB6000A012B3B900260022402501274023114628
:10BB7000204600F067FD2B46002280212046A4F8D5
:10BB80006471C4F8605100F05DFD3046A784256201
:10BB9000F8BD5B68002BE5D098470028E2D003266B
:10BBA000E1E701740020704790F89C32042B04D028
:10BBB00090F89C32DBB280F89D32042380F89C32EE
:10BBC0000020704790F89C32042B04D190F89D32ED
:10BBD000DBB280F89C320020704708B590F89C22B8
:10BBE000032A05D1D0F8B83213B1DB6903B1984705
:10BBF000002008BDD0F8D422AE3250F8222008B57B
:10BC00004AB190F89C32032B01D1136A0BB9002082
:10BC100008BD9847FBE70320FAE7D0F8D422AE32FC
:10BC200050F8222008B54AB190F89C32032B01D17C
:10BC3000536A0BB9002008BD9847FBE70320FAE7D9
:10BC400000207047012208B580F89C22D0F8B82265
:10BC50000AB9002008BD5268017990470028F8D041
:10BC60000320F7E7002070470020704710B5428896
:10BC700003789A4201D8002010BD04782044234460
:10BC800044789BB2052CF4D184788C42F1D1F3E74F
:10BC900010B50446802100F0EAFC00212046BDE8F2
:10BCA000104000F0E4BC000073B50B7804460D466C
:10BCB00003F06003202B09D0402B07D093B120461E
:10BCC000FFF7E6FF0025284602B070BDD4F8D43255
:10BCD00029462046AE3354F823309B6802B0BDE8B5
:10BCE000704018474B78092BE9D801A252F823F08D
:10BCF00039BF00087DBF0008BFBC000861BF000855
:10BD0000BFBC000833BE000819BD0008BFBC000856
:10BD10000DBF000875BE00080023ADF806304B8843
:10BD20001A0A013A0E2ACAD801A151F822F000BF1E
:10BD300077BD0008A9BD0008C3BD0008BFBC00084E
:10BD4000BFBC000805BE00081BBE0008BFBC000841
:10BD5000BFBC0008BFBC0008BFBC0008BFBC0008D7
:10BD6000BFBC0008BFBC00086DBD0008D0F8B432ED
:10BD7000DB691BB9A3E7D0F8B4321B680DF10601EB
:10BD8000207C9847EA88002A00F0A380BDF806309E
:10BD9000002B94D09A42014628BF1A46ADF80620DF
:10BDA000204600F0FEF98DE7027CD0F8B83232B9B7
:10BDB0009B6A0DF10600984702234370E2E7DB6AB5
:10BDC000F7E7DBB2052B3FF67AAFDFE803F00307B6
:10BDD0000B0F1317D0F8B4325B68CAE7D0F8B4324F
:10BDE0009B68C6E7D0F8B432DB68C2E7D0F8B4325B
:10BDF0001B69BEE7D0F8B4325B69BAE7D0F8B43259
:10BE00009B69B6E7037C002B7FF459AFD0F8B832BA
:10BE10000DF106005B6B9847B4E7037C002B7FF4C1
:10BE20004EAFD0F8B8320DF106001B6B98470723D0
:10BE3000C3E78B88002B7FF442AFCB88002B7FF4C5
:10BE40003EAF4D887F2D3FF63AAF90F89C32032BE2
:10BE50003FF435AFEDB2294680F89E5200F019FC50
:10BE6000204600F0C8F91DB1022384F89C3229E76E
:10BE70000123FAE78978474D0129297003D9FFF793
:10BE800007FF03251FE790F89C32022BDEB208D093
:10BE9000032E17D0FFF7FCFE29782046FFF791FD0F
:10BEA000EFE7B1B101214160FFF784FD054620466F
:10BEB00025B1FFF7EDFE84F89C6204E700F09BF9E2
:10BEC0000323D2E749B90223416080F89C32FFF78F
:10BED00078FD204600F08FF9F4E641680129F8D09A
:10BEE000C9B2FFF76EFD297820466160FFF762FD59
:10BEF00005460028EDD02046FFF7CAFE21792046EE
:10BF0000FFF75FFD022384F89C32DCE6CA88012A31
:10BF10007FF4D5AE90F89C120229CBB207D8002B43
:10BF20003FF4CDAE0146002341F8083F38E7032B2C
:10BF30007FF4C5AE011D33E790F89C32013B022B24
:10BF40003FF6BDAECA88022A7FF4B9AED0F8A4325B
:10BF50000146002B0CBF0123032341F80C3F1FE7D0
:10BF60004B88012B02D1C4F8A432B2E7022B7FF434
:10BF7000A6AE8B881B0A80F8A032AAE790F89C3204
:10BF8000013B022B3FF69BAE4B88012B7FF49AAE10
:10BF90000023E8E7884C002470B50B7804460E4671
:10BFA00003F060025B0601D5402A1FD194F89C3251
:10BFB000013B022B1AD831792046012917D8FFF707
:10BFC00051FE88B9D4F8B8329B686BB1C4F8D4027A
:10BFD0003146204698470546F3881BB915B92046D7
:10BFE00000F009F9284670BD0325F5E72046002535
:10BFF000FFF74EFEF6E770B50B7804460E468A88CA
:10C0000003F060030D79202B59D0402B57D01BB182
:10C010002046FFF73DFE3EE04B78012B3DD0032B41
:10C0200026D0002BF4D190F89C32022BD9B262D0EA
:10C030000329EDD105F00F0312F0800F4FF0140229
:10C0400002FB030368D09B8C002BE1D005F07F0638
:10C05000802D06F1010606EB860600EB860667D00A
:10C060002946204600F0C4FA002866D0012360E08B
:10C0700090F89C32022BDAB233D0032AC8D14B8815
:10C0800033B9690604D0F38813B9294600F0EFFAF2
:10C09000204600F0B0F8002070BD90F89C32022BD2
:10C0A000DAB21ED0032AB3D14B88002BF3D16B0632
:10C0B00002D0294600F0E4FA204600F09CF8294618
:10C0C0002046FFF7D1FD0028E5D1D4F8B832C4F8F6
:10C0D000D4029B68002BDED031462046BDE870407C
:10C0E00018476A0694D0294600F0C1FA80212046FC
:10C0F00000F0BDFACFE769068AD113064FF00003BE
:10C100004FF002024CBF00F1140100F5AA710B6060
:10C11000204600F046F8BEE7B3F86431002B3FF448
:10C1200077AF142606FB050606F5AA76002D97D1F3
:10C130000023336002223146EAE73060FAE70B78E9
:10C1400003704B7843704B8843808B888380CB8807
:10C15000C380704710B50446802100F088FA0021A2
:10C160002046BDE8104000F082BA70B50D46164674
:10C17000044670B1F4F7BCF8013CC3B200210133AE
:10C180005B0033802B7003236B70022314F8012FA4
:10C1900002B970BDEA545A1C0233D2B2DBB2A954C0
:10C1A000F4E71346022210B5C0F894220A46002193
:10C1B000C0E9063300F076FA002010BD08B513463A
:10C1C0000A46002100F06EFA002008BD1346032243
:10C1D00010B5C0F894220A460021C0E9563300F099
:10C1E0006AFA002010BD08B513460A46002100F087
:10C1F00062FA002008BD08B504220023C0F894228A
:10C2000019461A4600F04EFA002008BD08B505226E
:10C210000023C0F8942219461A4600F04CFA002078
:10C2200008BD000008B501220E490F48FFF794FB36
:10C2300008B1F4F719FF0D490B48FFF7A0FB08B14F
:10C24000F4F712FF0A490848FFF730FB08B1F4F78A
:10C250000BFF0548FFF7ACFB18B1BDE80840F4F749
:10C2600003BF08BDD80300248C4C00244C030024D9
:10C27000900300240020704738B50446074D0A6833
:10C2800001460020F5F7CEFE21462846FFF727FBA2
:10C290002846FFF74BFB002038BD00BF8C4C002424
:10C2A00010B5064C002206492046FFF70AFB054957
:10C2B0002046FFF714FB002010BD00BF8C4C00246B
:10C2C000684F002468570024222808B504D10022B2
:10C2D00002201146F5F7A6FE002008BD012A08B588
:10C2E0000346104603D10A681946F5F79BFE002065
:10C2F00008BD000010B5094C0A46D4F8BC32D3F88A
:10C30000143243B901462046FFF7DBFA2046BDE868
:10C310001040FFF7F0BA012010BD00BF8C4C002484
:10C32000122301480B807047C403002404230148F2
:10C330000B807047C0030024002370B54D1C1E46BF
:10C34000040FB0F1204F4FEA001034BF30343734BF
:10C3500001F8134005F813600133DCB2A242EFD8B4
:10C3600070BD00001A2310B50B800A4BD3F80008EB
:10C37000D3F8082880180AD0D3F8044808220649C0
:10C38000FFF7DAFF042210312046FFF7D5FF0348FC
:10C3900010BD00BF00F0FF08A6030024A403002482
:10C3A00010B5044C0A4604482146FFF7DEFE20463D
:10C3B00010BD00BF685F0024B5DA000810B5044C5A
:10C3C0000A4604482146FFF7D0FE204610BD00BFB4
:10C3D000685F0024C0DA000810B5044C0A4604481F
:10C3E0002146FFF7C2FE204610BD00BF685F002453
:10C3F000CDDA000810B5044C0A4604482146FFF780
:10C40000B4FE204610BD00BF685F0024D8DA0008E3
:10C4100030B5ABB004461422002104A800F054F952
:10C420008422002109A800F04FF92268204B9A428B
:10C430003BD14FF0804309A80993FBF725FD08B1D4
:10C44000F4F712FE1B4CFAF76BFE002504A9D4F892
:10C450004031194843F48053C4F84031D4F8403196
:10C4600006950193019B4FF48073CDE90435F8F7ED
:10C470008BFCD4F838315B202A4643F00073294600
:10C48000C4F83831D4F838310293029BD4F83831EB
:10C4900043F08063C4F83831D4F838310393039BF8
:10C4A000F7F752FD5B20F7F781FD2BB030BD00BFE1
:10C4B00000000440004402580030025800F29C4141
:10C4C000D0F8E004FFF786BA242303FB0103D0F879
:10C4D000E004D3F86022FFF7ADBA242303FB010385
:10C4E000D0F8E0041A6AFFF7DABAD0F8E004FFF7F0
:10C4F00074BB10B5C179044621B1022901D0F4F70B
:10C50000B3FD0121D4F8E004FFF74BFBD4F8E004BD
:10C51000BDE81040FFF716BB10B50446D0F8E004A4
:10C52000FFF742FBE37A33B1F7F7EEFC024A1369F7
:10C5300043F00603136110BD00ED00E010B5C37AAF
:10C54000044633B1F7F7E7FC084A136923F0060302
:10C5500013612268D4F8E004D2F8003E23F001030E
:10C56000BDE81040C2F8003EFFF72CBB00ED00E034
:10C57000D0F8E004FFF751BBD0F8E004FFF73ABB76
:10C58000D0F8E004FFF75CBBD0F8E004FFF75ABB3B
:10C5900008B502780346012A23D11348C0F8E034D5
:10C5A000C3F8C802114BC28003600923C281037122
:10C5B00003234372002343810373F9F7F7FF08B1A4
:10C5C000F4F752FD4FF400710748FAF740FD40229E
:10C5D00000210548FAF71CFD802201210248FAF7E4
:10C5E00017FD002008BD00BF886300240000044040
:10C5F00011F0800FD0F8C8324FF0240217BF01F0BD
:10C600007F0102FB013302FB0133987D08BF93F8E1
:10C6100056027047D0F8C802FAF7F3B800487047DE
:10C6200068610024704718B102280CBF0120032064
:10C63000704708B5D0F8C802FAF72EF8BDE80840F0
:10C64000FFF7F1BF10B51446D0F8C8021A462346CA
:10C65000FAF754F8BDE81040FFF7E5BF08B5D0F889
:10C66000C802FAF782F8BDE80840FFF7DCBF08B55A
:10C67000D0F8C802FAF7E7F8BDE80840FFF7D3BFE3
:10C6800008B5D0F8C802FAF715F9BDE80840FFF779
:10C69000CABF08B5D0F8C802FAF71DF8BDE80840CF
:10C6A000FFF7C1BF08B5D0F8C802FAF7B2F8BDE885
:10C6B0000840FFF7B8BF08B5D0F8C802FAF783F80A
:10C6C000BDE80840FFF7AFBF02440346934200D1E4
:10C6D000704703F8011BF9E770B50D4D0D4C641B55
:10C6E000A4100026A64209D10B4D0C4C00F02EF8E8
:10C6F000641BA4100026A64205D170BD55F8043B6A
:10C7000098470136EEE755F8043B98470136F2E7C3
:10C7100048DB000848DB000848DB00084CDB000869
:10C72000034611F8012B03F8012B002AF9D17047B9
:10C730000A44914200F1FF3300D1704710B511F85F
:10C74000014B03F8014F9142F9D110BDF8B500BF7C
:10C75000F8BC08BC9E467047F8B500BFF8BC08BCE2
:04C760009E4670473A
:10C76400ED008C000AD7A33B00000000000000008D
:10C7740000000000CDCCCC3D0000003FCDCC4C3EB1
:10C78400CDCC4C3D000005800F800A001B801E00AC
:10C7940014001180338036003C00398028002D803D
:10C7A40027802200638066006C00698078007D80A9
:10C7B40077807200500055805F805A004B804E0095
:10C7C40044004180C380C600CC00C980D800DD800D
:10C7D400D780D200F000F580FF80FA00EB80EE00F5
:10C7E400E400E180A000A580AF80AA00BB80BE0069
:10C7F400B400B180938096009C00998088008D805D
:10C8040087808200838186018C01898198019D81C2
:10C8140097819201B001B581BF81BA01AB81AE01AC
:10C82400A401A181E001E581EF81EA01FB81FE0120
:10C83400F401F181D381D601DC01D981C801CD8114
:10C84400C781C201400145814F814A015B815E017C
:10C8540054015181738176017C01798168016D8174
:10C8640067816201238126012C01298138013D81E0
:10C8740037813201100115811F811A010B810E01CC
:10C8840004010181038306030C03098318031D8338
:10C8940017831203300335833F833A032B832E031C
:10C8A40024032183600365836F836A037B837E0390
:10C8B40074037183538356035C03598348034D8384
:10C8C40047834203C003C583CF83CA03DB83DE03EC
:10C8D400D403D183F383F603FC03F983E803ED83E4
:10C8E400E783E203A383A603AC03A983B803BD8350
:10C8F400B783B203900395839F839A038B838E033C
:10C9040084038183800285828F828A029B829E02B5
:10C9140094029182B382B602BC02B982A802AD82AB
:10C92400A782A202E382E602EC02E982F802FD8217
:10C93400F782F202D002D582DF82DA02CB82CE0203
:10C94400C402C182438246024C02498258025D827B
:10C9540057825202700275827F827A026B826E0263
:10C9640064026182200225822F822A023B823E02D7
:10C9740034023182138216021C02198208020D82CB
:10C98400078202025B25396C755D205B4144435F7D
:10C994004D414E41474552204552524F525D20571A
:10C9A400726974696E6720746F2062756666657259
:10C9B400207768696C652072656164696E672120FF
:10C9C4000D0A005B25396C755D205B4144435F4D66
:10C9D400414E41474552204552524F525D205472B8
:10C9E40079696E6720746F2072656164206D6F725F
:10C9F400652073616D706C6573207468616E20616D
:10CA0400726520617661696C61626C65200D0A0053
:10CA14005B25396C755D205B4144435F4D414E415C
:10CA2400474552204552524F525D2053504920658C
:10CA340072726F722C20636F64653A2025642C2017
:10CA440073746174653A2025642C20646D61727876
:10CA54002073746174653A2025640D0A005B2539DE
:10CA64006C755D205B4144435F4D414E41474552E7
:10CA7400204552524F525D20496E76616C696420A4
:10CA840053616D706C6520526174652025640D0AD4
:10CA9400005B25396C755D205B4144435F4D414E1D
:10CAA40041474552204552524F525D20444D41204A
:10CAB4006E6F742072656164792E2053746174659D
:10CAC4003A2025640D0A005B25396C755D205B41B5
:10CAD40044435F4D414E41474552204552524F52C7
:10CAE4005D2053504920444D412073746172742079
:10CAF4006661696C65642E204572726F723A2025F6
:10CB0400642C20535049204572726F723A20256478
:10CB14002C20444D41204572726F723A2025640DD9
:10CB24000A005B25396C755D205B524547495354B7
:10CB3400455253204552524F525D20496E76616CE6
:10CB4400696420656E756D2076616C756520256459
:10CB540020666F722072656769737465722030781D
:10CB640025580D0A005B25396C755D205B524547DD
:10CB7400495354455253204552524F525D20496EF9
:10CB840076616C696420617474656D707420746F6F
:10CB940020777269746520746F2072656164206FF8
:10CBA4006E6C7920726567697374657220307825BC
:10CBB400580D0A005B25396C755D205B5245474969
:10CBC4005354455253204552524F525D20556E6B7B
:10CBD4006E6F776E207265676973746572207479FD
:10CBE400706520666F722072656769737465722060
:10CBF400307825580D0A005B25396C755D205B5231
:10CC04004547495354455253204552524F525D2093
:10CC14005265676973746572205570646174652C1C
:10CC2400205265673A307825582C2056616C3A2595
:10CC34006420307825580D0A004552524F523A204C
:10CC44004D616C666F726D656420747270735F659C
:10CC540076745F7573625F72656365697665204596
:10CC640056542C206461746120706F696E7465720F
:10CC7400203D202030782558206C656E677468202C
:10CC84003D2025640A004552524F523A20545250D6
:10CC94005320455654202564204E6F742048616EFD
:10CCA400646C65640A005B25396C755D205B5553C3
:10CCB40042204552524F525D20496E76616C696440
:10CCC400207573625F73656E645F73616D706C650C
:10CCD4007320706172616D657465720D0A005B2565
:10CCE400396C755D205B555342204552524F525D5D
:10CCF40020496E76616C6964207573625F73656E3A
:10CD0400645F73616D706C6573206C656E677468C5
:10CD14000D0A005B25396C755D205B44594E414D0D
:10CD24004958454C204552524F525D2043616E6E26
:10CD34006F742073656E6420696E737472756374A6
:10CD4400696F6E3A20436F6D6D756E6963617469C6
:10CD54006F6E206E6F742072656164790A005B25C2
:10CD6400396C755D205B44594E414D4958454C2002
:10CD74004552524F525D204661696C656420746F60
:10CD840020737461727420444D41207472616E7317
:10CD94006D697373696F6E0A005B25396C755D206C
:10CDA4005B44594E414D4958454C204552524F52CF
:10CDB4005D204661696C656420746F2073746172D0
:10CDC4007420444D41206865616465722072780A5C
:10CDD400005B25396C755D205B44594E414D4958C3
:10CDE400454C204552524F525D204661696C656442
:10CDF40020746F20737461727420444D41207265F5
:10CE040063657074696F6E20666F72207061636B06
:10CE1400657420626F64790A005B25396C755D2046
:10CE24005B44594E414D4958454C204552524F524E
:10CE34005D20435243206D69736D617463680A0019
:10CE44005B25396C755D205B4C45414B5F44455413
:10CE54004543544F5220494E464F5D2053746174EC
:10CE640065206368616E67656420746F2025730DA7
:10CE74000A005B25396C755D205B4C45414B5F4472
:10CE840045544543544F5220494E464F5D204C650E
:10CE9400616B2064657465637465643A2025730D61
:10CEA4000A004C45414B5F53544154455F484F4C35
:10CEB40044004C45414B5F53544154455F545241E7
:10CEC4004E534954494F4E004C45414B5F535441D6
:10CED40054455F534554544C45004C45414B5F53B6
:10CEE400544154455F4C45414B004C45414B5F4ECA
:10CEF4004F5F4C45414B004C45414B5F5452414EB2
:10CF0400534954494F4E5F50524553535552455F10
:10CF140044524F50004C45414B5F5052455353557A
:10CF240052455F44524F505F4D414A4F52004C4569
:10CF3400414B5F50524553535552455F4445564902
:10CF44004154494F4E004C45414B5F44524946546D
:10CF5400004C45414B5F4450445831004C45414BD3
:10CF64005F4450445832005B25396C755D205B503A
:10CF74004C554E474552204552524F525D20536501
:10CF840072766F206861726477617265206572726F
:10CF94006F720D0A005B25396C755D205B504C5532
:10CFA4004E474552204552524F525D204661696CAE
:10CFB400656420746F20696E697469616C697A654F
:10CFC40020736572766F0D0A005B25396C755D20E0
:10CFD4005B50524553535552455F434F4E54524F45
:10CFE4004C4C4552204552524F525D204661696C6B
:10CFF400656420746F20696E697469616C697A650F
:10D0040020706C756E67657220636F6E74726F6CDE
:10D014006C65723A2025640D0A005B25396C755DD8
:10D02400205B50524553535552455F434F4E545223
:10D034004F4C4C4552204552524F525D2046616937
:10D044006C656420746F20696E697469616C697AB7
:10D05400652070726573737572652073656E736F86
:10D06400723A2025640D0A005B25396C755D205BDE
:10D0740050524553535552455F434F4E54524F4CB3
:10D084004C4552204552524F525D204661696C65B1
:10D094006420746F20696E697469616C697A6520B3
:10D0A40074656D70657261747572652073656E73F5
:10D0B4006F723A2025640D0A005B25396C755D207A
:10D0C4005B50524553535552455F434F4E54524F54
:10D0D4004C4C4552204552524F525D20507265735C
:10D0E4007375726520636F6E74726F6C6C657220F9
:10D0F4006E6F7420696E697469616C697A65640D18
:10D104000A005B25396C755D205B505245535355BD
:10D1140052455F434F4E54524F4C4C45522045525A
:10D12400524F525D20496E76616C696420636F6E64
:10D1340066696720706172616D657465720D0A00BD
:10D144005B25396C755D205B5052455353555245F0
:10D154005F434F4E54524F4C4C4552204552524F10
:10D16400525D204C65616B2064657465637465640D
:10D1740021204D6F76696E6720686F6D650D0A001A
:10D184005B25396C755D205B5052455353555245B0
:10D194005F434F4E54524F4C4C4552204552524FD0
:10D1A400525D204661696C656420746F20737461FC
:10D1B400727420706C756E6765722063616C69624D
:10D1C400726174696F6E3A2025640D0A005B25391B
:10D1D4006C755D205B50524553535552455F434F28
:10D1E4004E54524F4C4C4552204552524F525D20A2
:10D1F4004661696C656420746F2072656164207097
:10D20400726573737572652073656E736F723A20FD
:10D2140025640D0A005B25396C755D205B50524511
:10D2240053535552455F434F4E54524F4C4C455205
:10D23400204552524F525D204661696C65642074EA
:10D244006F20726561642074656D706572617475B8
:10D2540072652073656E736F723A2025640D0A003F
:10D264005B25396C755D205B5052455353555245CF
:10D274005F434F4E54524F4C4C4552204552524FEF
:10D28400525D204661696C656420746F2073657417
:10D2940020706C756E6765722050574D3A20256476
:10D2A4000D0A005B25396C755D205B505245535364
:10D2B4005552455F434F4E54524F4C4C45522045B6
:10D2C40052524F525D2050726573737572652063BC
:10D2D4006F6E74726F6C6C6572206E6F7720696EFE
:10D2E400206572726F72206D6F64650D0A005B2594
:10D2F400396C755D205B50524553535552455F431D
:10D304004F4E54524F4C4C4552204552524F525D51
:10D3140020507265737375726520636F6E74726FDB
:10D324006C6C6572206E6F7720696E20756E6B6E03
:10D334006F776E206D6F64650D0A005B25396C751F
:10D344005D205B50524553535552455F434F4E54F5
:10D35400524F4C4C4552204552524F525D20507210
:10D3640065737375726520636F6E74726F6C6C6530
:10D374007220706C756E676572206C696D697420BB
:10D384006578636565646564212052657475726EA1
:10D39400696E6720686F6D650D0A005B25396C75D1
:10D3A4005D205B50524553535552455F434F4E5495
:10D3B400524F4C4C4552204552524F525D204661CB
:10D3C400696C656420746F20737461727420746571
:10D3D4006D70657261747572652072656164696EE1
:10D3E400670D0A005B25396C755D205B505245530F
:10D3F400535552455F434F4E54524F4C4C45522067
:10D404004552524F525D2054656D7065726174755A
:10D4140072652073656E736F72206572726F72200D
:10D42400647572696E6720726561640D0A005B251C
:10D43400396C755D205B50524553535552455F43DB
:10D444004F4E54524F4C4C4552204552524F525D10
:10D45400204661696C656420746F20737461727412
:10D464002070726573737572652072656164696E8C
:10D47400670D0A005B25396C755D205B505245537E
:10D48400535552455F434F4E54524F4C4C455220D6
:10D494004552524F525D2050726573737572652008
:10D4A40073656E736F72206572726F722064757229
:10D4B400696E6720726561640D0A005B25396C75BD
:10D4C4005D205B50524553535552455F434F4E5474
:10D4D400524F4C4C4552204552524F525D20496E9A
:10D4E40076616C696420706172616D6574657273D4
:10D4F40020666F72206765745F73746174650D0ACA
:10D50400005B25396C755D205B5052455353555271
:10D51400455F434F4E54524F4C4C45522045525256
:10D524004F525D20507265737375726520636F6E20
:10D5340074726F6C6C657220636F6E74726F6C20A2
:10D544007570646174652066756E6374696F6E20AE
:10D5540063616C6C65642077697468204E554C4C2B
:10D5640020636F6E746578740D0A005B25396C75E1
:10D574005D205B50524553535552455F53454E53BE
:10D584004F52204552524F525D20496E76616C696C
:10D594006420686172647761726520636F6E666986
:10D5A4006775726174696F6E0D0A005B25396C755D
:10D5B4005D205B50524553535552455F53454E537E
:10D5C4004F52204552524F525D204465766963653F
:10D5D400206E6F7420726573706F6E64696E67215C
:10D5E400205374617475733A2025640D0A005B2519
:10D5F400396C755D205B50524553535552455F530A
:10D60400454E534F52204552524F525D2046616958
:10D614006C656420746F20737461727420444D418E
:10D62400207265616421205374617475733A2025F6
:10D63400640D0A005B25396C755D205B50524553BF
:10D64400535552455F53454E534F52204552524F06
:10D65400525D2053656E736F7220737461747573B9
:10D664002062697473206572726F723A2025640DAA
:10D674000A005B25396C755D205B534552564F207B
:10D684004552524F525D20556E6B6E6F776E20611E
:10D6940064647265737320256420696E2064796EF6
:10D6A400616D6978656C20726573706F6E73652047
:10D6B40068616E646C65720D0A005B25396C755D7A
:10D6C400205B534552564F204552524F525D2047DE
:10D6D4006F7420616E20756E65787065637465641F
:10D6E4002064796E616D6978656C20726573706F02
:10D6F4006E736520286C61737420636F6D6D616E49
:10D704006420776173202564290D0A005B25396C38
:10D71400755D205B534552564F204552524F525D22
:10D72400204661696C656420746F2067657420729B
:10D734006573706F6E73653A2025640D0A005B256E
:10D74400396C755D205B534552564F204552524FFC
:10D75400525D20556E6B6E6F776E20736572766FB7
:10D764002073746174653A2025640D0A005B2539C1
:10D774006C755D205B534552564F204552524F52B3
:10D784005D20536572766F206F7065726174696F86
:10D794006E2074696D6564206F75742E20526573F4
:10D7A400656E64696E67206C61737420636F6D6D60
:10D7B400616E642E0D0A005B25396C755D205B5328
:10D7C4004552564F204552524F525D205365727652
:10D7D4006F206E6F7420696E697469616C697A6513
:10D7E400640D0A005B25396C755D205B5345525608
:10D7F4004F204552524F525D20536572766F20621E
:10D804007573790D0A005B25396C755D205B534592
:10D8140052564F204552524F525D2044796E616DED
:10D824006978656C20636F6D6D616E6420666169F3
:10D834006C65643A2025640D0A005B25396C755DBE
:10D84400205B534552564F204552524F525D20465D
:10D8540061696C656420746F20696E697469616CB8
:10D86400697A652044796E616D6978656C20696EAA
:10D87400746572666163650D0A005B25396C755DBC
:10D88400205B54454D50455241545552455F5345D4
:10D894004E534F52204552524F525D20496E76618D
:10D8A4006C696420686172647761726520636F6E6D
:10D8B40066696775726174696F6E0D0A005B25395C
:10D8C4006C755D205B54454D50455241545552454D
:10D8D4005F53454E534F52204552524F525D2044A0
:10D8E4006576696365206E6F7420726573706F6E00
:10D8F40064696E6721205374617475733A202564DA
:10D904000D0A005B25396C755D205B54454D50450F
:10D914005241545552455F53454E534F5220455240
:10D92400524F525D204661696C656420746F2063B8
:10D934006F6E6669677572652064657669636521D3
:10D94400205374617475733A2025640D0A005B25B5
:10D95400396C755D205B54454D50455241545552C8
:10D96400455F53454E534F52204552524F525D200E
:10D974004661696C656420746F20766572696679A6
:10D9840020636F6E66696775726174696F6E2120BA
:10D994005374617475733A2025640D0A005B25394C
:10D9A4006C755D205B54454D50455241545552456C
:10D9B4005F53454E534F52204552524F525D2043C0
:10D9C4006F6E66696775726174696F6E206D6973D5
:10D9D4006D6174636821205365743A203078253072
:10D9E40034582C20526561643A20307825303458FC
:10D9F40020286D61736B6564290D0A005B25396C01
:10DA0400755D205B54454D50455241545552455F18
:10DA140053454E534F52204552524F525D2046615A
:10DA2400696C656420746F2073657420726567691E
:10DA34007374657220706F696E74657221205374FB
:10DA4400617475733A2025640D0A005B25396C7581
:10DA54005D205B54454D50455241545552455F53EA
:10DA6400454E534F52204552524F525D20466169F4
:10DA74006C656420746F20737461727420444D412A
:10DA8400207265616421205374617475733A202592
:10DA9400640D0A005465726D696E616C00525454D1
:10DAA400005345474745520001020304060708098D
:10DAB40000545250532047656E203200497A6F6EED
:10DAC40020536369656E63650043444320436F6E6E
:10DAD4006669670043444320496E746572666163F6
:10DAE4006500080402001400C8007D00FA00F40177
:10DAF400E803000001000200030004000500060022
:10DB04000000010030313233343536373839414280
:10DB140043444546010002000400060008000A00D0
:10DB24000C001000200040008000000108040204E2
:0CDB3400080101010101010307010000CC
:08DB4000B027FF7F0100000087
:04DB4800D5020008FA
:04DB4C00B10200081A
:10DB50000090D003FFFF0000100000241000000020
:10DB6000400000000000000018020024EEDA000867
:10DB70000400000001010000F1070008000000009F
:10DB800042000000000000001A02002404DB00082C
:10DB90000200000001010000000000000000000081
:10DBA00053000000000000001C020024F6DA000808
:10DBB0000700000001010000E131000834020024E8
:10DBC00048000000000000001E020024EADA0008FD
:10DBD0000200000001010000991A00080000000086
:10DBE000430030F8D00700002002002400000000AD
:10DBF0000000000000010000F5090008000000001E
:10DC00004500D08A30750000240200240000000086
:10DC10000000000000010000791A00080000000068
:10DC20004E0000000100000030020024000000004F
:10DC30000000000000010000B51A0008000000000C
:10DC40004400000000000000220200240000000048
:10DC500000000000020000000000000000000000C2
:10DC600049000000000000002A020024000000001B
:10DC700000000000020000000000000000000000A2
:10DC80004A000000000000002C02002400000000F8
:10DC90000000000002000000000000000000000082
:10DCA0004D000000000000002E02002400000000D3
:10DCB0000000000002000000000000000000000062
:10DCC0004C000000000000002802002400000000BA
:10DCD0000000000002000000000000000000000042
:10DCE0004B0000000000000026020024000000009D
:10DCF0000000000002000000000000000000000022
:10DD000050000000FF7F00003402002400000000EB
:10DD10000000000000010000000000000000000002
:10DD200051000000FF7F00003602002400000000C8
:10DD300000000000000100000000000000000000E2
:10DD400052000000FF7F00003802002400000000A5
:10DD500000000000000100000000000000000000C2
:10DD6000B0280024130000007D0000000000C8005F
:10DD7000000000000000000000000100060000009C
:10DD8000000000000F000A0008000100902A002493
:10DD90000000000000000000000000000200000081
:10DDA00004000000982A0024000000000000000089
:10DDB000000000001400000004000000E82A002415
:10DDC00000000000E832002400000000E83A0024CF
:10DDD00000000000A6CE0008B6CE0008CCCE000899
:10DDE000DECE0008EECE0008FBCE000819CF0008FA
:10DDF00032CF00084ACF000855CF000860CF000896
:10DE00000030025801000000000000000000000087
:10DE10000030025802000000000000000000000076
:10DE200000000000000000000000000000000000F2
:10DE300000000000010000000000000000000000E1
:10DE400001000000000000000000000001000000D0
:10DE5000010000001000000009024300020100C0A0
:10DE6000320904000001020201000524001001052E
:10DE70002401000104240202052406000107058292
:10DE80000308001009040100020A00000007050150
:10DE9000024000000705810240000000E7B70008CB
:10DEA0008DB700089DB600080000000029B50008E5
:10DEB00039B6000801B600080000000000000000AC
:10DEC00000000000B9B500086DB50008B5B5000840
:10DED00061B500080A0600020000004001000000D1
:10DEE000A1C2000875C20008C9C2000879C20008B2
:10DEF000DDC200081A03000000000000000000005E
:10DF00000000000000000000000000000000000011
:10DF10000403090412010002020200408304405776
:10DF2000000201020301000021C300082DC3000804
:10DF3000BDC30008A1C3000865C30008D9C3000819
:08DF4000F5C300080000000019
:04000005080038DDDA
:00000001FF
